:020000040800F2
:1000000000040020A51F0008F71F0008F71F0008C4
:10001000F71F0008F71F0008F71F00080000000086
:10002000000000000000000000000000F71F0008B2
:10003000F71F000800000000F71F00081109020860
:100040009D0A02089F0A0208A10A0208A50A0208DE
:10005000C50A0208C70A0208C90A0208ED0A02080E
:10006000110B0208350B0208590B02087D0B020820
:100070007F0B0208810B0208830B0208850B020824
:10008000870B0208890B02088B0B0208F71F000878
:10009000F71F0008F71F0008F71F00088D0B020864
:1000A000D90B0208DB0B0208DD0B0208DF0B02088C
:1000B000E10B0208E50B0208110C0208810C020892
:1000C000830C0208850C0208870C0208890C0208C0
:1000D0008D0C0208FD0D0208250D0208C10E020854
:1000E0007D0F020841100208431002084510020863
:1000F00049100208B1100208B3100208B510020836
:10010000B7100208B9100208BB100208BD1002089F
:10011000C1100208951102089711020899110208EE
:10012000A5120208A7120208A9120208AB120208BF
:1001300000000000000000000000000000000000BF
:1001400000000000000000000000000000000000AF
:10015000000000000000000000000000000000009F
:10016000000000000000000000000000000000008F
:10017000000000000000000000000000000000007F
:10018000000000000000000000000000000000006F
:10019000000000000000000000000000000000005F
:1001A000000000000000000000000000000000004F
:1001B000000000000000000000000000000000003F
:1001C000000000000000000000000000000000002F
:1001D000000000000000000000000000000000001F
:0401E0005FF8E0F1F3
:1001E800032A70B404460D4626D941EA000313F0E9
:1001F800030F13D020782B78984208BF294606D0E1
:100208001EE014F8010F11F8013F984218D1012A95
:1002180002F1FF32F5D1002070BC70470B4604464E
:1002280051F8045B50F8046BAE4204D1043A04461A
:10023800032A0B46F2D81D461046002ADAD1EBE70E
:10024800C01AE9E7032A2DE9F00109D82AB10023E9
:10025800CC5CC45401339342FAD1BDE8F001704735
:100268000B468218014603E02478013301F8014B5C
:1002780011F0030F1C46F7D113F003055DD06E4251
:10028800C5F1040CED009B594FEACC0C08E004348E
:10029800A7593B4607FA0CF748EA070741F8047BD9
:1002A800571A23FA05F8032FF1DC03E014F8013B91
:1002B80001F8013B8A42F9D8CFE753F8404C41F89E
:1002C800404C53F83C4C41F83C4C53F8384C41F8FE
:1002D800384C53F8344C41F8344C53F8304C41F80E
:1002E800304C53F82C4C41F82C4C53F8284C41F81E
:1002F800284C53F8244C41F8244C53F8204C41F82E
:10030800204C53F81C4C41F81C4C53F8184C41F83D
:10031800184C53F8144C41F8144C53F8104C41F84D
:10032800104C53F80C4C41F80C4C53F8084C41F85D
:10033800084C53F8044C41F8044C561A1D460C4618
:10034800403340313F2EB8DC2B460FE053F8101CE9
:1003580044F8101C53F80C1C44F80C1C53F8081CE7
:1003680044F8081C53F8041C44F8041C161B2146C6
:100378001D46103410330F2EE8DC2B4602E02468AB
:1003880041F8044B551A1C46032D03F10403F6DC0F
:1003980090E700BF032AC9B270B408D82AB103464F
:1003A800121803F8011B9342FBD170BC70478218E6
:1003B800044601E004F8011B14F0030FFAD14FF0D2
:1003C800013303FB01F31FE044F8403C44F83C3C94
:1003D80044F8383C44F8343C44F8303C44F82C3C6D
:1003E80044F8283C44F8243C44F8203C44F81C3C9D
:1003F80044F8183C44F8143C44F8103C44F80C3CCD
:1004080044F8083C44F8043C161B254640343F2E6B
:10041800DADC2C4607E044F8103C44F80C3C44F87D
:10042800083C44F8043C161B254610340F2EF2DC19
:1004380001E045F8043B541B032CFADC01E005F805
:10044800011B9542FBD3B0E710F0030F38B5044603
:1004580012D10368A3F1013222EA030313F0803FAB
:100468000AD1031D184653F8042BA2F1013525EAD9
:10047800020212F0803FF5D003782BB1431C1846D6
:1004880013F8012B002AFAD100F076F9204638BD7E
:10049800C9B2F0B4002950D010F0030F10D003787F
:1004A800002B79D0994246D0431C05E013F8012B64
:1004B800002A3FD091423ED013F0030F1846F5D1E1
:1004C800036841EA01270646A3F1013247EA0747D4
:1004D80022EA030212F0803F1DD187EA0303A3F149
:1004E800013222EA030313F0803F14D1043002E002
:1004F80012F0803F0FD1064650F8043BA3F10135B6
:1005080087EA030225EA0303A2F1013413F0803FCE
:1005180024EA0202ECD033783046002B3CD09942D2
:1005280009D0731C01E0914205D0184613F8012B3D
:10053800002AF8D11046F0BC704710F0030F0CD019
:100548000378002BF7D0431C03E013F8012B002A93
:10055800F1D013F0030F1846F7D102680346A2F151
:10056800013121EA020212F0803F0AD10430034629
:1005780050F8042BA2F1013121EA020212F0803F67
:10058800F5D01A781846002AD5D00133184613F842
:10059800012B002AFAD1CEE71846CCE780EA0102FF
:1005A80012F0030F3AD110F0030220F0030021F0FB
:1005B800030150F804CB08BF51F8043B0DD082F07A
:1005C80003024FEAC2026FF07F4323FA02F251F8A6
:1005D800043B4CEA020C43EA020300BFACF10132CF
:1005E8009C4501BF22EA0C0212F0803F50F804CB70
:1005F80051F8043BF2D04FEA0C604FEA1C2C01285A
:1006080028BFB0EB036F08BF1B0AF4D003F0FF0349
:100618004FEA1060A0EB0300704700BF10F0030F13
:100628000AD010F8012B11F8013B012A28BF9A4281
:10063800F4D0A2EB030070474DF8045D4DF8044D6B
:100648004FF0010242EA022242EA024201F0030CA0
:1006580021F0030150F8044B51F8045BBCF1020F80
:1006680026D04BD824F07F4CBCEB152FA4EB02030B
:1006780023EA04030DD113EAC21308BF51F8045B3F
:100688000AD18CEA040CBCEB056F0CD150F8044B72
:10069800E8E74FEA15255CE033F07F4352D10D7847
:1006A8004FEA146C55E04FEA146C05F0FF0550E072
:1006B8004FEA044CA4EB02034FEA1C4C23EA040360
:1006C800BCEB154F17D113EAC21308BF51F8045BEE
:1006D80007D18CEA040CBCEB054F08D150F8044B49
:1006E800E6E71B042ED10D884FEA144C31E04FEA9F
:1006F80005454FEA144C4FEA15452AE004F0FF0C73
:10070800BCEB156FA4EB020323EA04030DD113EA33
:10071800C21308BF51F8045B0AD18CEA040CBCEB85
:10072800052F0AD150F8044BE8E74FEA156510E0A9
:1007380014F0FF0F06D051F8045B4FEA142C25F093
:100748007F4506E04FF000005DF8044B5DF8045B60
:1007580070470CF0FF0205F0FF00012828BF904207
:1007680004BF4FEA1C2C2D0AF3D0A2EB00005DF861
:10077800044B5DF8045B704780EA0102844612F07E
:10078800030F4FD111F0030F32D14DF8044D11F082
:10079800040F51F8043B0BD0A3F101329A4312F035
:1007A800803F04BF4CF8043B51F8043B16D100BF0E
:1007B80051F8044BA3F101329A4312F0803FA4F19F
:1007C80001320BD14CF8043BA24312F0803F04BF26
:1007D80051F8043B4CF8044BEAD023460CF8013B93
:1007E80013F0FF0F4FEA3323F8D15DF8044B70473D
:1007F80011F0010F06D011F8012B0CF8012B002A7B
:1008080008BF704711F0020FBFD031F8022B12F069
:10081800FF0F16BF2CF8022B8CF8002012F47F4F24
:10082800B3D1704711F8012B0CF8012B002AF9D12C
:10083800704700BF20F0030110F00300C0F1000072
:1008480051F8043B00F1040C4FEACC0C6FF00002A5
:100858001CBF22FA0CF213434FF0010C4CEA0C2C8B
:100868004CEA0C4CA3EB0C0222EA030212EACC126B
:1008780004BF51F8043B0430F4D013F0FF0F1FBF3E
:10088800013013F47F4F013013F47F0F18BF01308C
:10089800704700BFF0B4002A46D041EA000313F0C5
:1008A80003032CD1032A07460E4643D904680D6872
:1008B800AC423FD1043A37D0A4F1013525EA04040B
:1008C80014F0803F18BF18462CD1041D0D1D0EE0F2
:1008D80054F8043B55F8041BA3F101308B4220EA7D
:1008E800030027D1043A1FD010F0803F1ED1032AFD
:1008F80027462E46ECD820462946002A1DD00478E3
:10090800013A0D78AC420CD172B18CB1002302E0EF
:1009180093420BD064B1013310F8014FCD5CAC4267
:10092800F6D0601BF0BC70471046FBE70020F9E7E3
:100938002046F7E738463146E1E724782D78F0E796
:1009480041EA000313F0030F0B4670B414BF0024F0
:100958000124032A94BF002404F001040546D4B9F5
:10096800BAB10E782B46013A03F8016B56B1AC1CAC
:100978007AB111F8015F2346013A04F8015C0134A9
:10098800002DF5D12AB19A18002103F8011B9342D2
:10099800FBD170BC7047194653F8044BA4F10136DB
:1009A80026EA040616F0803FDAD1043A45F8044BEB
:1009B800032A1946EFD8D3E701232DE9F0071D468E
:1009C80000264FF0FF37AC1900EB070C8C420DD214
:1009D8001CF805C010F80480E0452ED201252646F3
:1009E800E31BAC198C4200EB070CF1D34FF0010963
:1009F80000264D464FF0FF3C1360AC1900EB0C0885
:100A0800A1420ED918F8058010F804A0C2451AD9D9
:100A180001252646CCEB0409AC19A14200EB0C08D1
:100A2800F0D80CF101000137B8423CBF994638466E
:100A3800C2F80090BDE8F00770470BD00123374695
:100A48001D46F618BFE709D04FF00109B4464D46D8
:100A58004E44D2E79D4205D00135B4E74D4505D057
:100A68000135CAE72B4626460125ACE7A9462646A6
:100A78000125C2E72DE9F04FADF5826D81B014462E
:100A8800074610460DF580628B460C3219461D4606
:100A9800FFF792FF03AE04A901F57E72331F0090A1
:100AA80043F8045F9342FBD14DB1681E0023E25C1A
:100AB800C11A013303AEAB4246F82210F7D1DDF874
:100AC8000C142046009A6118FFF78AFB002877D19A
:100AD8000099814605F1FF380646C1F101020192ED
:100AE8005A46AB4609EB0B0501F1FF3AB81800214D
:100AF800AA1A00F0E5F900284FD1002D00F0C080B7
:100B08007B1903A913F8013C51F82330002B4CD171
:100B1800009B9E4228BF334698450FD903EB090135
:100B2800E05C7A18795C884205D038E012F8011F39
:100B3800E05C884233D101339845F7D8009A964251
:100B480080F0A48007EB090214F80A10534612F843
:100B58000A20914204BF0AEB0901791807D095E0F1
:100B680014F802C011F8010D844503D113465A1E2A
:100B7800B342F5D101369E4200F28D80DDF80C6457
:100B88002A46B144C6EB0B0609EB0B05B818002141
:100B9800AA1A00F095F90028AFD0002071E0019A58
:100BA8000026914499442A46EEE7002EFAD0DDF853
:100BB8000C2493423CBFC2EB0B0306469944F2E770
:100BC800009E4FF000080099AB1BB34238BF334674
:100BD800C1F101026E1E019201F1FF3A5A4689469F
:100BE800AB460133CDF80C3408EB0B05B8180021DF
:100BF800AA1A00F065F90028CFD1002D40D07B1942
:100C080003A913F8013C51F82330002B30D1B1452A
:100C180013D208EB090314F80910FA18FB5C99427F
:100C280018BF4B4627D14B4604E012F8011FE05C81
:100C3800884220D10133B342F7D3BAF1FF3F53467C
:100C48002CD007EB080C14F80A101CF80A20914263
:100C58000CD10AEB0802BA1804E0E05C12F8011D96
:100C6800884203D1013BF8D260460AE0DDF80C3433
:100C780098442A46B8E701992A4688449844B3E735
:100C8800284605B00DF5806DBDE8F08F009B013654
:100C98009E427FF673AF07EB0900F2E707EB080CFB
:100CA8006046EEE72DE9F04F8346037885B00C46A1
:100CB800002B00F0F9800A78A2B106460131012024
:100CC80002E011F8012B8AB1934214BF002000F012
:100CD800010016F8013F0D46002BF2D12B782BB1FD
:100CE8004FF0000B584605B0BDE8F08F0028F9D149
:100CF8000BF101002178FFF7CBFB2D1BA5F10102B9
:100D0800534243EB0203002808BF43F001030746A0
:100D180083B90BEB0508404594BFC0EB08084FF0BA
:100D280001081F2D08D9414622462B46FFF7A2FE8F
:100D38008346D7E78346D5E7294603AA2046FFF727
:100D48003BFE03996118814620464A46FFF748FA58
:100D580000284FD109F1FF33C9F10102064601927B
:100D680082464246C84699460AEB050BB818002148
:100D7800C2EB0B0200F0A4F80028B1D1BBF1000FC0
:100D8800B0D046452CBF334643469D420FD903EBAE
:100D98000A01E05C7A18795C884205D075E012F89F
:100DA800011FE05C884270D101339D42F7D1B04504
:100DB8007DD907EB0A0214F809104B4612F80920EE
:100DC800914202BF09EB0A01AC46791806D06EE0E1
:100DD800A55C11F8010D854203D113465A1EB34292
:100DE800F6D1654601369E4267D8039E5A46B244FC
:100DF800AE1BB9E7C9F10101C9EB0503424600265C
:100E080009F1FF3A88464B4538BF4B4601330393F7
:100E180006EB050BB8180021C2EB0B0200F050F8E6
:100E280000287FF45DAFBBF1000F3FF45BAF4D4589
:100E380012D906EB090314F80910FA18FB5C994259
:100E480008BF4B4605D026E012F8011FE05C884237
:100E580022D101339D42F7D1BAF1FF3F534628D042
:100E680007EB060C14F80A101CF80A20914217D157
:100E78000AEB0602BA1804E0E05C12F8011D884289
:100E88000ED1013BF8D2E3462CE7019A00269244A2
:100E98005A469A4468E74B4646445A46F618B7E716
:100EA800039B5A46F618B3E70D46012016E743465A
:100EB80098E707EB060CE34614E707EB0A0B11E784
:100EC80010F0030F034670B4C9B211D0002A22D023
:100ED80003788B421DD0013A013005E0DAB110F8F1
:100EE800014B013A8C4218D010F0030F0346F5D19C
:100EF800032A14D87AB1187888420ED0541E5D1C83
:100F080003E015F8016B8E4203D0013C2846F8D265
:100F1800002070BC70471046FBE71846F9E741EA25
:100F2800012646EA0646184653F8044B86EA0404A6
:100F3800A4F1013525EA040414F0803F03D1043AF2
:100F48001846032AEFD80346D4E700BF0000000084
:100F5800C1F30A5C0246ACF57E7C2DE9F84FACF192
:100F68000704132C0B4606460F468946804627DCA5
:100F7800002C52DB4FF6FF7CC0F20F0C4CFA04FA3F
:100F88000AEA0105054317D037A3D3E9002300F087
:100F980075F80022002300F0B3FC002856D0002F7B
:100FA80005DD4FF4801353FA04F407EB040929EA2A
:100FB8000A0900264B46324610461946BDE8F88F06
:100FC800332C07DDB4F5806FF6D100F057F80246F0
:100FD8000B46F1E74FF0FF3BACF11B0C2BFA0CFB77
:100FE8001BEA000FE8D020A3D3E9002300F046F85D
:100FF8000022002300F084FC40B3002F0ADD142CEB
:1010080006D00126C4F13404A64016EB080601D325
:1010180007F1010926EA0B0619E013A3D3E9002317
:1010280000F02CF80022002300F06AFC78B1002FB1
:1010380013DB46EA07054FF000094D45C3F6F07982
:101048000CBF2E46002608BFA94600E0B9464B460D
:10105800324610461946BDE8F88F00264FF0004981
:10106800F5E700BFAFF300809C7500883CE4377E4D
:1010780081F0004102E000BF83F0004330B54FEA41
:1010880041044FEA430594EA050F08BF90EA020FAE
:101098001FBF54EA000C55EA020C7FEA645C7FEA41
:1010A800655C00F0E2804FEA5454D4EB5555B8BF64
:1010B8006D420CDD2C4480EA020281EA030382EAD5
:1010C800000083EA010180EA020281EA0303362D67
:1010D80088BF30BD11F0004F4FEA01314FF4801C3A
:1010E8004CEA113102D0404261EB410113F0004F4C
:1010F8004FEA03334CEA133302D0524263EB430303
:1011080094EA050F00F0A780A4F10104D5F1200EA0
:101118000DDB02FA0EFC22FA05F2801841F10001FB
:1011280003FA0EF2801843FA05F359410EE0A5F1CF
:1011380020050EF1200E012A03FA0EFC28BF4CF000
:10114800020C43FA05F3C01851EBE37101F00045B6
:1011580007D54FF0000EDCF1000C7EEB00006EEBC3
:101168000101B1F5801F1BD3B1F5001F0CD349084D
:101178005FEA30004FEA3C0C04F101044FEA4452A4
:1011880012F5800F80F09A80BCF1004F08BF5FEA2B
:10119800500C50F1000041EB045141EA050130BD0B
:1011A8005FEA4C0C404141EB010111F4801FA4F1AE
:1011B8000104E9D191F0000F04BF01460020B1FA03
:1011C80081F308BF2033A3F10B03B3F120020CDA3B
:1011D8000C3208DD02F1140CC2F10C0201FA0CF019
:1011E80021FA02F10CE002F11402D8BFC2F1200C7E
:1011F80001FA02F120FA0CFCDCBF41EA0C01904034
:10120800E41AA2BF01EB0451294330BD6FEA04047C
:101218001F3C1CDA0C340EDC04F11404C4F1200267
:1012280020FA04F001FA02F340EA030021FA04F379
:1012380045EA030130BDC4F10C04C4F1200220FAD0
:1012480002F001FA04F340EA0300294630BD21FA0E
:1012580004F0294630BD94F0000F83F4801306BFD4
:1012680081F480110134013D4EE77FEA645C18BFC8
:101278007FEA655C29D094EA050F08BF90EA020F5F
:1012880005D054EA000C04BF1946104630BD91EA57
:10129800030F1EBF0021002030BD5FEA545C05D15A
:1012A8004000494128BF41F0004130BD14F5800499
:1012B8003CBF01F5801130BD01F0004545F0FE410D
:1012C80041F470014FF0000030BD7FEA645C1ABF42
:1012D800194610467FEA655C1CBF0B46024650EA79
:1012E800013406BF52EA033591EA030F41F40021A5
:1012F80030BD00BF90F0000F04BF0021704730B52B
:101308004FF4806404F132044FF000054FF00001FF
:1013180050E700BF90F0000F04BF0021704730B5C0
:101328004FF4806404F1320410F0004548BF404295
:101338004FF000013EE700BF42004FEAE2014FEAEA
:1013480031014FEA02701FBF12F07F4393F07F4FC5
:1013580081F06051704792F0000F14BF93F07F4FF7
:10136800704730B54FF4607401F0004521F000413A
:1013780020E700BF50EA010208BF704730B54FF0C0
:1013880000050AE050EA010208BF704730B511F0C5
:10139800004502D5404261EB41014FF4806404F1FD
:1013A80032045FEA915C3FF4DCAE4FF003025FEA7F
:1013B800DC0C18BF03325FEADC0C18BF033202EB07
:1013C800DC02C2F1200300FA03FC20FA02F001FA61
:1013D80003FE40EA0E0021FA02F11444C1E600BF00
:1013E80070B54FF0FF0C4CF4E06C1CEA11541DBFB3
:1013F8001CEA135594EA0C0F95EA0C0F00F0DEF87E
:101408002C4481EA030621EA4C5123EA4C5350EA62
:10141800013518BF52EA033541F4801143F48013B3
:1014280038D0A0FB02CE4FF00005E1FB02E506F044
:101438000042E0FB03E54FF00006E1FB03569CF099
:10144800000F18BF4EF0010EA4F1FF04B6F5007F9F
:1014580064F5407404D25FEA4E0E6D4146EB060611
:1014680042EAC62141EA55514FEAC52040EA5E509A
:101478004FEACE2EB4F1FD0C88BFBCF5E06F1ED844
:10148800BEF1004F08BF5FEA500E50F1000041EB7B
:10149800045170BD06F0004646EA010140EA020028
:1014A80081EA0301B4EB5C04C2BFD4EB0C0541EA4A
:1014B800045170BD41F480114FF0000E013C00F35F
:1014C800AB8014F1360FDEBF002001F0004170BD83
:1014D800C4F10004203C35DA0C341BDC04F114049C
:1014E800C4F1200500FA05F320FA04F001FA05F228
:1014F80040EA020001F0004221F0004110EBD370F5
:1015080021FA04F642EB06015EEA430E08BF20EA20
:10151800D37070BDC4F10C04C4F1200500FA04F3C3
:1015280020FA05F001FA04F240EA020001F0004155
:1015380010EBD37041F100015EEA430E08BF20EAC8
:10154800D37070BDC4F1200500FA05F24EEA020E10
:1015580020FA04F301FA05F243EA020321FA04F03F
:1015680001F0004121FA04F220EA020000EBD370F6
:101578005EEA430E08BF20EAD37070BD94F0000FF6
:101588000FD101F00046400041EB010111F4801F2A
:1015980008BF013CF7D041EA060195F0000F18BFDB
:1015A800704703F00046520043EB030313F4801F17
:1015B80008BF013DF7D043EA0603704794EA0C0FD1
:1015C8000CEA135518BF95EA0C0F0CD050EA4106E7
:1015D80018BF52EA4306D1D181EA030101F0004164
:1015E8004FF0000070BD50EA410606BF104619468C
:1015F80052EA430619D094EA0C0F02D150EA013698
:1016080013D195EA0C0F05D152EA03361CBF1046D8
:1016180019460AD181EA030101F0004141F0FE4177
:1016280041F470014FF0000070BD41F0FE4141F4FB
:10163800780170BD70B54FF0FF0C4CF4E06C1CEAFB
:1016480011541DBF1CEA135594EA0C0F95EA0C0FB0
:1016580000F0A7F8A4EB050481EA030E52EA03356B
:101668004FEA013100F088804FEA03334FF080558C
:1016780045EA131343EA12634FEA022245EA1115B9
:1016880045EA10654FEA00260EF000419D4208BF6A
:10169800964244F1FD0404F5407402D25B084FEA17
:1016A8003202B61A65EB03055B084FEA32024FF4C3
:1016B80080104FF4002CB6EB020E75EB030E22BF20
:1016C800B61A754640EA0C005B084FEA3202B6EBE0
:1016D800020E75EB030E22BFB61A754640EA5C008F
:1016E8005B084FEA3202B6EB020E75EB030E22BF1F
:1016F800B61A754640EA9C005B084FEA3202B6EB20
:10170800020E75EB030E22BFB61A754640EADC00DE
:1017180055EA060E18D04FEA051545EA16754FEA40
:1017280006164FEAC30343EA52734FEAC2025FEA5E
:101738001C1CC0D111F4801F0BD141EA00014FF0ED
:1017480000004FF0004CB6E711F4801F04BF0143BE
:101758000020B4F1FD0C88BFBCF5E06F3FF6AFAEDA
:10176800B5EB030C04BFB6EB020C5FEA500C50F16A
:10177800000041EB045170BD0EF0004E4EEA1131ED
:1017880014EB5C04C2BFD4EB0C0541EA045170BDF4
:1017980041F480114FF0000E013C90E645EA060E38
:1017A8008DE60CEA135594EA0C0F08BF95EA0C0F66
:1017B8003FF43BAF94EA0C0F0AD150EA01347FF4AE
:1017C80034AF95EA0C0F7FF425AF104619462CE785
:1017D80095EA0C0F06D152EA03353FF4FDAE1046E8
:1017E800194622E750EA410618BF52EA43067FF439
:1017F800C5AE50EA41047FF40DAF52EA43057FF4C9
:10180800EBAE12E74FF0FF3C06E000BF4FF0010CD3
:1018180002E000BF4FF0010C4DF804CD4FEA410C37
:101828007FEA6C5C4FEA430C18BF7FEA6C5C1BD004
:1018380001B050EA410C0CBF52EA430C91EA030F85
:1018480002BF90EA020F0020704710F1000F91EAE2
:10185800030F58BF994208BF90422CBFD8176FEAB0
:10186800E37040F0010070474FEA410C7FEA6C5C7E
:1018780002D150EA013C07D14FEA430C7FEA6C5C85
:10188800D6D152EA033CD3D05DF8040B704700BFB1
:101898008446104662468C461946634600E000BFFF
:1018A80001B5FFF7B7FF002848BF10F1000F01BDD1
:1018B8004DF808EDFFF7F4FF0CBF012000205DF89C
:1018C80008FB00BF4DF808EDFFF7EAFF34BF012021
:1018D80000205DF808FB00BF4DF808EDFFF7E0FFBA
:1018E80094BF012000205DF808FB00BF4DF808ED0B
:1018F800FFF7CEFF94BF012000205DF808FB00BF72
:101908004DF808EDFFF7C4FF34BF012000205DF853
:1019180008FB00BF4FEA4102B2F1E04324BFB3F530
:10192800001CDCF1FE5C0DD901F0004C4FEAC0024E
:101938004CEA5070B2F1004F40EB830008BF20F032
:101948000100704711F0804F21D113F13872BCBFEC
:1019580001F00040704741F480114FEA5252C2F141
:101968001802C2F1200C10FA0CF320FA02F018BF8A
:1019780040F001004FEAC1234FEAD32303FA0CFCDD
:1019880040EA0C0023FA02F34FEA4303CCE77FEA6C
:10199800625307D150EA01331EBF4FF0FE4040F4B6
:1019A8004000704701F0004040F0FE4040F4000065
:1019B800704700BF80F0004002E000BF81F00041A6
:1019C80042001FBF5FEA410392EA030F7FEA226CDD
:1019D8007FEA236C6AD04FEA1262D2EB1363C1BF6D
:1019E800D218414048404140B8BF5B42192B88BFDC
:1019F800704710F0004F40F4000020F07F4018BFFF
:101A0800404211F0004F41F4000121F07F4118BF1E
:101A1800494292EA030F3FD0A2F1010241FA03FCC6
:101A280010EB0C00C3F1200301FA03F100F00043AE
:101A380002D5494260EB4000B0F5000F13D3B0F176
:101A4800807F06D340084FEA310102F10102FE2AE5
:101A580051D2B1F1004F40EBC25008BF20F0010055
:101A680040EA03007047490040EB000010F4000F03
:101A7800A2F10102EDD1B0FA80FCACF1080CB2EB96
:101A88000C0200FA0CF0AABF00EBC25052421843F5
:101A9800BCBFD0401843704792F0000F81F400019A
:101AA80006BF80F400000132013BB5E74FEA41036D
:101AB8007FEA226C18BF7FEA236C21D092EA030FD9
:101AC80004D092F0000F08BF0846704790EA010F53
:101AD8001CBF0020704712F07F4F04D1400028BF80
:101AE80040F00040704712F100723CBF00F5000062
:101AF800704700F0004343F0FE4040F40000704798
:101B08007FEA226216BF08467FEA23630146420243
:101B180006BF5FEA412390EA010F40F48000704756
:101B28004FF0000304E000BF10F0004348BF4042FC
:101B38005FEA000C08BF704743F0964301464FF038
:101B480000001CE050EA010208BF70474FF0000394
:101B58000AE000BF50EA010208BF704711F00043D5
:101B680002D5404261EB41015FEA010C02BF8446A5
:101B78000146002043F0B64308BFA3F18053A3F504
:101B88000003BCFA8CF2083AA3EBC25310DB01FA4B
:101B980002FC634400FA02FCC2F12002BCF1004FCF
:101BA80020FA02F243EB020008BF20F00100704760
:101BB80002F1200201FA02FCC2F1200250EA4C00B4
:101BC80021FA02F243EB020008BF20EADC707047FA
:101BD8004FF0FF0C1CEAD0521EBF1CEAD15392EA08
:101BE8000C0F93EA0C0F6FD01A4480EA010C4002E4
:101BF80018BF5FEA41211ED04FF0006343EA50103E
:101C080043EA5111A0FB01310CF00040B1F5000F7F
:101C18003EBF490041EAD3715B0040EA010062F12E
:101C28007F02FD2A1DD8B3F1004F40EBC25008BF18
:101C380020F00100704790F0000F0CF0004C08BF36
:101C480049024CEA502040EA51207F3AC2BFD2F103
:101C5800FF0340EAC250704740F400004FF0000311
:101C6800013A5DDC12F1190FDCBF00F0004070474B
:101C7800C2F10002410021FA02F1C2F1200200FA89
:101C880002FC5FEA310040F1000053EA4C0308BF50
:101C980020EADC70704792F0000F00F0004C02BFA1
:101CA800400010F4000F013AF9D040EA0C0093F01C
:101CB800000F01F0004C02BF490011F4000F013B76
:101CC800F9D041EA0C018FE70CEAD15392EA0C0FE4
:101CD80018BF93EA0C0F0AD030F0004C18BF31F04F
:101CE800004CD8D180EA010000F00040704790F025
:101CF800000F17BF90F0004F084691F0000F91F0C9
:101D0800004F14D092EA0C0F01D142020FD193EA8E
:101D18000C0F03D14B0218BF084608D180EA010016
:101D280000F0004040F0FE4040F40000704740F0F2
:101D3800FE4040F4400070474FF0FF0C1CEAD052C0
:101D48001EBF1CEAD15392EA0C0F93EA0C0F69D01C
:101D5800A2EB030280EA010C49024FEA402037D087
:101D68004FF0805343EA111143EA10130CF000407E
:101D78008B4238BF5B0042F17D024FF4000C8B426E
:101D880024BF5B1A40EA0C00B3EB510F24BFA3EB4E
:101D9800510340EA5C00B3EB910F24BFA3EB91031E
:101DA80040EA9C00B3EBD10F24BFA3EBD10340EA78
:101DB800DC001B0118BF5FEA1C1CE0D1FD2A3FF6BE
:101DC80050AF8B4240EBC25008BF20F00100704773
:101DD8000CF0004C4CEA50207F32C2BFD2F1FF0316
:101DE80040EAC250704740F400004FF00003013A47
:101DF80037E792F0000F00F0004C02BF400010F4EB
:101E0800000F013AF9D040EA0C0093F0000F01F0FE
:101E1800004C02BF490011F4000F013BF9D041EA20
:101E28000C0195E70CEAD15392EA0C0F08D1420253
:101E38007FF47DAF93EA0C0F7FF470AF084676E726
:101E480093EA0C0F04D14B023FF44CAF08466EE7FF
:101E580030F0004C18BF31F0004CCAD130F00042CD
:101E68007FF45CAF31F000437FF43CAF5FE700BF25
:101E78004FF0FF3C06E000BF4FF0010C02E000BF4E
:101E88004FF0010C4DF804CD4FEA40024FEA4103F0
:101E98007FEA226C18BF7FEA236C11D001B052EAA6
:101EA800530C18BF90EA010F58BFB2EB030088BF6C
:101EB800C81738BF6FEAE17018BF40F001007047DB
:101EC8007FEA226C02D15FEA402C05D17FEA236CBD
:101ED800E4D15FEA412CE1D05DF8040B704700BF04
:101EE800844608466146FFE70FB5FFF7C9FF00289B
:101EF80048BF10F1000F0FBD4DF808EDFFF7F4FFD4
:101F08000CBF012000205DF808FB00BF4DF808ED6C
:101F1800FFF7EAFF34BF012000205DF808FB00BF8F
:101F28004DF808EDFFF7E0FF94BF012000205DF8B1
:101F380008FB00BF4DF808EDFFF7D2FF94BF012062
:101F480000205DF808FB00BF4DF808EDFFF7C8FF5B
:101F580034BF012000205DF808FB00BF42000ED20C
:101F6800B2F1FE4F0BD34FF09E03B3EB126209D4CC
:101F78004FEA002343F0004323FA02F070474FF082
:101F88000000704712F1610F01D1420202D14FF0F7
:101F9800FF3070474FF00000704700BF00F026F890
:101FA8000C4880F30888002103E00B4B5B58435032
:101FB80004310A480A4B42189A42F6D3094A02E009
:101FC800002342F8043B084B9A42F9D317F0EEFD80
:101FD8007047000000C0002058800308000000205F
:101FE800600E0020600E0020944700207047FEE736
:101FF80010B586B0002301244FF46022114801A9CE
:1020080001938DF80930039204938DF808408DF8F8
:10201800144025F099FB0B48214625F0BBFB0948E5
:1020280025F0C2FB074825F0C4FB0028FAD1054873
:1020380025F0C3FB034825F0C5FB0028FAD106B0FC
:1020480010BD00BF00240140014610B50D48012213
:10205800032325F0C5FB0B48012125F0B7FB7F20A2
:1020680026F0F4F90748022125F004FC0028F6D0F0
:102078000448022125F004FC0248BDE8104025F080
:10208800F6BB00BF002401400C4A0C2303FB0123CC
:1020980010B59C880CB9588010BD5B8803F11304F7
:1020A800844204DA142B07D9133B834204DC0C2343
:1020B80003FB012102238B8010BD00BFBC2500203B
:1020C8000A4B10B500241C7021464FF4E0720848F2
:1020D800FEF760F9074B4FF474501C70064B1C70E8
:1020E8000FF016F8054B187010BD00BFDC1000206B
:1020F800A8120020F314002070140020721400208D
:10210800074B1978013101F01F011970054B1A7836
:102118008A4203D1013202F01F021A70704700BFD1
:1021280070140020F314002010B50E4A0E2303FB90
:1021380000200D4A014614780C4A03FB042300F1E1
:102148000C0251F8044B914243F8044BF9D10A8828
:1021580000211A800E22FEF71DF9BDE81040FFF796
:10216800CFBF00BFE010002070140020A81200208C
:10217800084B1A5C002352FA03F111F0010FD8B290
:1021880002D00130C0B270470133042BF3D10120D3
:10219800704700BFA015002000F07F0000F57450C4
:1021A8002DE9F84305300C46154698460EF0B0FF69
:1021B80000284ED043F63837002638460EF0A8FFE0
:1021C800C0B25FFA86F988B120280FD04FEA5909C2
:1021D8004AF28B6048440EF09BFFC0B208B1022857
:1021E80004D10123B34022781343237011370136F9
:1021F800B7F56F5FE1D14AF232500EF089FFC0B2F5
:1022080080B120280ED02B784AF2215043F00103E8
:102218002B700EF07DFFC0B220B1202802D0012320
:1022280088F800304AF263500EF072FFC0B280B1F5
:1022380020280ED02B784AF2215043F002032B704D
:102248000EF066FFC0B220B1202802D0012388F822
:102258000030BDE8F8830000034610465A1E10B54A
:10226800032A1CD8DFE802F00E0E0207114A527842
:1022780002F0100203E00F4A527802F00802D2B2CC
:1022880072B10BE00C4A927802F04002D2B23AB135
:102298000A4A127802F003029A4200D140B10022A1
:1022A8000748105C984203D00132052AF8D1002172
:1022B800084610BD98410020C03100209335002009
:1022C800A0120020F8B5064643F638350024284603
:1022D8000EF01EFFC0B2E7B268B120280BD07F080D
:1022E8004AF28B6038180EF013FF012803D1A04082
:1022F80033781843307001341135082CE7D1F8BD14
:1023080003780E2202FB0313084AD3189978002396
:1023180051FA03F010F00100DAB202D0501CC0B23A
:1023280070470133082BF3D1704700BFA812002073
:102338002DE9F04101248C40284A29490346E4B29A
:10234800107891F800C019E0264F0E2606FB00769B
:10235800F178A9B996F80680B8F1000F10D196F86F
:102368000580B8F1000F0BD196F80480B8F1000F82
:1023780006D1F67926B9013000F01F00054626E09F
:10238800FBB1012B05D0022B06D10E2101FB0077F2
:1023980039790C4218D014E0042B04D10E2101FB2A
:1023A8000077B9790CE0032B04D10E2101FB0077EB
:1023B800797905E0052B07D10E2101FB0077F97922
:1023C80011B11570BDE8F081013000F01F006045C3
:1023D800BAD11570FF20BDE8F08100BFF3140020CA
:1023E80070140020A81200202DE9F043434D444BFF
:1023F8002A780E2101FB0232917A85B0044698466C
:1024080031B101390523594301F56F5189B201E012
:102418004FF46F51204604220EF08BFE2B780E25C8
:1024280005FB038393F80B80354E344FB8F1000F4A
:1024380025D131232371073363713B7801A86B439E
:102448000422F15E06F0C4FA3B7802A805FB036398
:102458000222997A06F0BCFA3B780DF10A0005FBD6
:1024680003650322697A06F0B3FAA01D01A90922BF
:10247800FEF766FA4FF00F0984F8108012E0B8F101
:10248800010F0FD132232371053363713B784FF06D
:10249800080905FB036393F90130E3713B785D4359
:1024A800735BA371002320461A4612E010F8011B43
:1024B800A1F13005EDB2092D04D8EB183029DBB2B3
:1024C80003D004E037395B1800E00A33DBB201328D
:1024D800D2B24A45EAD10F21B3FBF1F10801411A02
:1024E8005B1AC3F10F03DBB2092BA35401D83033B5
:1024F80000E03733A35405B0BDE8F083A6120020EE
:10250800A8120020024B1A7842F001021A70704794
:10251800D517002008B50C4B0C4A1B780E2101FB7F
:102528000323D97A21B101290CBF0921002100E038
:10253800102140221346064806F06EF8054B1A781B
:1025480042F002021A7008BDA6120020A81200204C
:1025580073140020D5170020034B1A7802F0F802F4
:102568006FF3C3021A707047D5170020024B1A7810
:1025780042F004021A707047D5170020024B1A78EF
:1025880042F008021A707047D517002038B5114B71
:102598001C7814F0010502D1FFF7B4FF05E004F040
:1025A8000405EDB21DB9FFF7E1FF284638BD04F078
:1025B8000805EDB215B9FFF7E1FFF6E704F00204EC
:1025C800E4B21CB9FFF7A6FF204638BDFFF7C4FFE9
:1025D800012038BDD5170020014B1878704700BF7F
:1025E800DC10002030B51E4B85B01B780446002B4C
:1025F80034D11C4D2B78034113F0010F2ED01A4B08
:102608001A4A1B780E2101FB0323DA78024112F0E3
:10261800010F1CD11B79034113F0010317D110F0EE
:10262800010001F1F1014FEA540206D00132009194
:10263800019302926D20FE3905E00132009101906C
:1026480002923C20012103220B460EF0DFFD0123FC
:1026580013FA04F42B7823EA04042C7005B030BD77
:102668007214002069140020F3140020A81200201E
:10267800037830B513F0010F144A4FF00E0419D146
:1026880004FB01210133012212FA03F3CD7825EA74
:102698000303CB7004780D79A41812FA04F425EA20
:1026A80004040C7103789B189A408B7823EA020281
:1026B8008A7030BD04FB0121013B012212FA03F3A9
:1026C8008A7822EA03038B7030BD00BFA81200206D
:1026D80010B500230278590052FA01F404F00304FB
:1026E800022C05D1013414FA01F122EA0102027028
:1026F8000133042BEED110BD2DE9F04F85B00192C6
:10270800BDF838201C46744B0092DA78054612F062
:1027180020028B4640F0D9808DF80E208DF80F20CE
:102728008DF80D20DCB99B7803F04003DBB21BB1B8
:1027380001238DF80F3020E0684B5B7803F002032B
:10274800DBB21BB101238DF80E3016E00DF10F013D
:102758000DF10E020DF10D03FFF71EFD0DE0012C2A
:102768000BD19B7803F04003DBB223B90DF10F00C6
:10277800FFF7A8FD01E08DF80F409DF80F3023B951
:102788009DF80E00002800F0A38044B905F07F01F1
:10279800490001F574510DF10A0062310AE0012C7B
:1027A8000BD1E90101F50C4101F5DE710DF10A00CB
:1027B80001EB4B0102220EF0BCFCBDF90A3013B943
:1027C800002C00F08480009B33B9454B454F93F8AB
:1027D8000080FFF795FC08E0434B444F93F80080D6
:1027E80008F1010202F01F021A700DF10F00FFF745
:1027F8006FFF002C44D1BDF80A3069B240F6B832F8
:1028080012EA210238BF4FF47A72D2180E2303FB62
:1028180008F3ADF80A20FA529DF80F90224649466F
:102828000120FE18FFF718FD4946F07022460220E5
:10283800FFF712FD86F8029030719DF80E9022463F
:1028480049460420FFF708FD4946B07182462246F2
:102858000320FFF701FD05F07F0570713572BAF1AD
:10286800000F00D128B1224B1B7813B99DF80D3009
:1028780000E00023F37186F809B0019AB2721CE0F7
:10288800012C1AD10E2303FB08F3BDF80A202046B9
:10289800FA529DF80F6000223146FD18FFF7DCFC64
:1028A8003146E87000220220FFF7D6FC0023287189
:1028B800AE70AB716B71EB71AB720E2303FB0877D3
:1028C800FC72009B0120BB8102E0002000E0204652
:1028D80005B0BDE8F08F00BFC0310020984100204E
:1028E80070140020A8120020DB100020E010002047
:1028F800BA17002073B5154B04461B780E46D3B1A2
:102908001348214620F02FFC0546A0B9012E04F1FA
:10291800010606D12046FFF72BFC009502468120D0
:1029280005E02046FFF724FC009502469820314632
:102938002B46FFF7E1FE2146054820F0FEFB05483F
:10294800214602B0BDE8704020F002BC711400209E
:10295800DA160020031500202DE9F7437B4B0446C7
:102968001B7843B17A4B1B7803F02403042B02D164
:10297800002900F0E880774B774F1B78002B00F098
:10298800C7807648214620F0EEFB002840F0C08042
:1029980007F5C470214620F0E6FB8046002840F089
:1029A800B7803B1993F880302D2B01D0532B3AD1A7
:1029B8006B4E357845B30EF01FFF04F1010805464C
:1029C80050B12046FFF7D4FB337802461E330093FC
:1029D80093204146002307E02046FFF7C9FB0095F6
:1029E8000246414693202B46FFF786FE0EF004FF71
:1029F800014628B1337803201E330093002101E0FB
:102A0800009003200A4680E02046FFF7B1FB611CD6
:102A180002462B4693200095FFF76EFE0095032093
:102A280029462A4671E0542B09D12046FFF7A0FB1E
:102A3800CDF800800246611C9420434666E0462B90
:102A4800474D20D12E78BEB10EF0D6FE04F1010913
:102A5800064648B12046FFF78BFB2B7802461E330B
:102A680000939A20494622E02046FFF781FB009612
:102A7800024649469A2025E02046FFF779FB009652
:102A880002469A2039E02E78002E2CD00EF0B4FEA3
:102A980004F11C09064660B12046FFF769FB2B7854
:102AA80002461E3369F07F000093C0B2611C4346A2
:102AB80009E02046FFF75CFB024669F07F000096BC
:102AC800C0B2611C3346FFF717FE0EF095FE21B227
:102AD800024628B12B7803201E330093002214E00D
:102AE8000090032011E02046FFF742FB024604F164
:102AF8001C0060F07F000096C0B2611C3346FFF7EF
:102B0800FBFD00960320214632460123FFF7F4FD22
:102B1800124821463F1920F010FB97F880302D2BE2
:102B28000AD0532B08D0542B06D0462B04D00D487E
:102B3800214620F018FB30B10B48214603B0BDE810
:102B4800F04320F005BB03B0BDE8F083DE100020A1
:102B5800C816002071140020E8230020DA1600208F
:102B68003217002070250020D2160020002302789A
:102B78000E2101FB0232044901338A180021062B79
:102B88009170F4D1704700BFA8120020064B0020B6
:102B98001870064B1A78064B1B789A4202D00146E9
:102BA800FFF7C6BBFF207047DC1000207014002020
:102BB800F31400200121814038B5114BC9431A781C
:102BC800104BC9B202F0030203F5E074012A04D1E4
:102BD800DD7801EA0505DD7005E0022A03D11D79DB
:102BE80001EA05051D710E33A342EFD1FFF7FAFC88
:102BF8004FF474500EF08CFA034B187038BD00BFB8
:102C080093350020A8120020721400202DE9F74304
:102C1800A34D8DF807002B78A24C1BB12378C2B2C4
:102C28009A4204D04FF474500EF072FA28709DF84E
:102C3800073023709C4C2278072A00F22D81DFE8A8
:102C480012F008002400360054005D0072008D0068
:102C5800BA00964A3C211170954A1946107800F03E
:102C68000300FFF765FB934BFF28187000F03681CF
:102C78001EF07AFF904B002093F8742042F0010276
:102C880083F874208D4B187064E0884B1B78002BF8
:102C980000F024811FF030F9012840F04D8123789D
:102CA800142201332370864B01381A7047E17F4B99
:102CB8001B78002B00F01281814E307808B901236F
:102CC8004AE01FF019F9022804D01FF015F903286B
:102CD80040F032811EF048FF23780422013323702C
:102CE8001D233370774B1A7026E1704B3C221A7003
:102CF8007548FFF779FB2378013323706B4B1B78FA
:102D0800002B00F0EB806E4B1D78002D40F01481F5
:102D18001020FFF73BFC002800F01181237828469B
:102D2800013323700BE1614B1B78002B00F0D68038
:102D380005F0DCFC002800F00281614B7D221A704E
:102D48005E4B002018705C4B93F8742042F001022F
:102D580083F87420237801332370F0E0534B1B78F9
:102D6800002B00F0BB801FF0C7F80128544E03D099
:102D78001FF0C2F803280FD19DF80720012111FA8E
:102D880002F2524B197821EA02021A706423337056
:102D9800237801332370CFE03078002840F0CC80CE
:102DA800484A032323701378013BDBB21370002BCE
:102DB80000F09480C3E0404A414E92F86A201AB16C
:102DC8003278002A40F0B88000223270013212FABC
:102DD80003F3DFF8E0803E4F98F800104FF00E093B
:102DE80009FB0172DB4392F803E0DBB203EA0E0E43
:102DF800907882F803E092F804E003EA0E0E0340AC
:102E0800937082F804E00DF10700FFF731FC98F8A1
:102E1800003009FB0372D278DFF894902AB999F848
:102E2800002002F00302012A0AD00E2202FB0372DC
:102E38001279B2B999F8002002F00302022A10D1DF
:102E48000E2202FB0377BA785AB9224F3A789A428F
:102E580007D11848FFF78AFE3B78013303F01F03B8
:102E68003B7099F800009DF8071000F00300FFF789
:102E78005FFA144B0422FF281A7088F80000164BDA
:102E880042D0987800F04000C0B200283CD103231B
:102E980023701A33337052E0002020704FE000BFD7
:102EA80072140020DF100020DC1000206A140020BB
:102EB80093350020A612002018350020DD100020D0
:102EC800DA10002068140020731400206914002010
:102ED800A8120020F3140020C0310020FFF73CFBAB
:102EE800002323701EF040FE2B78013BDBB22B70D1
:102EF8002BB1144B9B7803F04003DBB2F3B19DF880
:102F08000700FFF757FE19E09B780E4A03F04003CD
:102F1800DBB22BB1136843F400031360FFF7D0F85A
:102F2800FFF71AFB1EF020FE002323704FF47450A5
:102F38000EF0EEF8287001E0002000E0FF20BDE868
:102F4800FE8300BFC0310020044B1A780AB1013A51
:102F58001A701B780BB9FFF72DBE7047721400204A
:102F6800044A054B10781B7803EA501000F0010062
:102F7800704700BFC0310020A2160020044B054A4C
:102F88001B781078C3F3400303EA1010704700BFA2
:102F9800A2160020C0310020034B044A1B78D078C9
:102FA800C3F3800318407047A2160020C0310020E8
:102FB800044B054A1B78D078C3F3C00303EA5000DA
:102FC800704700BFA2160020C0310020044B054AFC
:102FD8001B78D078C3F3001303EA9000704700BF52
:102FE800A2160020C0310020044B1878044BDB786F
:102FF8005B005BB2DB1103EAD0107047A216002019
:10300800C03100202DE9F041154E0024B04620E0E3
:10301800204629461BF078FD90B1F35DFF2B0FD0B9
:103028004FF4A07363430A2202FB053318F80330F8
:10303800DB0905D00B4B1878C0F30010BDE8F08110
:1030480001350A37202DE3D10134022C06F5A0768C
:1030580002D000273D46DBE70020BDE8F08100BF35
:1030680065360020A216002008B51BF04FF9034B67
:103078001B7800EA931000F0010008BDA21600209A
:10308800044B054A1B78D078C3F3401303EAD000F9
:10309800704700BFA2160020C03100202DE9F84F6C
:1030A800FFF75EFF8146FFF769FF8246FFF774FF6F
:1030B8008346FFF77DFF8046FFF788FF0446FFF74A
:1030C800A1FF0546FFF7DCFF0746FFF7CDFF0646E1
:1030D800FFF78AFF4FEA8B0343EA4A0343EA0903EF
:1030E80043EAC80343EA471343EA861345EA04045C
:1030F80043EAC013E0B243EA0010BDE8F88F0000CD
:10310800044B987800F00F00A0F10203584240EBFE
:103118000300704740150020044B987800F00F001A
:10312800A0F10102504240EB020070474015002018
:10313800044B987800F00F00A0F10301484240EBDF
:103148000100704740150020054B987800F00F00EB
:10315800A0F1060CDCF1000040EB0C00704700BF4A
:1031680040150020514AF0B513781446012B29D098
:1031780003D3022B40F098805EE04D484D4B047815
:1031880019786FF3C304047001F0F80158786FF3ED
:10319800C301197000F08001C9B2002900F08480D1
:1031A800012111709C78062204F00F045443024652
:1031B8004148005D60F306025A701A7861F3020212
:1031C8001A70F0BD3B494D780B4625F07F0000286A
:1031D80038D00A7802F00802D2B222B9344A1178FB
:1031E80041F0080111709A7802F00F02012A04D107
:1031F8002F4A117841F00101117015F07F0F53D15A
:1032080019789E7801F00700062206F00F0602FBE7
:103218000606294F5D78BE5D013066F3060500F0AD
:1032280007005D7090FBF2F502FB150262F30201E4
:10323800197002232370F0BD1E494D780B4625F006
:103248007F0028B98B7860F303038B701070F0BD92
:10325800174A11786FF3C3011170997801F00F01C3
:10326800012903D111786FF30001117015F07F0F58
:103278001AD119789E7801F00700062206F00F0689
:1032880002FB06060C4F5D78BE5D013066F306054D
:1032980000F007005D7090FBF2F502FB150262F387
:1032A8000201197001232370F0BD00BF8F150020A3
:1032B8000215002040150020F484020810B51F4AAA
:1032C8001F4B92F9031009B1002231E008B1032124
:1032D80019701978032930D8DFE801F00209192C90
:1032E8001178002929D0154881700121197092F9A7
:1032F8000200124920B1134B1A786FF3861217E0B7
:10330800487808B9032213E088700221197092F9ED
:1033180002100A4889B90B4A147861F386141470AC
:10332800026861F30F22D1B261F3174202600122F1
:103338001A7010BD00211160197010BD34170020DB
:10334800FD140020F833002038B5044643F6EF2377
:1033580043F6F020012A08BF18460D460DF0D8FEA6
:103368002378C0B21842104C09D043F6EE200DF075
:10337800CFFE236860F307036FF30F230CE02B786D
:1033880018420AD043F6EE200DF0C2FE2368C0B200
:1033980060F3070360F30F23236094F9003013B13F
:1033A800014B0F22DA7038BD3417002008B543F6F8
:1033B800F7200DF0ADFE014B187008BDFE1400207B
:1033C800014B1870704700BFAB1600202DE9F0477D
:1033D8004FEAD20808F5264909F1330902F0070334
:1033E8000446012748460D469F4016460DF090FEBC
:1033F800FFB2C1B215B921EA070100E0394308F567
:10340800D048484608F14A080DF078FE40460DF0CD
:103418007FFEC1B214B921EA070100E039434046F2
:103428000DF06CFE254305D105483146BDE8F0474F
:103438001FF08EBE02483146BDE8F0471FF07DBE42
:1034480043150020024B1A5C6FF303021A547047AD
:10345800E915002070B50C46C10001F5D2411B48A2
:103468000B3108220DF065FE002518482946EEB2FA
:103478001FF079FE08B9237823BB154B2278EB5C43
:103488001A421FD13046F608FFF7DCFF06F5264042
:1034980033300DF03DFE05F00703C0B2184110F0BF
:1034A800010F0FD10B4829461FF05DFE50B1294688
:1034B80008481FF04DFE074B06F5D0404A30995D8D
:1034C8000DF01CFE0135402DCFD170BDAD1600208A
:1034D800A01500204315002038B546F69205402473
:1034E8002046FFF7AFFFA5F5D043094A523BD15C10
:1034F80011F0100F06D06FF30411D15428460021A3
:103508000DF0FCFD0134E4B20135B92CE8D138BD29
:10351800E91500203F287FB5054607D800F5E440A7
:103528008D300DF0F5FDC3B22BB92AE1994A147814
:10353800002C00F02B81984E725D02F00F014C1C9C
:1035480004F00F0464F303023F2D725533D8002CA6
:1035580000F01C8101339C4240F015818F4B5A19B1
:1035680092F88020522A725D03D161F303027255EA
:1035780009E16FF30302EC081B19725593F89021C7
:1035880005F0070352FA03F313F0010F40F0FD8032
:10359800294683481FF0D1FD814B04F5D040195DC1
:1035A8004A3001240DF0AAFD2D190223009301943D
:1035B80002951820CEE0002C00F0E880754B1B78AF
:1035C80001339C4240F0DF80735D05F5D0406FF316
:1035D80003035230012173550DF090FD735D43F0E4
:1035E80010037355A5F14003DBB2032B07D804225F
:1035F8000092013302320192029319202FE0A5F1C3
:103608004803DBB2032B07D80422009201330332AC
:10361800019202931A2060E0A5F15003DBB2012B5E
:1036280007D80422009201330332019202931B202F
:1036380053E0572D07D1042300930124033301934A
:103648000294212086E0A5F15B03DBB2012B09D8A7
:1036580004220092013302320192029322200121B6
:10366800033A8AE05D2D06D1042300930193043BBD
:10367800029328467FE05E2D07D10423009301338F
:103688000193053B02935E2075E0A5F15F03DBB271
:103698003F2B09D804220092013392180192029319
:1036A80033200121053A68E005F16103DBB2032B01
:1036B80007D80422009201330332019202935F205B
:1036C8000BE005F15903DBB2012B09D80422009263
:1036D800013303320192029360200121043A4CE045
:1036E800AA2D07D1042300930124043B01940293DB
:1036F80061202FE0A92D07D104230093023B0193F9
:10370800023B0293622036E0AD2D08D104230093DA
:103718000322043B01920293632001212DE0AB2D8B
:1037280006D104230093043B01930293642022E012
:10373800AC2D06D104230093043B0193029370201F
:1037480019E0AE2D0CD10423009301240233019318
:10375800029468202146032223460DF057FD15E008
:103768004E35EDB2012D10D80423009301350233F4
:10377800019302956A20012103220B460DF046FDB4
:1037880003E01C4602E0002400E00124204604B0C7
:1037980070BD00BF00000020E9150020E8230020CC
:1037A80043150020024B185CC0F30010704700BF9F
:1037B800E9150020F8B508220E4600210746FCF757
:1037C800E9FD46F60B1500243378234113F0010F69
:1037D80008D02946064808220DF0ABFC38460449B3
:1037E8001FF079FC01340835042CEDD1F8BD00BF79
:1037F800B7160020024846F64A0108220DF099BC87
:103808004315002070B5044600F56A5044300DF0A9
:103818007FFC0B4D06462B7813F0010F02D1CC200C
:1038280020F0C6FA2B8843F001032B80054B1E5568
:10383800054B13F8242042F0010203F8242070BD40
:10384800C81600202415002013150020024B185C10
:10385800084100F001007047A015002070B505462A
:103868000024094BE0B2E618E35C4BB12946FFF7A8
:10387800EDFF28B100233370044821461FF068FC8F
:103888000134402CEDD170BDEA160020301500201F
:1038980038B5054600242846E1B2FFF7D7FF10B136
:1038A800044BE35C23B90134042CF4D1002038BD67
:1038B800012038BD2415002038B505460DF09CFFC1
:1038C800A0B100242846E1B2FFF7C0FF40B1084B81
:1038D80013F8243013F0010F02D0064BE35C23B138
:1038E8000134042CEED1002038BD012038BD00BFC2
:1038F8001315002024150020F8B511480021402296
:10390800FCF748FD46F60B15002401270D4829460B
:103918000822A7400DF00DFCFFB2002609483146E9
:103928001FF021FC20B1064BF25C47EA0202F25478
:103938000136402EF2D101340835042CE5D1F8BD0A
:10394800A0150020B71600202DE9FF4100263446B7
:10395800B0461A4B1B78234113F00102184B23D0B1
:10396800184F1D5D17F82430A84538BFA84613F036
:10397800010F1AD0CDB965F3000307F8243023B23C
:103988000122F71902935B2029462B4600920195E4
:103998000DF03CFC7B78B878F9781843621C2B460C
:1039A8000095FEF7A9FE00E01A5501340436042CF0
:1039B800CFD1054B83F80080BDE8FF81FE140020BD
:1039C8002415002013150020FC14002010B50C4B02
:1039D8001B78A3B10B4B1B788BB100240A482146F6
:1039E8001FF0C1FB40B1094821461FF0BCFB18B9C4
:1039F80020460121FEF7B0FF0134402CEED110BD66
:103A080071140020DE100020D21600204E1E002067
:103A18002DE9F043324C334A238800266FF386138E
:103A28006FF3C4032380304B304F85B016701E707F
:103A38009146984617F8013B5BB32278D20052B200
:103A480043EAA2122388402E62F3C40343F04003E2
:103A580023801ED000253046E9B2FFF7F7FEA8B153
:103A680017F8013C13F0010F06D00122AA4099F87B
:103A780000100A4389F8002013F0020F06D0012332
:103A8800AB4098F80020134388F800300135042D26
:103A9800E1D10136F6B2412ECCD1237803F04005AE
:103AA800EDB2D5B903F02403042B0BD1FFF78EFF39
:103AB800FF2300934020294601222B4601950295B9
:103AC8000DF0A4FB238800226FF345136FF38203E4
:103AD8006FF3C4032380064B1A7005B0BDE8F0836A
:103AE800C816002094330020B13300204E15002062
:103AF800AC16002010B50024054821461FF033FB02
:103B080008B9044BE0540134402CF5D110BD00BF76
:103B1800A31600204E15002010B5127804469DF813
:103B28000810DAB1D3B111B10D491FF0C9FAACB11F
:103B3800082246F64A010B480DF0FBFA21460948CF
:103B48001FF0C9FA0749082246F64A000DF0EBFAB9
:103B580005480449BDE810401FF0D3BA10BD00BFA6
:103B680080250020F41400204315002030B5064BB2
:103B780004781D7824EA05040C7001781B7823EA80
:103B88000103137030BD00BFFE14002038B50A4D84
:103B9800002415F8013F2D2B09D0532B07D0542BA7
:103BA80005D0462B03D0054821461FF0D1FA013431
:103BB800402CEED138BD00BF67240020D21600206B
:103BC80010B50F481FF074FA00240E4821461FF064
:103BD800CAFA80B10C4BE31893F88030482B06D012
:103BE80003D82D2B03D0462B00E0542B03D10448D7
:103BF80021461FF0A2FA0134402CE6D110BD00BFC7
:103C080090150020D2160020E8230020094A0A4B0C
:103C1800117831B1997801F00F01814201D000216A
:103C280011709A7860F303029A705A7842F0800211
:103C38005A7070478F15002040150020F0B56E4B64
:103C4800164685B01A7804460F4600236B4911F8CA
:103C5800231011F0010F05D001219940C1F10F0186
:103C680001EA02020133042BF0D1654B1A70002CD3
:103C780000F0878014F0010F0CD00121FF230025EC
:103C8800009352200B460A46019502950DF0BEFAA4
:103C98005C4B1D7014F0020F0DD0FF23012100931F
:103CA800FF3B019302930A460B4653200DF0AEFAF0
:103CB800544B01221A7014F0040F0DD0FF23012178
:103CC8000093FF3B019302930A460B4654200DF0E4
:103CD8009DFA4C4B02221A7014F0080F0DD0FF23E6
:103CE80001210093FF3B019302930A460B4655209E
:103CF8000DF08CFA434B03221A7014F0100F0DD0FC
:103D0800FF2301210093FF3B019302930A460B46D0
:103D180056200DF07BFA3B4B04221A7014F0200F4A
:103D28000DD0FF2301210093FF3B019302930A4624
:103D38000B4657200DF06AFA324B05221A7014F020
:103D4800400F0DD0FF2301210093FF3B0193029305
:103D58000A460B4658200DF059FA2A4B06221A70CB
:103D680014F0800F0DD0FF2301210093FF3B019336
:103D780002930A460B4659200DF048FA214B0722B8
:103D88001A70E7B11F4B08221A70002430462146EA
:103D98001FF0E9F960B1FF230093FF3B0193631C17
:103DA8001BB2012102935A200A460B460DF02EFA47
:103DB8002146304601341FF0CBF9402CE6D110489B
:103DC8001149124AFFF7D2FE114B00221A70013234
:103DD800009206320192083202920B490B4A0848B7
:103DE8000AF0DEFA0B4B3C2251201A7005B0BDE8F0
:103DF800F0400DF0E7BD00BFFE14002013150020B1
:103E08004018002059460020161900200A190020E1
:103E1800051800202315002010B5FFF73FF90446C8
:103E280007481FF073F9D0F1010138BF002104B928
:103E380029B1034A2046BDE81040FFF7FFBE10BD78
:103E4800E1150020054B03EBD00393F8903100F007
:103E5800070053FA00F000F001007047E823002043
:103E680010B50F4B04461B7813F0010315D0FFF76C
:103E78000FFD28B90B4B1B1993F88030462B0DD139
:103E88000DF0BAFC18B92046FFF7DCFF30B1064840
:103E980021461FF052F9012010BD184610BD00BF81
:103EA800C8160020E8230020E1150020024B1878EE
:103EB800003818BF012070472315002010B5034CA7
:103EC80004EB830358709970DA7010BD1315002045
:103ED80010B500240948002100190E220E34FCF701
:103EE80059FAB4F5E07FF5D1054A00231370054A65
:103EF800002199520233AA2BF9D110BDE0100020FD
:103F0800DB1000208A190020044B187800F02400E8
:103F1800A0F10403584240EB03007047C816002084
:103F28007FB5474B04461B780E46AA2B78D04548E8
:103F380021461FF018F90546002871D12046FFF7E1
:103F48008FFF00286DD1404821461FF00CF950B969
:103F58003E4821461FF007F9054620B92046FFF7DD
:103F6800D9FA00285DD13A4B1B7823B9394B1B7815
:103F780013F0010F09D1384BDB7803F02003DBB2D3
:103F88001BB9364B032283F84020012E05D82E4852
:103F980021461FF0E8F840B142E0022E07D12B4835
:103FA80021461FF0E0F810B13AE0274800E0274822
:103FB80021461FF0C2F82A4821461FF0C9F8022EF0
:103FC80015D10125294603222B4600964A20661959
:103FD800019502960DF01AF92046FEF7C9F800235C
:103FE8000246314618200093FEF786FB19E0012EA1
:103FF80009D102230093631C0293019612203146D3
:104008000322334609E07EB9012102230093631895
:1040180002930191112003220B460DF0F7F803E0FB
:104028000025284604B070BD2046FEF7A1F80246D8
:1040380001200023211800930125FEF75DFBF0E71E
:10404800AB16002043150020031500202A17002076
:10405800FE14002086190020C03100204E150020D3
:10406800DA1600202DE9FF4704460D46754821461B
:104078001FF079F88146002840F0DF80214671481A
:104088001FF05BF8704821461FF062F86F4E0DBBB9
:1040980001274FF00208E3190293424603203946EC
:1040A8003B46CDF8008001970DF0B0F8327862B148
:1040B8000DF0A2FB024630B1337840461E33009320
:1040C80021462A4604E0009000E00092404621463E
:1040D8003B4628E0012D2BD15D4B04F5E4408D30A3
:1040E8001F5D0DF015F807F00F07874209DA631C0A
:1040F800022202930E2029462B46009201950DF0CC
:1041080085F8327892B10DF077FB024638B14F4B03
:104118000D201B7821461E330093002202E00090F8
:104128000D2021460123FEF7E7FA5EE00092F7E74B
:10413800022D0BD101230193E31802931420494661
:104148002A464B4600950DF061F84EE0032D4CD100
:1041580001272A464FF0020804EB070A4D2039468A
:104168003B46CDF800800197CDF808A00DF04EF839
:1041780035783DB30DF040FB024630B13378404608
:104188001E33009321464A4602E0009021464046ED
:104198003B46FEF7B1FA0DF02FFB671C054648B108
:1041A8002046FDF7E5FF337802461E3300931A20B8
:1041B80039462CE02046FDF7DBFF009502463946DC
:1041C8001A202DE021462A463B4640460095FEF738
:1041D80093FA2046FDF7CCFF514602462B461A209B
:1041E8000095FEF789FA384628E03578EDB10DF0EC
:1041F80003FB04F11C06054658B12046FDF7B8FF3D
:10420800124B02461B7830461E330093611C002374
:1042180007E02046FDF7ACFF009502463046611CDA
:104228002B46FEF769FA012008E02046FDF7A0FFBB
:104238000095024604F11C00F1E7002004B0BDE837
:10424800F08700BFD2160020DA16002032170020AF
:10425800E9150020064B1B1893F84001492804D0A3
:10426800452814BF0320022070470120704700BF73
:10427800E82300202DE9F041244F00243C70244815
:1042880021461EF070FFE5B2224B002837D01E5D94
:104298003B789E4200D303B93E70002E30D13146A0
:1042A8001C484022FCF776F81B4B1C4803EBD5034F
:1042B80093F8888104F0070348FA03F8214608F0C8
:1042C80001081EF050FF68B9B8F1000F02D0284667
:1042D800022101E028463146FFF7C4FE28460DF0CA
:1042E80071FB0DE0B8F1000F0AD12846FFF7B2FFC5
:1042F8000B4BDB7803F02003DBB20BB9094B1855E5
:104308000134402CBBD1BDE8F08100BF321700203A
:1043180030150020EA160020E8230020D2160020DD
:10432800C03100204E1500202DE9F04F914B89B087
:104338001B7813F0010F06D08F4B1A786FF3861293
:104348001A7001F069BA8D498D4A0B7810788D4D35
:10435800984218BF8C49137018BF0B706B7803F024
:104368000803DBB24BB143F6CF200CF0D1FE864BED
:1043780018702B886FF3CB232B80844B1B78AA2BC8
:1043880008D18349AA3B0B702B8843F080032B800C
:1043980000F09CBE6A787B4B02F01002D2B27D4CD2
:1043A800A2B11A886FF30C321A807B4B1B7823B9A1
:1043B8007A4B1B7813F0010F08D1E37803F0200340
:1043C800DBB21BB9764B032283F840202368754F74
:1043D8006FF3186323603A7802F00202D2B232B95E
:1043E8006B494A781AB16B4A43F080731360E678D8
:1043F80016F0010648D05D20FFF7D4F900285AD1FD
:104408006B78DFF8808103F00203DBB22BBB5D30F1
:10441800FFF780F8064600BBB8F80030012143F4E6
:104428000073A8F80030042303220093019302903C
:104438000B460D200CF0EAFE45200DF0C3FA31467C
:10444800012233460D200096FEF756F90920314621
:10445800324601230096FEF74FF96B7803F002030A
:10446800DBB243B34C4B1B7823B94C4B1B7813F08E
:10447800010F20D1E37803F02003DBB2DBB9484B0E
:10448800032283F8402016E06B7803F00203DBB2C6
:104498006BB13146324601230A200096FEF72CF90B
:1044A8008D203146012233460096FEF725F92B88E8
:1044B8006FF349232B802368354A6FF359632360D0
:1044C80093787BB1D37823B93B7813F00C0F05D1DF
:1044D80008E03B7803F00C03042B03D0236843F077
:1044E80000732360E17801F00201C9B200295BD0B2
:1044F8005E20FFF757F9002865D16B78214F03F04C
:104508000403DBB2EBB95E30FFF704F80646C0B926
:104518003B88012143F480633B80042300930133EB
:104528000322019302900B4617200CF06FFE4520E2
:104538000DF048FA0D203146012233460096FEF769
:10454800DBF86B7803F00403DBB2002B3BD0124B93
:104558001B7823B9114B1B7813F0010F33D1E37883
:1045680003F02003DBB273BB0D4B032283F840201A
:1045780029E000BF41180020F8330020B5160020BC
:10458800B6160020C816002033170020AB160020EE
:10459800600E0020C0310020FE1400208619002083
:1045A8004E150020E62300206B7803F00403DBB2ED
:1045B8002BB18D2001220B460091FEF79DF82B8828
:1045C8006FF38A232B802368DFF8DCB26FF3DF7385
:1045D80023605F2307930026D94696E03046394684
:1045E8001AF092FA002871D01BF80A30FF2B6DD010
:1045F8004FF4A0727243A8F15E03DBB206930A235C
:1046080003FB072219F802E009EB02035FEADE1E4A
:1046180050D02268404642F0004222600593FFF7DE
:10462800C1F8059B00285CD11A7912F0040F24D137
:104638004046FEF76FFF059B8446F0B91A79322091
:1046480042F004021A710699042300930291DB18C0
:104658000121032201930B46CDF814C00CF0D6FDBE
:104668004A200DF0AFF9DDF814C00C20069901229C
:104678006346CDF800C0FEF73FF84FF4A0737343CC
:104688000A2202FB07334B441B7913F0040F28D08E
:10469800804B1B7823B9804B1B7813F0010F20D176
:1046A800E37803F02003DBB2DBB97C4B032283F809
:1046B800402016E01B7913F0040F07D08C200699D0
:1046C80001227346CDF800E0FEF716F84FF4A07308
:1046D80073430A2202FB07334B441A796FF38202B1
:1046E8001A71013708F10108202F5FFA88F80AF1DA
:1046F8000A0A7FF473AF079A013602F12003DBB28E
:10470800022E0BF5A07B079305D04FF0000ADDF8C9
:104718001C80574662E72368614923F080636FF382
:104728009E7323600B79002B00F024845D4ADFF828
:104738007CB106924FF09F0800271BF8011F3E46E8
:104748000137002952D02368A8F15F0A43F080633B
:104758005FFA8AFA23605046FFF724F800285CD1F4
:1047680029237343DFF8489119F8032012F0100F3A
:1047780023D150460593FEF7CDFE059B8246E0B94E
:1047880019F80320012142F0100209F8032004233C
:104798000093023301933BB2032202930F200B468E
:1047A8000CF034FD45200DF00DF90D205146012285
:1047B8005346CDF800A0FDF79FFF2923734319F84E
:1047C800033013F0100F28D0324B1B7823B9324B2B
:1047D8001B7813F0010F20D1E37803F02003DBB23C
:1047E800DBB92E4B032283F8402016E029237343BC
:1047F800DFF8BC9019F8033013F0100F05D08D20A6
:1048080001220B460091FDF777FF2923734319F81E
:1048180003206FF3041209F80320069A12F8011F07
:104828000692002946D02368404643F0804323601F
:10483800FEF7B8FF002854D14FF0290909FB06F903
:10484800DFF86CA01AF8093013F0200F49D1404660
:10485800FEF760FE0646002843D11AF80930012108
:1048680043F020030AF8093004230093033301932B
:104878003BB2032202934B200B460CF0C7FC50209E
:104888000DF0A0F819203146012233460096FDF7B5
:1048980033FF26E0FE140020861900204E15002064
:1048A800600E0020BB32002065360020E032002078
:1048B800EB32002029237343DFF80C9319F80330F7
:1048C80013F0200F05D0992001220B460091FDF727
:1048D80013FF29235E4319F806306FF3451309F8CF
:1048E800063008F10108042F5FFA88F87FF425AF35
:1048F800AE4ADFF8D8B206924FF05008043F1BF8D2
:10490800011F3E460137002952D0236808F1620A88
:1049180043F080635FFA8AFA23605046FEF742FF4D
:1049280000285CD122237343DFF8A49219F80320EE
:1049380012F0400F23D150460593FEF7EBFD059B7F
:104948008246E0B919F80320012142F0400209F833
:10495800032004230093023301933BB20322029302
:1049680069200B460CF052FC45200DF02BF80D2069
:10497800514601225346CDF800A0FDF7BDFE222383
:10498800734319F8033013F0400F28D0884B1B7875
:1049980023B9884B1B7813F0010F20D1E37803F07B
:1049A8002003DBB2DBB9844B032283F8402016E0F6
:1049B80022237343DFF8189219F8033013F0400FDD
:1049C80005D08D2001220B460091FDF795FE22238C
:1049D800734319F803206FF3861209F80320069A27
:1049E80012F8011F0692002935D02368404643F08B
:1049F80080432360FEF7D6FE002843D14FF02209FA
:104A080009FB06F9DFF8C8A11AF8093013F0200FDE
:104A180038D14046FEF77EFD064698BB1AF80930A5
:104A2800012143F020030AF80930042300930333DB
:104A380001933BB20322029310200B460CF0E6FBD5
:104A480050200CF0BFFF1920314601223346009652
:104A5800FDF752FE16E022237343DFF8749119F82C
:104A6800033013F0200F05D0992001220B46009146
:104A7800FDF742FE22235E4319F806306FF3451313
:104A880009F8063008F10108022F5FFA88F87FF468
:104A980036AF4A4B1978002946D02368AE2043F038
:104AA80080632360FEF77EFE00284CD1444B1A78C1
:104AB800984612F0400F20D1AE30FEF72BFD074686
:104AC800D8B998F80030012643F0400388F8003040
:104AD80004230093023331460322019367203346AF
:104AE80002960CF093FB45200CF06CFF0D20394624
:104AF80032463B460097FDF7FFFD98F8003013F06B
:104B0800400F20D02A4B1B7823B92A4B1B7813F06F
:104B1800010F18D1E37803F02003DBB29BB9264BD1
:104B2800032283F840200EE0254E337813F0400F1F
:104B380005D08D2001220B460091FDF7DDFD33786D
:104B48006FF3861333701F4B1978002942D02368FE
:104B5800572043F080432360FEF724FE002848D105
:104B6800174E337813F0200F43D15730FEF7D2FC9D
:104B7800074600283DD13378032243F020033370E1
:104B88000423012600930333314601931F20334643
:104B980002960CF03BFB50200CF014FF192039460C
:104BA80032463B460097FDF7A7FD22E0C3310020BF
:104BB800FE140020861900204E1500201C3200200B
:104BC8003532002021320020EB320020AD320020A7
:104BD8006A3200209E4E337813F0200F05D09920BA
:104BE80001220B460091FDF787FD33786FF34513DB
:104BF80033704FF000094FF0A70AC8464E46954B50
:104C080008F10108F15C00294ED02368AAF14C0B89
:104C180043F080635FFA8BFB23605846FEF7C2FDC2
:104C2800002854D12A2373438B4FFA5C12F0200FCB
:104C380022D158460593FEF76DFC059B8346D8B9EB
:104C4800FA5C012142F02002FA5404230093023353
:104C580001930FFA88F30322029320200B460CF0ED
:104C6800D5FA45200CF0AEFE0D20594601225B46D0
:104C7800CDF800B0FDF740FD2A237343FB5C13F029
:104C8800200F24D0754B1B7823B9754B1B7813F074
:104C9800010F1CD1E37803F02003DBB2BBB9714BE1
:104CA800032283F8402012E02A2373436A4FFB5CF7
:104CB80013F0200F05D08D2001220B460091FDF73F
:104CC8001BFD2A237343FA5C6FF34512FA54664BB3
:104CD800F15C002936D02368504643F080432360B6
:104CE800FEF760FD002842D15B4B4FF02A0B0BFB0F
:104CF800063B9BF8013013F0200F38D15046FEF7E1
:104D080009FC0746002832D19BF80130012143F005
:104D180020038BF8013004230093033301930FFA27
:104D280088F3032202934C200B460CF06FFA5020B4
:104D38000CF048FE1920394601223B460097FDF742
:104D4800DBFC14E0444F2A2303FB06735B7813F063
:104D5800200F05D0992001220B460091FDF7CCFCCD
:104D68002A2303FB06777B786FF345137B703F4B51
:104D78001B78002B00F090803D4B374FF35C2A22C4
:104D8800002B77D002FB06F3FA5C07EB0901C2F3AC
:104D9800801BBBF1000F1BD142F04002FA5478226D
:104DA80004234A800093DB18012101930FFA88F34A
:104DB800032202932E200B460CF028FA46200CF012
:104DC80001FECDF800B00920414601225B4661E0B2
:104DD800B1F9021029BB5FEAD21B22D143F6DE20CB
:104DE80005930CF095F9059BD8B1FA5C012142F0C6
:104DF8008002FA5404230093DB1801930FFA88F316
:104E0800032202932F200B460CF000FA47200CF0E7
:104E1800D9FD0920414601225B46CDF800B0FDF7D7
:104E28006BFC2A237343FB5CDB0935D00B4B1B78E7
:104E380023B90B4B1B7813F0010F2DD1E37803F046
:104E48002003DBB243BB074B032283F8402023E057
:104E580035320020B9320020C8310020FE1400206D
:104E6800861900204E150020B13200202A32002079
:104E7800233200207243B95C11F0400F0CD063F369
:104E8800861163F3C711B9544F447B80892000937E
:104E980041460122FDF730FC01360AF1010A022ED3
:104EA80009F12A095FFA8AFA7FF4A9AEDFF8B4A1FA
:104EB8004827023E1AF8013FB04601362BB9614B2C
:104EC800F31813F8011C002937D02368384643F03B
:104ED80080432360FEF766FC002847D14FF037096E
:104EE80009FB08F9DFF880B11BF8093013F0200F2F
:104EF8003CD13846FEF70EFB8046002836D11BF819
:104F08000930012143F020030BF8093004230093F2
:104F18000333019333B20322029313200B460CF0A0
:104F280075F950200CF04EFD1920414601224346E8
:104F3800CDF80080FDF7E0FB18E0372303FB08F30A
:104F4800DFF8249119F8033013F0200F05D09920C9
:104F580001220B460091FDF7CFFB372303FB08F82E
:104F680019F808306FF3451309F808300137042E93
:104F7800FFB29FD1A37803F00803DBB2002B40F007
:104F8800A58048F67254A4F50C47A7F5B9772E48C2
:104F980039461EF0E8F830B92C4839461EF0E3F8D7
:104FA800002800F08D802A4839461EF0DCF80028D9
:104FB80040F08680394626481EF0BFF820460CF09F
:104FC800A7F8244EC0B23070002879D00138C0B29A
:104FD80030700AF093FC002872D130781E4E00F52C
:104FE8006A5078300CF094F81C4BC0B2E31813F8F0
:104FF800B28C307000EA0808394613481EF0B3F83E
:10500800DFF868A0DFF8589038B1104839461EF02C
:10501800AAF810B99AF800302AE00C4839461EF070
:10502800A2F838B1084839461EF09DF810B99AF828
:10503800003004E09AF8003018EA030F18D023EA89
:10504800080817E05D320020CC230020D42300207C
:10505800DC230020E0150020D6180020E897FF1F69
:10506800401800206532002024340020FE1400205F
:1050780048EA0308A648A74989F80080A64AFEF727
:1050880075FDA448A54912F0D1FA68B10CF0B4FB3B
:1050980050B9A24809F0F6F930B901239F48A04950
:1050A8009C4A0093FEF738FD0023009301330193D7
:1050B8003378974802939749974A994B09F070F9C2
:1050C800013448F6B2539C427FF45DAF954E737835
:1050D8006FF3C71373702B7803F08002D2B2002AE3
:1050E80000F0C38090490C78002C40F0BE8003F09B
:1050F8002403042B0BD1FEF769FCFF230093402007
:10510800214601222346019402940CF07FF82B8853
:1051180000246FF3C7136FF3820364F3451364F33A
:10512800410364F30003814A64F3492364F38A2347
:1051380014702B807E4B1A7842F0C0021A705A788D
:1051480064F3C3025A70FEF721FD7A481DF0B0FFE0
:1051580079481DF0ADFF79481DF0AAFF4122784833
:105168002146FBF717F9774B1A7802F0DF0264F350
:1051780004121A7093F8292002F0DF0264F3041273
:1051880083F8292093F8522002F0DF0264F3041216
:1051980083F8522093F87B2002F0DF0264F30412B4
:1051A80083F87B20684B1A7802F0DF0264F38612DA
:1051B8001A7093F8222002F0DF0264F3861283F853
:1051C8002220624B1A7864F345121A7093F837203C
:1051D80064F3451283F8372093F86E2064F3451280
:1051E80083F86E2093F8A52064F3451283F8A52070
:1051F800574B1A7802F0DF0264F386121A70554B87
:105208005A7864F345125A701A7802F07F0264F3F0
:1052180045121A7093F82B2064F3451283F82B205B
:1052280093F82A2002F07F0264F3451283F82A20BB
:1052380011E04FF4A07262430A2101FB03224649A0
:1052480001338A181179202B6FF382011171F0D183
:105258000134022C01D00023EBE704223F4800214F
:10526800FBF798F83E4B00221A703E4C2378002B2F
:1052780040F08A8029783C4A01F00201C9B201B3A2
:105288003A49487863F3820048702948118847787A
:1052980063F34D3163F3C30741F080014770118018
:1052A800CA201EF085FDC6201EF082FD1EF0CEFD30
:1052B8001D4A13780BB90CF011FCFEF70DF9FEF737
:1052C80007FE2B4A2B8811786FF341036FF3000117
:1052D8006FF3000311702748002140222B80FBF751
:1052E80059F825481DF0E4FE24481DF0E1FE134856
:1052F8001DF0DEFE22481DF0DFFE042217480021C3
:10530800FBF748F8164A002313701E4A1370A6E0EC
:1053180040180020161900200A1900200B1500203B
:105328000518002040150020600E0020AC16002053
:10533800F83300202A17002003150020301500201C
:105348004E150020EB3200206A3200202434002061
:1053580035320020C8310020653600202415002091
:10536800FC140020FE140020C81600200F34002072
:1053780002150020EA1600202D290020A31600207F
:10538800E2160020321700202F7807F00203DBB264
:1053980093B917F001070FD176481DF089FE2378DD
:1053A800F8B23B4113F0010F03D0FEF72BFA0CF0D3
:1053B80019FA0137042FF2D12B786F4F13F0010F30
:1053C80025D0FEF729FD3B8843F002033B80FEF71A
:1053D800BBFA6A4B93F80080B8F1000F14D1CA20C9
:1053E8001EF0E6FCCD201EF0E3FC3B88644868F321
:1053F80000033B80634B1A7842F001021A701DF0DB
:1054080057FEFEF769F802E00120FEF7FFFB2B7854
:1054180003F00202D2B212B35B4A12782AB113F037
:10542800010F02D10220FEF7F1FBFEF723FF5749D7
:1054380057481DF05BFE564956481DF041FEFEF7E1
:10544800BFFB534954481DF03BFE544952481DF0D8
:1054580042FEFEF74FFB52484D491DF052FE4B49A4
:1054680050481DF02DFE50490B780BB9FEF7D0FAC5
:10547800737803F08003DBB2CBB9FEF745FD30B19A
:1054880043F6EC200BF044FE08B106200DE0FEF7D1
:105498000DFD08B1052008E00CF00AFC08B1032056
:1054A80003E001F08BF810B10420FEF7AFFB3F4B8F
:1054B8001B781BB173786FF3C71373703C4A13786A
:1054C80013B13C4B1B78CBB12B782B4E03F0440324
:1054D800402B13D10021BF3300933F200B460222FB
:1054E800019102910BF092FE338843F6CE2043F0EF
:1054F800040333800BF00CFE2F4B18702C492F4EF1
:105508000B789BB12B4B197881B92A781A4B02F08A
:105518004002D2B252B11A8861F382021A803378FB
:1055280023B943F6CE200BF0F3FD30702A78DFF86C
:10553800488002F00400C0B2214B002800F0AA8085
:1055480002F02000C0B21C4F00283BD01A7800207F
:1055580042F0C0021A70FDF7B1FE3B78002B40F014
:105568009F80B8F8002063F3820263F34512A8F81D
:10557800002095E02D290020C8160020FC140020EA
:10558800E1150020021500203217002043150020E5
:10559800A316002030150020D216002090150020F8
:1055A800E216002028150020600E00207E3B002017
:1055B800B516002033170020AC1600204D1500202A
:1055C800F8330020D20052B219789211D2B241F0C9
:1055D800C00112F0010F197003D0C9B260F3C711EE
:1055E800197012F0020F03D01A786FF386121A702E
:1055F8001B788B4A03F04003DBB273B9537843F04E
:1056080008035370237843B12B8843F400532B804D
:10561800844B5A7842F004025A700120FDF74EFE7E
:1056280043F6CD200BF074FDC0B20128307002D1D2
:105638007D4B02221A703C78002C31D1FEF7C6F956
:10564800FF2301220093402021462346019402941F
:105658000BF0DCFD2B8843F6CD2043F020032B8094
:105668000BF056FD714B724A1870724B14701A7811
:105678000AB1013A1A70197891B96F4A13787BB157
:10568800FF230093412002220B46019102910BF067
:10569800BDFD05E01A7842F0C0021A70FDF70EFE53
:1056A8000CF0B6FA65481DF031FD654B18B91A784B
:1056B80060F3820202E01A7842F004021A706A78F3
:1056C800604812F001011A780CBF61F3410242F000
:1056D80002021A705C491DF014FD5C4959481DF01E
:1056E800FAFC58485A491DF0F6FC3378012B40F073
:1056F80093802B8800246FF349236FF38A232B8030
:10570800494B41221C7021465248FAF743FE524841
:105718001DF0CEFCFEF73AFA4C481DF0C9FC4C4887
:105728001DF0C6FC4D4B1A7802F0DF0264F3041238
:105738001A7093F8292002F0DF0264F3041283F848
:10574800292093F8522002F0DF0264F3041283F850
:10575800522093F87B2002F0DF0264F3041283F8EE
:105768007B203F4B1A7802F0DF0264F386121A702E
:1057780093F8222002F0DF0264F3861283F82220D5
:10578800384B1A7864F345121A7093F8372064F38B
:10579800451283F8372093F86E2064F3451283F896
:1057A8006E2093F8A52064F3451283F8A5202E4BAC
:1057B8001A7802F0DF0264F386121A702B4B5A78BB
:1057C80064F345125A701A7802F07F0264F34512A6
:1057D8001A7093F82B2064F3451283F82B2093F862
:1057E8002A2002F07F0264F3451283F82A2011E090
:1057F8004FF4A07262430A2101FB03221C490133C2
:105808008A181179202B6FF382011171F0D10134BC
:10581800022C01D00023EBE709B0BDE8F08F00BFF0
:10582800F83300200F3400204D150020AC1600205E
:10583800600E002033170020B516002098150020B0
:1058480002150020B22D0020D216002003150020DA
:105858002A1700204E15002030150020EB320020BA
:105868006A3200202434002035320020C83100205C
:10587800653600202DE9FF4104460D460CF0F2F98B
:10588800A04B1A1992F880709F4A98461278AA2A53
:105898000AD1A7F14F03DAB20B2A00F2AD819B4A75
:1058A8005BB29A4040F1A881994B0C2202FB043369
:1058B8005A7A0833AA42C0F09F81FF2A00F09C81DF
:1058C800FF229A70934808EBD403214693F8885135
:1058D8001DF049FC0646002840F08E8104F00703BD
:1058E8001D41502F05F0010500F0268114D8462FE0
:1058F80000F0F28009D8412F00F09E80452F00F07B
:105908001B812D2F40F0768134E0482F00F0C580B0
:105918004F2F40F06F810EE0542F67D006D8522FDA
:1059280000F08A80532F40F065811CE0A7F15903ED
:10593800012B00F25F81784821461DF014FC0646D1
:10594800002840F059815A2F01D1744802E0592F9C
:1059580004D1734821461DF0F0FB54E121466F48FD
:105968001DF0EBFBF5E76F4821461DF0FCFB002816
:1059780000F042816C4821461DF0F5FB8046002866
:1059880040F03A81214668481DF0D7FB6748214618
:105998001DF0DEFB0227012655B1A419142041464B
:1059A8003A4643460097019602940BF02FFC2AE1F1
:1059B80029463A46334604F101080A200097019621
:1059C800CDF808800BF022FC2046FCF7D1FB4146BD
:1059D80002462B4613200095FCF78EFE38462946D2
:1059E8002A4633460095FCF787FE0CE14E482146CF
:1059F8001DF0B9FB0746002840F005810126022268
:105A080031463346A5193E200092019602950BF0C7
:105A1800FDFB2046FCF7ACFB294602463B4614201A
:105A28000097FCF769FE21463F481DF086FB21469A
:105A38003E481DF08DFBE6E03A4821461DF093FBF9
:105A48000646002800F0DF80374821461DF08BFB12
:105A5800064628B92046FDF75DFD002840F0D380B2
:105A6800002D40F08E802046FEF7FAF9002840F01D
:105A7800C5802046FEF7EEFB2D4BDB7803F02003B4
:105A8800DBB20BB92B4B1855412F00F08880522FF1
:105A980040F0B0802046012183E0234821461DF0D4
:105AA80062FB28B92046FDF735FD002840F0A480A8
:105AB800002D66D12046FEF7D3F9002840F09E80DD
:105AC8001B4BDB7803F02003DBB2002B67D1194BAB
:105AD800032283F8402062E0134821461DF043FB6F
:105AE800064628B92046FDF715FD002840F08B80B2
:105AF8002046FEF7B5F900287ED1002D41D1204679
:105B080003214EE0E8230020AB160020000030807F
:105B1800BC25002043150020DC230020CC230020D6
:105B2800D4230020A3160020D2160020DA16002065
:105B3800C03100204E150020354821461DF013FBCA
:105B4800064600285FD02046FDF7B6FE20B1214664
:105B580030481DF0F2FA4FE0502F28D12E4B1B7819
:105B68002BBB2046FDF794FE08BB2C4821461DF0B0
:105B7800FAFA064620B92046FDF7CCFC002842D1A7
:105B880015B1204602210CE02046FEF763FB244BAA
:105B9800DB7803F02003DBB20BB9224B1855204603
:105BA8000021FEF75FFA061E18BF01262BE02046EB
:105BB800FDF76EFE0546F8B91B4821461DF0D3FADD
:105BC8000646D8B92046FDF7A5FC0746D8B91648B9
:105BD80021461DF0B2FA154A135D8BB910494E786B
:105BE80006F02006F6B26EB908EB040393F800310C
:105BF800135508E0012606E0002604E02E4602E0E0
:105C08003E4600E01E46304604B0BDE8F08100BFC5
:105C1800A3160020E115002032170020D21600201C
:105C2800C03100204E15002030150020EA16002053
:105C3800032210B505490648FAF782FE05480649C9
:105C48000222BDE81040FAF77BBE00BF27210020E2
:105C580004020020090200202521002070B57F4B96
:105C68001B7813F0010F0AD00BF0CEFD38B10020DD
:105C78007B4902F087FE7B4B7B48197847E07B4DD8
:105C88002B78002B48D00BF0C5FD002844D0784B6A
:105C98001B7863B9774B5B7813F0010F07D00BF0D3
:105CA800ABFD20B9FEF730F908B10320B6E0724C1D
:105CB800207870B10020714902F064FE2178012239
:105CC8006F4802F085FE00201021621C08F06AF877
:105CD80002E06C4902F056FE6B4C644808F088F804
:105CE8002378002B00F00F810BF08EFD002800F0C8
:105CF8000A81664966481022FAF722FE64485B2149
:105D0800FAF7C6FB002800F0FE80217801308322D4
:105D1800BDE8704002F05CBE5E4C237803F00503DA
:105D2800012B5DD100205C4902F02CFE20211022BD
:105D38005A48FAF72FFB601D59490322FAF7AAFDC2
:105D480040BBE01C57490222FAF7A4FD30B9564877
:105D5800FAF770FD5449024650480BE0E01C5349DD
:105D68000222FAF797FD40B95148FAF763FD504906
:105D780002464A48FAF7E4FD0EE0E01C4D490222CB
:105D8800FAF788FD30B94C48FAF754FD4A490246FB
:105D98004248EFE7FFF74CFF6278303AD3B2092B5D
:105DA80000F2B1803B4B9B78303BDBB2092B00F211
:105DB800AA800A2101FB0231C9B2002900F0A380A0
:105DC800334BFF220C291A7740F29D8010295A770D
:105DD80040F2998013299A7740F29580DA7770BD5E
:105DE800234E3378F3B9234B5B7813F0010F19D0A6
:105DF8000BF002FDB0B931481DF088F968B1304C9C
:105E0800304B226802EA03033BB918F07FFA20B945
:105E1800E37803F04003DBB223B10020BDE8704013
:105E280009F04CB8337863B90BF0E6FC48B1264B5F
:105E38001B7803F00603042B03D02B780BB9012041
:105E4800ECE7FEF733F810B10020204957E0204B6B
:105E58001C78002C40D01F4951E000BFC816002014
:105E68003D1A0308FC14002000020020FE14002044
:105E7800D4180020861900202218002050EF0208AC
:105E8800050200200EEF0208321700202FEF02084B
:105E9800F40100202221002057F402080402002007
:105EA800607D0308647D0308BAF40208677D03086F
:105EB80099F402086A7D030878F40208981500200E
:105EC800C03100203000000F02150020E001030857
:105ED800650E002071EF02080B4802F002FD0A4827
:105EE80002F0F6FC094802F0F3FC1BF0BBFD084B7E
:105EF800DB7803F02003DBB22BB106492046BDE86E
:105F0800704002F03FBD70BD181900204C180020E9
:105F1800C031002069EE0208054B1B78D8019B01AF
:105F28005BB2DB1140B243EAE070C0B2704700BF19
:105F3800C816002070B50E4686B0410001220546FD
:105F480001F5E97105A80BF0F4F80021012E8DF890
:105F580015104FF0FF0205F1010305D100920191E0
:105F680002930920FB3A04E00092019102931E205B
:105F780004220B460BF04AF905A83D49FAF70EFB37
:105F880050B105A83B49FAF709FB28B105A83A49D9
:105F9800FAF704FB002867D105A83749FAF7FEFA93
:105FA800364B0446F8B95A78214642F010025A7026
:105FB800FF23022200930190FE3B02903D200BF04C
:105FC80025F94D200BF0FEFC691C01222346122006
:105FD8000094FCF791FB12202146224601230094ED
:105FE800FCF78AFB03E05A786FF304125A70002416
:105FF800E0B2552115F0DCFB38B12846214615F0F2
:1060080078FD10B1204615F063FD0134082CEFD15E
:106018003EBB1B481B491C4AFDF7A8FD19481B49F4
:1060280011F004FB68B10BF0E7FB50B9174808F012
:1060380029FA30B9012315481549124A0093FDF78A
:106048006BFD144B0F491D7000230093053301931A
:10605800114B0D4A1B780A4802930D4B08F0A0F922
:1060680002E00E4B00221A7005A806B070BD00BFF2
:10607800F17D03086D7D0308FD7F0308F8330020D8
:1060880040180020161900200A1900200B150020BE
:106098000518002013340020D618002023150020EE
:1060A80007B54100012201A801F5E9710BF041F89B
:1060B800002301A804498DF80530FAF76FFAD0F1EA
:1060C800010038BF00200EBDF17D030807B541006F
:1060D800012201A801F5E9710BF02BF8002301A8B2
:1060E80004498DF80530FAF759FAD0F1010038BFA4
:1060F80000200EBDBA7F030870B5154B04461B1867
:1061080093F88050B1B1134821461DF02CF888B996
:10611800114821461DF011F8A5F15903DBB2012BF6
:106128000CD94F2D0AD0542D08D021460B481DF00C
:1061380004F807E0084821461DF00AF807482146F8
:106148001DF006F804480649BDE870401CF0B8BFC9
:10615800E82300204315002098150020381500205A
:10616800E2160020024B1878C0F38000704700BF89
:1061780002150020024B1A8860F308221A80704723
:10618800C8160020034B5878C00140B2C011C0B2F5
:10619800704700BFC8160020014B1878704700BF31
:1061A800FE14002030B5457800230021C2189170F4
:1061B80055FA03F111F0010F08D0064959188C7CE3
:1061C800017804EA0101A14208BF91700133042B50
:1061D800EBD130BD2218002046F6F54104220AF022
:1061E800A8BF000070B5104C0546112220460021BA
:1061F800FAF7D0F8002004F8010C2A78103414F8C3
:10620800011FC3B291420BD152B10849013301F8C1
:10621800013B112246F64573BDE8704002F0FEBA14
:1062280001300428EBD170BD23180020221800206B
:106238001FB520B1134B1A8842F480521A80124BB2
:1062480000245A78214642F010025A70FF23022295
:1062580000933D20FE3B019402940AF0D7FF4D20A5
:106268000BF0B0FB20210122234612200094FCF7FA
:1062780043FA12202146224601230094FCF73CFAF7
:106288001FBD00BFC8160020F83300202DE9F341D8
:106298002D4C0722E37848F6085702FB003348F6EE
:1062A8002950DBB218180AF033FF257964795FFAB0
:1062B80080F8002648FA06F313F0010F3AD0394661
:1062C800042201A80AF035FF9DF804009DF8053066
:1062D8009DF806109DF8072000282BD0002929D00A
:1062E800002B27D0002A25D0934204D19C4221D1EB
:1062F80085421FD30FE09A4210D99C421AD3944288
:1063080018D89C4201D994421AD39C4201D18542A3
:1063180016D294420ED18D420CD811E09C4201D184
:1063280085420DD2944201D18D4209D99C4207D8A9
:10633800944205D301360437082EBBD1002000E073
:106348000120BDE8FC8100BFEC38002010B50446F0
:1063580048F6615000EBD4000AF0DAFE04F00704B6
:10636800C0B2204100F0010010BD70B5C30848F666
:1063780061555D19044628460E460AF0C9FE04F028
:106388000704C0B2012126B9A14040EA0101C9B2FF
:1063980002E0A14020EA01012846BDE870400AF069
:1063A800ADBE0000F0B57D4B8DB0DD78042200EB6A
:1063B800C505EDB2E90001F5F24104A890310AF0F3
:1063C800B8FE774B774E1A78002304A9C95C3129A7
:1063D80005D13039994041EA0202D2B205E03029AC
:1063E80003D12F39994022EA01020133042BECD161
:1063F80032706C486C496D4AFDF7B8FB6A4B1B78E4
:1064080013B96A4B1B78F3B16748694911F00EF963
:1064180068B10BF0F1F950B9654808F033F830B9B4
:10642800012363486349604A0093FDF775FB002325
:10643800009302330193FD3302935A485A495B4A49
:106448005C4B07F0ADFF05EB0511002401F5F641A3
:10645800347004A8503108220AF06BFE2646E0B2D8
:10646800542115F0A5F9002838D004AB1B5D312B59
:1064780003D1204615F032FA38B104AB1B5D302B3E
:106488002CD1204615F02AFA40B34EB9FF230093C9
:106498003420314604223346019602960AF0B6FEAD
:1064A80004AE305D2146303815F026FA335D0126FA
:1064B800312B4FF0030306D10093A3191BB20196A9
:1064C8000293352005E00093631C1BB201960293EA
:1064D8003620002104220B460AF098FE0134082CCD
:1064E800BDD1A90101F5FE4104A8083120220AF016
:1064F80020FE083C04AD274615F8013BE6B20134FE
:10650800302B03D13046FFF721FF38B115F8013C95
:10651800312B2CD13046FFF719FF40B34FB9FF2379
:1065280000933420394604223B46019702970AF02B
:106538006DFE15F8011C30463039C9B2FFF715FF5A
:1065480015F8013C0021302B4FF0FF0305D10093D3
:1065580023B201910293372004E0009323B2019102
:106568000293382004220B460AF050FE0127202C03
:10657800C2D1114D6B7803F00403DBB263B1203C48
:106588002046FFF7E3FE38B90134E4B2202CF7D1F6
:106598006B7860F382036B700DB0F0BDEC380020AF
:1065A800FE14002040180020161900200A190020A7
:1065B8000B15002005180020F8330020014B18782F
:1065C800704700BF650E00202DE9F04F4E4B0022AA
:1065D8001A704E4A85B01678002E40F091804C4BC8
:1065E8004FF4B468DA78997808FB02F24FF03C0867
:1065F80008FB01285A78474F90441FFA88F8BA4692
:106608006CE03AF815303C24DAB2544304EB132416
:106618004C44A4B2042CEEB207D842F25A739845FF
:1066280003D904F51C546034A4B2444511D948F682
:1066380028500AF06DFDC8EB0403834209DC364B91
:106648001A787B1993F83830934302D02E490123E6
:106658000B702F4AD378B34232D142F26073B4FB45
:10666800F3F203FB12439BB2434523D12B4B9B7898
:1066780013F0090F44D12A4B5B7803F08003DBB297
:10668800002B3DD1274B5B7803F00203DBB2002BD4
:1066980036D1254B1A781BEA020F11D101990098BF
:1066A80041EA02021A70FFF7F1FD48B90098FFF7B6
:1066B80079FE05E01C4B02991A7801EA02021A7069
:1066C800013509F5B469072D1FFA89F999D1039E97
:1066D80007370136042E0AF10E0A11D04FF0010BCC
:1066E8000BFA06FB5FFA8BF301936FEA0B03F2B226
:1066F800DBB24FF00009009202934D46039680E703
:1067080005B0BDE8F08F00BF650E002039170020E6
:10671800EC3800203A170020FE140020C031002079
:1067280007340020AA2B00203817002073B50C4628
:1067380001EBC001C9B2C90001F5F24105460422C6
:1067480001A890310AF0F5FC104B002003EBC402BD
:10675800121B521982F8380001AA125C312A0AD198
:106768000121814003EBC402121B521992F83860D0
:10677800314382F8381001300428EDD101A93122C3
:1067880030231CF0F8FCC0B27CBD00BF3A170020D3
:1067980000B501EBC001C9B2890189B001F5FE411C
:1067A8000831202268460AF0C4FC202069463122BC
:1067B80030231CF0E0FCC0B209B000BD07B501EB06
:1067C800C001C9B201EB011101F5F64150310822AF
:1067D80068460AF0AEFC08206946312230231CF0D6
:1067E800CAFCC0B20EBD00002DE9F84300263446AD
:1067F8002BE021462846FFF799FF21468146284687
:10680800FFF7C6FF214640EA09092846FFF7D6FFE9
:106818005FFA89F949EA000010F0FF0F05D04046F9
:10682800394602220AF085FC03E04FF0FF33A8F84E
:1068380000300135EDB20237072D08F10208D8D132
:106848000134E4B20E3E042C07D0054BC6F5F247DE
:10685800C6EB030820370025CBE7BDE8F88300BF67
:106868003A17002010B521F085F94FF4803021F057
:10687800A1F921F0B9FA0128044628D1102021F005
:106888009BF8022021F08CF8002021F0D3F9002099
:1068980021F0E4F94FF4806021F0D6F94FF440403C
:1068A80021F0E6F94FF480304FF4E01121F09EF921
:1068B800204621F0A7F9392021F082FA0028FAD0E1
:1068C800022021F0A5F921F0ADF90828FBD17C20A0
:1068D800012121F03FFA46F60120012121F03AFA80
:1068E8000C48012121F042FA0B48012121F03EFA1F
:1068F8000420012121F03AFA7E2021F061FA38B112
:1069080021F088FA054B04211A7861F344021A70C1
:1069180010BD00BF0340060020080818613B002096
:1069280010B50C46014620B110220C48FAF708F8B9
:1069380004E00A4820211022F9F72CFD34B1084858
:1069480021461022BDE81040F9F7FABF044820217B
:106958001022BDE81040F9F71DBD00BFF40100206A
:106968000402002010B5FF2B1446029A03D04218E7
:1069780002F8013C08E06FF07F439A4204D01314F8
:10698800437013128370C27019F0A8FF02E07F20D1
:1069980021F05CFD19F08EFF0028F8D1ACB10B484E
:1069A80090F82010163001F00F0119F097FF02E05F
:1069B8007F2021F04BFD19F07DFF0028F8D1044B12
:1069C80093F8693013F0010FE9D110BD900C002045
:1069D8007C3A002010B50A4B002203EBC003013BB0
:1069E8001046084951184C7813F8011F8C4205D1FC
:1069F8000130C0B20C320828F3D1F73010BD00BF07
:106A08001E850208BC25002070B50D4C05460E46B3
:106A18004FF4007200212046F9F7BCFC2A463146A3
:106A280004F50070F9F70EFC642024F8035C1BF0F1
:106A3800EBFA0023A4F82D33024B64221A6070BDD0
:106A4800E53B00202C21002010B5054C00212046F4
:106A58004FF40072F9F79EFC0023A4F82D3310BD03
:106A6800E53B0020164B2DE9F0415D8A0746284694
:106A7800FBF756F81349FBF75FF9134B134E1860F1
:106A8800D723B5FBF3F5EDB2822229460446F01967
:106A980001F09EFF2846FBF747F801462046FAF723
:106AA8008DFF0B49FBF794F8FBF758FA0337BE192B
:106AB800C1B281223046BDE8F04101F089BF00BF74
:106AC800F82800200000574390170020F401002008
:106AD800000020410000000070B54B4D2868FAF70F
:106AE8002BFC45A3D3E90023FAF7C6FAFAF712FFFD
:106AF800FAF722FC42A3D3E90023FAF771FC3EA37C
:106B0800D3E90023FAF796FDFAF704FFFAF714FC25
:106B1800FAF71EFAFAF7FEFE3C4906462860FBF72C
:106B2800FFF920B13046FBF719FAC4B25EE03046EF
:106B38003649FBF709FA50B130463549FBF7F0F909
:106B480028B13046FBF70AFAC0B2441C4EE0304682
:106B58002F49FBF7F9F950B130462E49FBF7E0F918
:106B680028B13046FBF7FAF9C0B2841C3EE0304643
:106B78002849FBF7E9F950B130462749FBF7D0F926
:106B880028B13046FBF7EAF9C0B2C41C2EE0304603
:106B98002149FBF7D9F950B130462049FBF7C0F934
:106BA80028B13046FBF7DAF9C0B2041D1EE03046C2
:106BB8001A49FBF7C9F950B130461949FBF7B0F942
:106BC80028B13046FBF7CAF9C0B2441D0EE0304682
:106BD8001349FBF7B9F948B130461249FBF7A0F958
:106BE80020B13046FBF7BAF9C0B2841D0A2021460D
:106BF800BDE870400AF082BA736891ED7CFF7F406F
:106C08000000000080842E419417002000001041ED
:106C18000000F0410000484200008E420000B842E7
:106C28000000E0420000F2422DE9F04FA1B019F057
:106C3800EBFD09201BF084FB1BF06AF94FF461405F
:106C48001BF0BAFB09201BF037FC0022A3484FF4C5
:106C5800804120F016FFA248002121F0DFFAA14967
:106C680004224B78DFF8A0E26FF300034B709E4BD1
:106C78009E4C1A705A715A709A70DA701A719A7119
:106C8800DA719B4B033A1A709A4B00201F328EF828
:106C9800000020705A7105900546069006467F2030
:106CA80021F0D4FB23780E2B01F2B681DFE813F034
:106CB8000F004F009500E0007902DE0330048504E0
:106CC800EA06DC07EF075808B108D00882098A4E9F
:106CD8008A48317801F00F01013149014118FFF765
:106CE8001FFE337813F00F0308D1854A92F8012369
:106CF800012A41F09181834A138024E0012B03D1BA
:106D08007F4B93F819330BE0022B04D17C4B93F89B
:106D18000D33032B05E0032B06D1794B93F80D3384
:106D2800012B41F079810EE0774901220A707748FA
:106D38004FF4007120F0A5FE754BC8221A60337815
:106D48006FF30303BFE333785A1C01F05FB8704B4D
:106D58001A6822B96D484FF4007120F092FEDFF8EE
:106D680098816C4898F8001001F00F010131490131
:106D78004118FFF7D5FD36B198F800305A1C62F378
:106D8800030388F800305F4B00221A8098F800103F
:106D980001F00F02022A03D11A7842F010020AE029
:106DA800042A03D11A7842F0040204E0052A05D126
:106DB8001A7842F040021A7001F02EB9062A04D15E
:106DC8004D4B6FF3030119707EE301F00F010122AF
:106DD80012FA01F1198001F01FB9474E4E48317877
:106DE80001F00F01013149014118FFF799FD96F8AB
:106DF800008008F00F08B8F1070F27DC18F0010F22
:106E0800464B02D00020588002E04FF0FF315980F5
:106E18004FEA6809062209F1010902FB09394FF016
:106E2800FF32A9F802204046FFF7D4FDFF2806D01C
:106E38003B4B03EB40005823437401F0EDB80023AB
:106E4800A9F8023008F1010801F08AB800211022DF
:106E58001BA8F9F79FFA17A800211022F9F79AFA48
:106E680023780133237033786FF3030301F07BB881
:106E7800DFF884A09AF8008018F00F0840F03F81EE
:106E8800284E337803F04003DBB2F3B926486FF09D
:106E98007F43817A0122009301F00F01FF23FFF75E
:106EA80061FD224B93F8692012F0400F08D093F847
:106EB8006C3013F0040F03D0337843F04003337081
:106EC8007378142262F3C7037370737813F0F80FA2
:106ED80030D0174800F12001A7E300BF0018014097
:106EE800002C01401A290020E82300209A170020CE
:106EF800630E0020EB320020991700205E850208FF
:106F0800BC250020F83300205C210020000C014043
:106F18002C210020FE850208DE860208B2330020FC
:106F2800F4010020AB310020900C00207C3A0020B6
:106F3800FE870208BC4B1B7803F04003DBB2002B32
:106F480000F0D980DFF80483DFF8049398F8003064
:106F580013F00C0B30D1B54E6FF07F4396F82B1021
:106F680006F12100009301F00F0101220523FFF72C
:106F7800F9FC96F84C104FF4860A06F1420001F02D
:106F88000F010122FF23CDF800A0FFF7EBFC96F8D4
:106F98004110FF2306F1370001F00F015A46CDF8E2
:106FA80000A0FFF7DFFC042389F8003098F80030D0
:106FB80043F0080301F02EB803F00803DBB2002BFE
:106FC80039D099F800A0BAF1000F03D0984800F121
:106FD800400138E0954E6FF07F4B717D06F10B0054
:106FE80001F00F010122FF23CDF800B0FFF7BAFC32
:106FF80096F82B1006F1210001F00F01012207235A
:10700800CDF800B0FFF7AEFC96F836104FF48603C3
:10701800009306F12C00FF2301F00F015246FFF701
:10702800A1FC98F800306AF3C303DBB243F0040311
:1070380088F800305AE099F800C0BCF1000F08D079
:107048007B4800F16001FFF76BFC99F800203032B3
:1070580008E2764E6FF07F40717DFF23009001F0CB
:107068000F0106F10B000122CDF80CC0FFF77AFCE6
:107078009AF80030DFF8C4B103F0100A5FFA8AFA10
:10708800DDF80CC0BAF1000F0CD098F800206CF3B2
:10709800820288F800205A1C62F303038BF8003040
:1070A80000F0BABF96F82B106FF07F42009206F1FD
:1070B800210001F00F0101220C23FFF753FC96F881
:1070C80036104FF4860300935246FF2306F12C0036
:1070D80001F00F01FFF746FC9BF8003083F0100227
:1070E800C2F3001262F304138BF80030042389F80A
:1070F800003000F091BF4E4800F1800195E2B8F1F0
:10710800010F3CD14A4800F1A001FFF709FC002E0D
:1071180000F082879AF80030444E5A1C62F3030349
:107128008AF8003096F82B106FF07F4906F121009D
:1071380042460F2301F00F01CDF80090FFF712FC33
:1071480096F82B1006F1210042460E2301F00F019C
:10715800CDF80090FFF706FC96F82B1006F12100F9
:10716800424601F00F010F23CDF80090FFF7FAFB1C
:1071780030488021424620F084FC00F04DBF2C4866
:1071880000F1C001FFF7CCFB002E00F045872A4B29
:1071980096221A609AF800306FF303038AF80030D9
:1071A80092E1264E317811F00F0A16D1244800F1E9
:1071B8002001FFF7B5FB204B1B68002B40F02C8704
:1071C8001BA8F9F737FB4022134601461BA801F01C
:1071D80023FA3378012200F019BEBAF1010F39D130
:1071E80012486FF07F4390F8201000220093163069
:1071F80001F00F01FF23FFF7B5FB01F077FA002834
:1072080000F00A873378022262F3030333700D4BD0
:107218001A7842F080021A700B4B5A7842F0020238
:107228005A7000F0F9BE00BFAB310020900C00206E
:10723800FE870208001001402C2100209917002029
:10724800DE880208B03100208E3500200042002080
:107258008743002001F00F0101F10E0303F00F0333
:10726800012B44D89B4849014118FFF759FB9A481C
:107278006FF07F4390F8201000221630009301F041
:107288000F01FF23FFF76EFB1AF08AFC337803F037
:107298000F03022B13D117F005F8002800F0BC8665
:1072A8008E4B1A7842F040026FF304121A705A7823
:1072B8006FF345125A703378032200F0A7BD16F019
:1072C800DBFF78B117F07AF816F032FF844B002014
:1072D8001A7858816FF3C7121A703378042262F350
:1072E800030333707F4B1A786FF3000263E5BAF13A
:1072F800040F4DD1DFF8DC914901DFF810824944D1
:107308004846FFF70DFB98F80010774B01F0040290
:10731800D2B27AB941F004016F4883F800A088F826
:10732800001090F836104FF4860300932C3001F0CB
:107338000F01EEE293F800A0BAF1000F40F06C865E
:1073480065486FF07F45417D01220B3001F00F0148
:10735800FF230095FFF706FB64480122817AFF238B
:1073680001F00F010095FFF7FDFA98F800300522AB
:107378006AF3820388F800303378484662F30303DF
:10738800337009F1A001FFF7CBFA554600F044BE6F
:10739800DFF84481FF2398F8201000226FF07F491E
:1073A80008F1160001F00F01CDF80090FFF7DAFAA6
:1073B8002BB2072B18D1337808F121006FF30303A0
:1073C8003370237801220133237098F82B100E2391
:1073D80001F00F01CDF80090FFF7C4FA444880216E
:1073E800002220F04EFB0025424E96F86B3013F039
:1073F800040F00F0118698F857106FF07F430022B1
:1074080000933D48FF2301F00F01FFF7ABFA96F810
:107418006B303A4A03F00F03012B137003D1002D90
:1074280008BF01250CE0022B04D12BB2012B08BFA9
:10743800032505E0032B03D12BB2032B08BF072537
:10744800ABB213F0010F02D02D4A3121517713F05E
:10745800020F02D02A4A3221917713F0040F00F06C
:10746800DB853322264BDA7700F0D6BD1948254E46
:1074780000F1C001FFF754FA96F80090DFF85C803D
:1074880019F00F090CD116F06DFD98F8003069F36A
:10749800000388F8003033785A1C62F30303337012
:1074A80016F0F2FD98F8003013F0010F00F0B485E3
:1074B80000221548802120F0E4FA0A4B00225A7075
:1074C800337862F30303337023780133237000F0B9
:1074D800A3BD00BFDE880208900C00208E35002076
:1074E800B03100200635002087430020010000202D
:1074F800001001407C3A0020DD0C0020AA31002059
:10750800F4010020991700200018014000420020D3
:107518008648874E00F1E001FFF702FA17A8F9F74D
:1075280089F917A902468348F9F70AFA002182481F
:10753800B18090F8C5106FF07F4300220093BB30F4
:10754800FF2301F00F01FFF70DFA7C4A92F86B1048
:1075580092F86C30327843EA012312F0010FB380BD
:1075680010D0A3F1EB0292B20A2A04D9A3F5E6736C
:107578009BB2282B02D8F3880133F38033786FF35A
:10758800000333707378002B40F04685684AD28830
:107598007AB16B4A1FA8117863F30301117022783E
:1075A8008DF87F300132227028228DF87C2020F05F
:1075B80087FA0022F28000F02FBD624EDFF8ACA1FE
:1075C800337803F004085FFA88F8B8F1000F15D192
:1075D80011A841461522F8F7DDFE5B4BCAF800807A
:1075E8001B684546CDF847303368474643F00403E7
:1075F8003360564BA3F8368300F00EBD03F08003CA
:10760800DBB2002B67D1DAF80010002940F00485BE
:107618004F48FFF785F94F484FF4805120F027FA7B
:10762800012806D04A4800F1A001FFF779F900F0D7
:10763800F3BC4649B1F83623002A43D009314648FD
:10764800013AF9F77DF9444B03F1100113F8012BC6
:107658000D2A01D00A2A02D1202203F8012C8B42DC
:10766800F4D13E4B4FF03C0808FB073808F11E08E0
:107678004046F9F7DFF8414602463948F9F70AF972
:10768800D8B9022F03D1336843F0100304E0032F65
:1076980003D1336843F040033360327853005BB260
:1076A80003EAC263DB173268DBB263F3C7123260E6
:1076B8001BB1FFF7C9F900F0AFBC0137FFB2042FC7
:1076C80008BF0227254B3C2606FB07363046F9F74C
:1076D800B1F8314626E0DAF80080B8F1000F40F042
:1076E8009B84737803F02002D2B2002A40D11D4B4C
:1076F80011A81A889B781C498DF84630ADF84420AB
:10770800F8F7A2FE114B5B7A302B07D1FFF79CF9F3
:10771800336843F40053336000F07EBC11A8F9F7D6
:1077280089F811A9FFF770F900F076BCDE88020825
:107738000635002008020020900C00207C3A00202A
:1077480099170020302100206F7D0308DC3B0020C2
:10775800DE89020800080140040200200C00002015
:10776800E53B0020747D0308787D03082C21002068
:1077780003F04003DBB2002B40F08980B14800F1F0
:107788006001FFF7CDF8B048F9F754F88046AE49E4
:10779800AE484246F9F77EF8002873D1AC4B434413
:1077A8005B7A302B6ED1FFF74FF93368DFF8D09250
:1077B80043F48043336099F82B106FF07F430093B4
:1077C80009F12100082301F00F010122FFF7CAF88F
:1077D8006423CAF800307F2020F038FEDAF8003041
:1077E800002BF8D1984699F88E10D633994E89F81F
:1077F80086304B3B6FF07F4A89F88730964801F016
:107808000F0142467433CDF800A0FFF7ABF896F8A5
:10781800B91106F5D670033001F00F014246FF2377
:10782800CDF800A0FFF79EF896F8C41106F5DD70B4
:1078380001F00F014246FF23CDF800A0FFF792F8B0
:1078480096F8CF1106F5E270013001F00F014246BB
:10785800FF23CDF800A0FFF785F896F8DA1106F5B2
:10786800E87001F00F014246FF23CDF800A0FFF7B2
:1078780079F899F899107948CDF800A001F00F012E
:10788800424646E07648F8F7D5FF75494AE796F844
:1078980002B0DFF8EC910BF0020B5FFA8BFBBBF147
:1078A800000F3AD199F82010FF236FF07F4809F1B3
:1078B800160001F00F015A46CDF80080FFF752F884
:1078C800684B93F86B3003F00803DBB2002B00F031
:1078D800A38399F82B10012209F1210001F00F016F
:1078E8000323CDF80080FFF73DF83368554843F48B
:1078F800003300F180013360FFF712F855485A460B
:1079080090F8E51100F5EC70CDF80080033001F037
:107918000F01FF23FFF726F87EE3CAF8008099F8E5
:1079280020106FF07F4300934246FF2309F11600B1
:1079380001F00F01FFF716F82AB241F211139A422B
:107948001DD1434B5B7A302B13D1FFF77DF8336899
:10795800454668F3514368F38E3368F34D3333601B
:10796800414B1A7868F303021A70237801332370A5
:1079780052E33E48F8F75EFF3C49FFF745F8394EB9
:1079880096F86B3013F0040F00F0468325B9384899
:1079980020211022F8F7FEFC7F2020F057FD99F8EF
:1079A80057106FF07F43002200933248FF2301F005
:1079B8000F01FEF7D7FF96F86B202F4B02F00F024E
:1079C8000D2A1A7005D125B92C4A412191754FF419
:1079D80080551A78062A08D12AB2B2F5805F04D1F8
:1079E800264A3621D1754FF488551A78082A08D1C5
:1079F8002AB2B2F5885F04D1204A3821117641F2C3
:107A080010151B780B2B09D12AB241F210139A4298
:107A180004D11A4B2A225A7641F211150D486FF0FB
:107A28007F4390F8F0110022009300F5F370FF23D4
:107A380001F00F01FEF796FF96F86B3013F0010F77
:107A4800AAD0E9E2DE8902081A010020E53B0020FD
:107A5800DC3B002001000020140D00201F0D002039
:107A6800FC0000207C3A00209917002038010020F3
:107A780004020020DD0C0020AA310020F4010020BF
:107A8800900C0020A34B1A7842B300221A700F20E2
:107A9800FAF7DAFA06460A20FAF7D6FA9E4B9F4911
:107AA80058824A7812F0010F18D06436301A588379
:107AB8009B4B1A78642A01D19B321A701B78984E16
:107AC800FF2B0BD00A21B3FBF1F1964B193119802A
:107AD800954820F0A3FB337801333370DFF86482D4
:107AE80098F8003013F00F0612D18E4B19228B48EC
:107AF8001A804378192143F0010343708A4820F023
:107B08008DFB8A4800F12001FEF70AFF04967CE20B
:107B1800012E68D1804B5A8BA2F1690189B21129D3
:107B280008D8049911F0010F04D141F00101C9B23C
:107B380004910592049A12F0020F0DD15B8A7C4AD7
:107B48001380A3F5C263023B9BB2D72B04D80498D9
:107B580040F00203DBB204931B20FEF783FF059974
:107B6800744B0AB2632A05DD642192FBF1F23032CC
:107B78001A7401E0092A0CDD059A11B2642291FBFE
:107B8800F2F002FB10120A2012B292FBF0F230322D
:107B98005A74059802B2642092FBF0F100FB11219F
:107BA8000A2209B291FBF2F002FB101230329A74E9
:107BB8005B4B1B78FF2B08D158495B484B786FF318
:107BC80000034B70002120F029FB049A032A40F09F
:107BD80023825248002143786FF3000343705248D0
:107BE80020F01CFB11E2022E03D1534BC8221A606D
:107BF8000BE2032E16D1504B1B68002B40F00C8271
:107C08004A4800F14001FEF78BFE1B20FEF72AFFD1
:107C1800414B5B8AA3F51E630F3B9BB2542B00F2CA
:107C2800FB81F2E1042E0CD13B4B988A0FF0AEF8A1
:107C3800002840F0F1813D4800F16001FEF770FE38
:107C4800E3E1052E07D1344B988A0FF09FF80328FB
:107C580040F0E281D9E1062E40F0D78122786FF317
:107C6800030301322270D5E1344800F12001FEF708
:107C780057FE334B1B78002B00F0CE81237801335D
:107C88002370304B1A786FF30302FFF794B82D4E28
:107C9800DFF8A480337813F00F021AD12A4800F1D4
:107CA8002001FEF73DFE2948F8F7C4FD27490246A2
:107CB8002748F8F7C7FA2548F8F7BCFD254BA3F87D
:107CC800160233785A1C62F3030333701AF01EFC51
:107CD80091E0012A16D1D8F80030002B40F09C81A1
:107CE8001AF040FC012840F097811B48F8F7A2FDE4
:107CF800194902461948F8F7CDFD002840F08C8153
:107D080011486FE0D8F80020002A40F085810B2147
:107D18007BE000BF660E0020F82800201A2900200A
:107D2800A81700208C0C0020002C01409E8A020815
:107D38009C170020F40100202C2100201E8B020833
:107D480098170020991700205E8B02087401002004
:107D5800982F0020803F002092010020813F0020C2
:107D6800874E337813F00F080CD186484146FEF74A
:107D7800D7FD33785A1C62F303033370824BA3F8A0
:107D8800028049E1B8F1010F18D1804804211FF0A1
:107D98006EFE002800F040817A4800F12001FEF7CD
:107DA800BFFD33784FF0FF315A1C62F30303337081
:107DB800774B64221A60744B59802DE1B8F1020F99
:107DC800DFF8CC811BD1D8F80030002B40F024819B
:107DD8006E4804211FF04BFE002840F01D816A4BBD
:107DE8005880684800F14001FEF79AFD33785A1C24
:107DF80062F3030333706423C8F800300CE1D8F849
:107E08000020002A40F008810C21217062F303034E
:107E1800A9E0604910234FF40052CB700D3B8B70E2
:107E28000A805D481FF0D4FD0A2200215B48F8F75C
:107E3800B1FA80201FF030FD237801332370504BB6
:107E48001A786FF303021A70514BC8221A60E3E0E4
:107E58005348DFF848A100F12001FEF761FD9AF8C8
:107E68000030002B00F0D8804E48DAF80020444E4D
:107E78000260BAF8042082809AF80620827131786C
:107E880011F00F0159D1DFF80881D8F80010002946
:107E980040F0C2809AF80410A2F5A6524FF0640B85
:107EA800103A0BFB01229AF805004FF00A0909FB6A
:107EB80000200393F9F734FE3B49F9F73DFF0246EA
:107EC8009AF80200039BA0F5A65010380BFB030B91
:107ED8009AF80100354B09FB00B018600392F9F7D6
:107EE8001FFE039A01461046F9F76AFD304B1860E9
:107EF800F9F722FA1EA3D3E9002382468B46F9F745
:107F0800F5FC002800F08880504659461AA3D3E9AA
:107F18000023F9F7E1FC00287ED0FEF7DDFD337879
:107F280048465A1C62F303033370C823C8F800306C
:107F380009F0EEF8C0B207906EE001296CD10D305F
:107F48000799832200F044FD114BD3F80080B8F163
:107F5800000F61D140461FF09FFC23780133237046
:107F6800337868F30303337056E000BFAFF3008043
:107F7800736891ED7CFF7F400AD7A3703D00804075
:107F880099170020BE8B0208B2330020000C014074
:107F98002C2100201629002000100140B0170020D5
:107FA8001E8C02080402002000007A44AC1700204E
:107FB800941700208448854E00F12001FEF7B0FC9C
:107FC800F37913F0010F27D0DFF8488298F8009072
:107FD80019F00F0920D17E4B0A22597818781039E8
:107FE80002FB0011B1701979D878103902FB001121
:107FF8007170D9799B79103902FB0312327017F02E
:1080080015FCF37969F30003F37198F800305A1CF2
:1080180062F3030388F80030DFF8FC9199F80060F8
:1080280016F001063EF43BAE6A4B01221A7019F0B5
:1080380047FA2378092B01D00D2B28D10120664956
:1080480011F05CFF654B664A5B7803F01F03D35C55
:10805800644A522B137002D1634B01221A70634B8E
:10806800634A03F1200153F8040B8B4242F8040BD6
:10807800F9D1002109A811F07FFF09A80D211AF0F4
:10808800E1F95C4B1A78013202F003021A7099F890
:10809800006006F00206F6B2002E00F08B800FF0AA
:1080A80023F913F0B3FB06980322431C93FBF2F267
:1080B80002EB42029B1ADBB20693002B79D1DFF860
:1080C800488198F84960C246002E4DD0022E03D14F
:1080D80098F80130312B49D023780E2B13D146481C
:1080E80046490522F8F7D6FB8246002840D1B21F40
:1080F80037484349F8F724FC344B5646DA7942F0BE
:108108000102DA7135E00D2B03D13E483A490722C6
:1081180027E0032B22D13C4B002713F8012F2C2AF0
:1081280003D00137FFB2B742F7D11BA832493A460C
:10813800F8F706FC7B1C07E00AEB03025278303A9A
:10814800D2B2092A03D80133DBB2B342F4D30AEB23
:108158000701FA4317A80231D21802E0264911A8EC
:10816800721EF8F7EDFB03E0069E02E0012600E030
:1081780000261E4B204A03F1100153F8040B8B42D2
:1081880042F8040BF9D1214B214A03F1100153F8AD
:10819800040B8B4242F8040BF9D1402388F81130C4
:1081A8001C3B88F82230023B88F84B3019F0D2FE8D
:1081B80000E0002699F8003003F0F5036FF30003A0
:1081C80089F80030FEF76BBD5E8C0208EC380020A1
:1081D8009E170020660E00201D3F00201C3F002037
:1081E8001CC202085A32002098170020F40100200F
:1081F800C1320020C73100208B3B00207B7D030863
:10820800903B0020B01700208A3B00200402002089
:108218009C3B002099170020643B0020AFF30080AE
:1082280010B5044640181146F8F7A6FA2046F8F7A4
:1082380001FBC0B210BD42540131C8B27047000002
:1082480010B50C4B0C4A1B780C460E2101FB03237E
:10825800997A31B101390523594301F56F5189B232
:1082680001E04FF46F510019042208F062FF201D4D
:10827800C0B210BDA1410020A812002010B5054BC6
:108288000C46197800190131042200F0A1FB201DC9
:10829800C0B210BDA141002000F5244000F58F7048
:1082A80008B5013008F034FF10F0FF0F14BF0020AC
:1082B800012008BD10B50A4600210446FFF7B0FFAB
:1082C80001462046FFF7DAFF114A01462046FFF72C
:1082D800A7FF232201462046FFF7ADFF01462046AF
:1082E800FFF7AEFF5B2201462046FFF7A4FF2322DB
:1082F80001462046FFF79FFF01462046FFF7A0FFF3
:108308007C2201462046BDE81040FFF794BF00BF1D
:10831800817D030810B55D220446FFF78CFF0D220E
:1083280001462046FFF787FF0023235410BD38B5C8
:108338001D460C4640182C1911461A4600F048FBF9
:10834800E0B238BD2DE9F04118490446FFF7B2FF05
:10835800174F0E263B78174D73430146EA5A2046BD
:108368000423FFF7E4FF202201462046FFF763FFBE
:108378003B78014606FB035320469A7A0223FFF70F
:10838800D6FF202201462046FFF755FF3B780146DD
:1083980006FB035520466A7A0323FFF7C8FF014608
:1083A8002046BDE8F041FFF7B5BF00BF847D030854
:1083B800A1410020A81200202DE9F047264E0E22E8
:1083C8003378264F534337F90380FA1824494FF47A
:1083D8007A73044698FBF3F8157AFFF76BFF4E2281
:1083E80001462046FFF727FF1E4B1C2202FB0535DE
:1083F8005FFA88F8B8F1030F01460CBF05F11202C5
:1084080005F108022046FFF70BFFA146804600252C
:1084180019E019F8013BA32B07D133780E2202FB90
:108428000373204629465A7A08E0242B09D1337869
:108438000E2202FB03739A7A204629460223FFF78D
:1084480076FF0135EDB24545E3D120462946BDE822
:10845800F047FFF75FBF00BFA1410020A81200202E
:108468008E7D03083CC20208074B187800F0040010
:10847800C0B240B11A686FF382021A60034B00223F
:108488001A70034B18787047C0310020D4170020A9
:10849800BC170020054B00211970054B05481A68C8
:1084A80061F382021A601222F7F774BFD417002012
:1084B800C0310020BC17002038B5084C0849227884
:1084C8000546F7F7BFFE23780021E954054B1A68E3
:1084D80061F382021A60207838BD00BFD4170020EB
:1084E800BC170020C0310020064A07491378112B19
:1084F800C85401D801331370044A136843F00403C5
:1085080013607047D4170020BC170020C03100202A
:10851800054B1B7813F0010F05D1044B181810F800
:10852800010CFFF7E1BF7047D51700209E8C0208A9
:108538002DE9F041334C002314F8101094F82A2048
:1085480001F00F0161F3030284F82A2004EB4000D4
:1085580084F8293084F828304378DFF8B88063F34A
:108568000712638C4FF4D277E38498F800302A26F8
:108578007B4306FB0133244D2448E95A84F82A201A
:108588001FF04AFE98F8003094F82A207B4302F046
:108598000F0206FB0233EB1859881C48013989B2CF
:1085A8001FF03EFE01210A4618481FF005FE012172
:1085B80016481FF0F2FD98F8003094F82A207B4303
:1085C800120906FB02331248E95A1FF025FE98F8F3
:1085D800002094F82A3057431B0906FB0376AD198F
:1085E80069880B48013989B21FF018FE01210A4633
:1085F80007481FF0E1FD06480121BDE8F0411FF0E2
:10860800CCBD00BFD6170020AA8C02080008004085
:10861800003401400218002030B5164C94F82B5055
:10862800A38445F00105002384F82B50628484F864
:10863800211084F8203019E0C55CA5F13002D2B2CF
:10864800092A08D9A5F14102D2B2052A9ABFA5F193
:108658003702D2B22A46084D013305EB420292F89E
:10866800495392F84823257062700234DAB28A427C
:10867800E2D330BDD6170020AA8C0208124B10B5E1
:108688009A8C0024DA8483F8294083F8284022460B
:1086980001210E481FF090FD64210C481FF0BCFD1D
:1086A80032210A481FF0BCFD0121224608481FF06C
:1086B80083FD642106481FF0AFFD05483221BDE85F
:1086C80010401FF0ABBD00BFD617002000080040C7
:1086D8000034014010B500212C220348F7F75AFE58
:1086E800BDE81040FFF7CABFD617002070B5214C6F
:1086F8002378042B39D8DFE803F0030D152A30005E
:108708001D4B012093F82B3013F0010F30D020704F
:10871800013870BD184B93F82000FFF709FF0223BA
:10872800237022E0144DEE8CFEB9FFF7A7FF95F8F1
:10873800203095F821200133DBB29A4285F82030A9
:1087480001D8042300E003232370304670BD0A4B90
:10875800D88C50B90123237070BD074BDD8C35B917
:10876800FFF7B8FF2570012070BD002070BD002004
:1087780070BD00BF03180020D6170020044B00224C
:108788005A701A709A7842F001029A70704700BFC6
:1087980018190020202102480A46F7F7FBBD00BF40
:1087A800F401002038B5044608460D46F8F742F8AB
:1087B80098B10319202B094BC8BFC4F120001C191C
:1087C800002308E014F8012BE02A14BFEA5C2022F9
:1087D80004F8012C01338342F4DB38BDF401002096
:1087E8000D4B46F6B5421B689B6893420FD043F683
:1087F800F82293420BD0122B09D0B3F5E97F08D0A9
:1088080046F659501B1A584240EB030070470120A6
:1088180070470120704700BF3C180020F0B51F4684
:1088280087B006460C46084600211546F7F7B2FD04
:10883800244B07B19F80B3F9041005A801EB86010A
:10884800042208F076FC002605AB9B5D013BDBB2F9
:10885800B92B35D81D2B4FEA031209D8D31803F5C5
:108868001641684601F5E971112208F062FC0BE037
:108878001549D3185B186A4603F110071868596838
:108888000833BB4203C2F9D12046F7F7D3FFC7B27A
:108898006846F7F7CFFF3818A84203D8E0196946A9
:1088A800F7F76AFF6846F7F7C5FF7B1C1B18AB4252
:1088B80003D2E0190549F7F7C7FD0136042EC3D1E5
:1088C80007B0F0BD18190020D4580308A67D030886
:1088D80010B500216C220446F7F75CFD0123A37054
:1088E80010BD002343700370837843F00103837045
:1088F800704700002DE9F0419378804613F0010F8E
:108908000D4614463AD06FF30003937019F0FAFA43
:108918006378002B32D123780BB90A336370A378BC
:10892800174F6FF30003A37019F0ECFA217807EBE7
:1089380008066118073130462A46F8F701F830462C
:10894800F7F778FFC6B2AE420DD80AD200232370DB
:1089580006EB08000A33637038182021AA1BF7F7C2
:1089680019FDAE420AD12278A3181B7A1BB1013235
:108978002270BDE8F08123700A236370BDE8F0819E
:10898800F4010020054B1A780AB100221A701B78EE
:1089980046F68A4202FB0311FFF704BF1F180020A6
:1089A800F8B505460C460818002108F0A7FB013C5D
:1089B800E4B26719384608F0ABFBC6B2202E03D8DC
:1089C8003846002108F09AFB0CB1202EEFD9F8BDEB
:1089D80002F00F03032B22F07F0230B5D2B20CD97C
:1089E8004FF47A7491FBF4F42025E4B2057002B1D7
:1089F80014B13034047000220130B1F57A7F05DB00
:108A08004FF47A7491FBF4F504FB1511022B0BD982
:108A1800642491FBF4F42025E4B2057002B114B18A
:108A28003034047000220130632904DD642491FB92
:108A3800F4F504FB1511012B0AD90A2391FBF3F372
:108A48002024DBB2047002B10BB130330370013063
:108A5800092904DD0A2391FBF3F203FB12113031DB
:108A6800017030BD13B5104B01461B689A899C7B79
:108A780012F0100214BF0220012034B10B4C9B7C71
:108A88002478634303FB001109B23AB10DF10600E3
:108A9800022208F04EFBBDF8060002E0084608F086
:108AA80037FB00B21CBD00BF3C180020C9180020CD
:108AB80010B50F4B1B689A899C7B12F0100214BFEB
:108AC8000221012134B10B4C9B7C2478634303FBC6
:108AD800010000B22AB108490222BDE8104008F09E
:108AE80022BB054B1968BDE8104008F007BB00BF62
:108AF8003C180020C9180020E01800203038C0B207
:108B0800092894BFFF20002070470000024B1A7804
:108B18006FF300021A7070470919002070B5FFF74B
:108B2800F5FF884B1A781E2A01D91E221A70864C26
:108B38002678254606F0F006202E72D108F05CFE55
:108B480000286ED1814B1B7833B92378C3F3031205
:108B5800013262F307135EE07D4B1B7803F080035C
:108B6800DBB2002B59D07B48F7F764FEC5B27A4CCC
:108B7800BDB1204679493246F7F7E2FE0A2D0BD8F7
:108B88002A4620467349F7F7DBFE60193146C5F1DE
:108B98000A02F7F7FFFB04E020466E490A22F7F7BE
:108BA800CFFE6F4B1B7813F0010F01D0472300E075
:108BB8002023E372684C042204F10C00A521F7F786
:108BC800E9FB684B1A7852B1FF23012A237306D9AF
:108BD800022A637303D0032AA37318BFE373624C9A
:108BE800257815F0600502D194F8A33013B95F48D1
:108BF8005F4902E05D4804F1A3010622F7F7A0FEF1
:108C08005C4B1B78452B40F08D81002D40F08A810C
:108C1800237843F08003237070BD4F48564932468D
:108C280075E12C7804F0F004102C3FD108F0E4FD35
:108C380000283BD1202251494748F7F781FE464892
:108C48004E492246F7F77CFE4D4B1B7813F0010F77
:108C580006D04C48F7F7EEFD4A4902464A4805E077
:108C68004A48F7F7E7FD494902464748F7F768FEDB
:108C7800364B1B781BB946484649102247E1444801
:108C880045491022F7F75CFE314B1B7803F080034F
:108C9800DBB22BB13B48F7F7CDFD02463F484FE02A
:108CA8003A48F7F7C7FD02463C4842E02B7803F004
:108CB800F003302B7ED108F09FFD00287AD1264C96
:108CC800202237492046F7F73BFEA521052204F16B
:108CD8000B00F7F75FFB334B1B78042B02D9FF23FC
:108CE800E37300E002D1FF23A37301E0032B02D159
:108CF800FF23637301E0022B02D1FF23237300E0FB
:108D08000BB1FF23E372284B5B7813F0600F05D09B
:108D18003F23E37223736373A373E373234B1B78BB
:108D280003F02003DBB233B11848F7F783FD02469E
:108D38001F481649EBE01348F7F77CFD02461C482C
:108D48001049E4E015190020091900205C210020D1
:108D58003021002034210020F4010020C01E030827
:108D68009841002029220020642100200E020020C2
:108D7800DBF40208041800207E1E0308C35403080D
:108D88008E3500200D560308010200202E560308D8
:108D980004020020905A0308E4540308110200203A
:108DA80080F50208E723002020290020C031002098
:108DB8000F0200202B7813F0F0030CD120225A491F
:108DC8005A48F7F7BDFD5A4B584819888322BDE821
:108DD8007040FFF7FDBD602B1ED108F00DFDD8B91E
:108DE800544920225148F7F7ABFD5348F7F722FDC5
:108DF800514902465148F7F7A3FD5148F7F71AFDC4
:108E08004F4902464F48F7F79BFD4F48F7F712FDC9
:108E18004D4902464D487AE02B7803F0F003102BB9
:108E280006D108F0E9FC18B14048494920226EE013
:108E38002B7803F0F002402A02D0502A6BD10AE0C6
:108E4800444920223948F7F77BFD0EF0CDFF044650
:108E58000EF0E8FF09E0404920223448F7F770FD9A
:108E68000BF0C0FB04460BF0E1FBFF2806D13B48A2
:108E7800F7F7E0FC39490246394817E0FD2806D1E2
:108E88003848F7F7D7FC3749024635480EE002283C
:108E980006D13548F7F7CEFC33490246304805E09D
:108EA8003248F7F7C7FC314902462D48F7F748FD25
:108EB800202107222E48F7F76DFAFE2C06D1274805
:108EC800F7F7B8FC25490246294820E0012C06D1CD
:108ED8002848F7F7AFFC27490246254817E0022C37
:108EE80006D12548F7F7A6FC2349024620480EE09C
:108EF800042C06D12148F7F79DFC204902461C485E
:108F080005E01F48F7F796FC1D4902461848BDE8DA
:108F18007040F7F715BD1B4A6FF3071313701A4B10
:108F280000221A6070BD00BF1DF50208F401002080
:108F38001A180020FCF40208FCED0208F8010020D1
:108F480006EE02080802002001EE02080F020020C7
:108F58005FF5020805550308265503084F56030810
:108F6800FD01002070560308CB5503080D56030871
:108F78000D02002047550308685503088955030862
:108F8800AA550308091900203C180020204B70B589
:108F9800F022204D1A702B7813F0010F0BD01E4CC5
:108FA800207810F0010006D11C49FFF7EBFC23786C
:108FB80043F0010323701A4E3378532B0ED1164C0D
:108FC800237813F0010F07D000201649FFF7DAFCC9
:108FD80023786FF300032370FFF798FD3378232B72
:108FE80014D10D4B1B7813F0010F0FD1FFF78EFD35
:108FF8002B780D4A43F006032B701378013BDBB244
:1090080013700A4A52F82320094B1A6070BD00BF3A
:10901800151900200919002041180020944A030856
:1090280004180020734A0308F7180020F8180020D5
:109038003C1800202DE9F0415C4BF0225C4D1A7081
:109048002A7802F01003DBB2002B2DD1594963F3C3
:1090580047120B601C462A70574A9A5C2D2A01D089
:109068000134E4B20133082BF6D1544E3A2130468C
:10907800F7F70EFA38B1801BC0B20130301821461C
:109088000222FFF7A5FC4E4B1B78452B40F08B8046
:1090980000242046013412F011FC082CF9D12B7859
:1090A80043F010032B7038E0464C237813F0010F7F
:1090B80017D1404E4448FFF70BFC404F3168384603
:1090C80001310222FFF784FC2D23BB70307846F66D
:1090D800E1633E496522FFF7A1FB237843F00103D2
:1090E800237003200D21384AFFF704FC2D78304EF9
:1090F80015F0E00541D110203549FFF743FC304B0E
:109108001B78442B0DD12B4A136801332A4903F0ED
:109118000703C95C2D29F8D01360BDE8F041FFF7BB
:10912800F5BC532B0DD132784E3B63F347123270A6
:10913800204A28491268062000FB02125380BDE825
:10914800F081232B2FD11B4B1D60337803F0EF03E5
:1091580065F347133370FFF7D9FC23781E4A43F0B1
:10916800060323701378013BDBB213701B4A52F8D5
:1091780023201B4B1A60BDE8F081104C10201949C0
:10918800FFF700FC04F110002821F7F781F950B12E
:10919800001B3178C0B20130201849098022BDE88F
:1091A800F041FFF715BCBDE8F08100BF151900209C
:1091B80041180020E018002095330020F401002019
:1091C8000418002009190020181900201F19002070
:1091D800104A0308B2330020F7180020F8180020BE
:1091E8003C180020314A0308454B2DE9F041F02294
:1091F800444E1A703378444D43F0010333702B68A2
:10920800424C9B7C022B06D1414B1B7803F0400358
:10921800DBB23BB10FE0012B0DD13E4B1B7813F0B5
:10922800010F08D108F05AFC236800206FF355534A
:109238002360394944E0A378344F03F02003DBB2BC
:10924800C3B908F04BFCF87800F02000C0B288B928
:109258002968324B897C1A7861F301021A703B68DD
:109268002D4943F400133B60FFF78CFB2C4B802205
:1092780083F843200DF03AF9804678B12B689B7C3F
:10928800012B08D1234B5B7803F01003DBB213B139
:109298000020244914E00020234911E00DF056F97C
:1092A800074610B1404621490AE00DF097F910B180
:1092B80038461F4904E01A4B93F8433013B91D4947
:1092C800FFF760FB1C4B1B78232B16D1FFF71EFC06
:1092D800337843F00603337008F000FC23686FF31B
:1092E800555323600BF0DAFF144A1378013BDBB2C5
:1092F8001370134A52F823302B60BDE8F08100BF89
:1093080015190020091900203C180020C031002040
:10931800302100208E350020B54A030893350020FF
:10932800B11C0020F74A0308D64A0308394B030842
:10933800184B03085A4B030804180020F71800209C
:10934800F81800202DE9F3416E4B6F4DF0221A708A
:109358002B686E4C9B7C1BB9637843F0100302E0CA
:10936800637843F008036A4E6370337843F001036F
:109378003370238823F47E6323F01E03DB04DB0CA5
:10938800B3F5805F08D0634B1B7883B15F4B5B7884
:1093980003F00803DBB253B1637800206FF3410395
:1093A8005D496370FFF7EEFAF8F78AFE84E06378A8
:1093B800564F03F00203DBB2FBB9BB78EBB9574B4E
:1093C80093F8008018F0010817D1F8F779FE7B7838
:1093D80043F002037B702B68B3F91030022B7B78C3
:1093E8000CBF43F0040368F3820300217B7008205C
:1093F80001220B460091F9F77FF9A378434A032B22
:1094080028D003D8012B0BD00DD806E0052B2DD082
:10941800517825D3FF2B32D12BE000203E4949E07B
:1094280000203F4946E03F48F7F704FADFF82C816F
:10943800C7B23C4908F110003A46F7F781FA0F2FF6
:109448003AD807F1100040442021C7F11002F6F77E
:10945800A1FF31E0344B187800282DD1334929E099
:109468006FF3410151700020314923E00020314958
:1094780020E06FF34101517000202F491AE0053BAD
:10948800DBB26FF34101022B517002D100202B494E
:1094980010E0012B02D1002029490BE0032B02D157
:1094A8000020284906E0052B02D10020264901E0CA
:1094B80026490020FFF766FA637803F00203DBB25F
:1094C8000BB9F8F7FDFD224B1B78232B18D1FFF7BA
:1094D8001DFB3378002243F0060333706378A270D3
:1094E80003F0E50362F382036370F8F7E9FD194AB4
:1094F8001378013BDBB21370174A52F823302B6004
:10950800BDE8FC81151900203C1800209841002076
:1095180009190020BA2D0020B54A03089E410020F1
:10952800F8460308A74100209C410020194703087A
:10953800BD4B03089D470308004803083A47030842
:109548005B4703087C470308BE470308DF47030857
:1095580004180020F7180020F8180020F401002053
:109568007B4B2DE9F341F0227A4E1A7033787A4D0D
:1095780043F0010333702B68784C9B7C022B11D18C
:10958800774B1B7803F04003DBB293B1754B1B7824
:1095980003F02003DBB2BBB1A37803F04003DBB2D6
:1095A8003BB111E0012B0FD16F4B1B7813F0010F6A
:1095B8000AD1F8F785FD2368002023F480036FF3B0
:1095C800D753236069498FE0A778DFF8908107F0C7
:1095D8004003DFB2002F34D1F8F772FD2968644BDD
:1095E800897C1A78384661F301021A70D8F800307D
:1095F8005E4943F4800367F3D753C8F80030FFF798
:10960800C1F92B68198A21B90091082001220B465B
:1096180015E00BB2022B0CD101223B46082039463B
:109628000097F9F769F8534B1A7842F008021A7054
:1096380007E0012B05D100970E2039463A46F9F785
:109648005BF80CF053FF074678B12B689B7C012B25
:1096580008D1454B5B7803F01003DBB213B100204F
:10966800454941E0002045493EE0414B39461878DC
:1096780000F00300F8F75CFEFF280FD13D4B1B7884
:1096880003F01803182B31D0A07800F08000C0B286
:1096980010B138463A4927E03A4925E00CF056FF20
:1096A8008046E0B1334B187800F008085FFA88F874
:1096B800B8F1000F0AD1F8F78FFFC0B2022801D81D
:1096C80040460AE0062811D8404604E000F01000A1
:1096D800C0B210B138462C4906E02C4904E00CF021
:1096E8007DFF18B12A494046FFF74CF9294B1B78F2
:1096F800232B29D1FFF70AFA337843F00603337096
:10970800F8F7DEFC236823F480036FF3D753236054
:10971800184B1A786FF3C3021A701F4A1378013B6B
:10972800DBB213701D4A52F823302B60104B1B78A4
:1097380003F00303022B02D10CF0AEFE20B102B0FD
:10974800BDE8F0410BF0AABD02B0BDE8F08100BF52
:1097580015190020091900203C180020C0310020EC
:1097680030210020642100208E350020B54A0308EE
:1097780093350020401A0020F74A0308D64A030808
:10978800BD4B0308DE4B03089C4B03087B4B0308C7
:10979800184B030804180020F7180020F8180020B8
:1097A80010B5FFF7B3F9124B2522DA77114B124C9B
:1097B8001B682A219A7C01FB0242517801F00F00B4
:1097C8000F2814D00A2803DD0A2060F30301517022
:1097D8009B7C2A2202FB034463780A2103F00F03CF
:1097E800594306485932BDE81040FFF7F1B810BD9B
:1097F800F40100203C180020C8310020100200208D
:109808002DE9F74F984BDFF8B0A2F0221A70DAF87A
:109818000030D0469C6847F25B33E11A4C4244EB77
:109828000104C63A6243914B9D5C9F18C5F300053D
:10983800EEB29946002E29D130468D49FFF7A2F89D
:109848008C4B1B78232B40F038857B7866F3041308
:109858007B70FFF75BF9884B1A7842F006021A70A2
:10986800864A1378013BDBB21370854A52F82330DD
:10987800CAF80030834B1D70834B1D70834B1D70DD
:10988800834B1E60834B1D7000F017BD824E814DC7
:10989800337893B1814A4FF4A071137803F01F0015
:1098A8005B0959430A2303FB00137D49CB18DB7876
:1098B800002B40F06682137084E06E4B1B78532BAC
:1098C80040F0FC8095F80080B8F1000F2ED140469A
:1098D800214615F062FB5FFA80FABAF1000F25D035
:1098E8007B7868F304137B706E4F3A781AB9204678
:1098F80015F06AFA13E0531E6B49002B184603EA69
:109908000101B8BF02F11E004011002903DA013934
:1099180061F01F01013115F0A3FA00233B7015F027
:10992800CFFB85F800A00022594BE2E02B78002BF2
:1099380000F0278256490A680F460B2A01D10C23EA
:1099480016E00C2A11D1013B6101544A59181170D3
:10995800554903EA0101002903DA013961F01F01C1
:109968000131204615F07CFA1CE0092A02D10A23AD
:109978000B60D0E10A2A27D14B49013B03EA0101D8
:10998800002903DA013961F01F010131204615F081
:10999800A9FA2B786201D318DBB2404A591E11701C
:1099A800404A13704FF00008C7F80080FFF7AEF880
:1099B8002A2303FB04935A7842F010025A7085F860
:1099C800008014233370DCE1043A042A3FD8374975
:1099D800D2B20878364F60B300200870397841B1A8
:1099E8003448401810F8010C032802D0002840F031
:1099F800C881013B0A2058434FF4A07E0EFB0400A7
:109A0800DFF89CE070448018417160011B18D8B2DF
:109A180000EB800000F5EE40DF30801807F06EFBA9
:109A2800387818B1013815F0B3FBAAE10DF008FD3C
:109A3800A7E101200870013B0A214B434FF4A071B4
:109A480001FB04331649CB189A1853790AE00F4FD3
:109A58003B7823B901223A700A4A137091E1FFF763
:109A680055F800233B708CE115190020C8310020FF
:109A78004B0303080418002009190020F7180020D8
:109A8800F8180020211800204A180020C9180020C2
:109A9800E0180020D318002018180020CA18002049
:109AA80065360020851900201F000080DF1800207F
:109AB80084190020E82300203C180020432B1AD1E9
:109AC800964A1278002A40F043812B78002B00F048
:109AD8005881934B1A78002A40F05381914B1968AA
:109AE8000C2903D00A2903D02A7014E10B2200E0C4
:109AF80009221A600FE1232B7ED1884A1278002AA6
:109B080040F026812978DFF818A2002935D09AF884
:109B1800003053B184490F2B0A7084490A7000F24F
:109B2800308101338AF800302BE17E4A1368082B14
:109B38001ED84FF4A077674301394FF00A0E0EFB89
:109B480001717B4F181F7918C9780627013907FB5F
:109B58000101784800EB810151F8040F0133002816
:109B680040F0D880032B40F2D580082BF4D9D1E0FF
:109B7800092B40F006810233CCE07B786E4E61F30E
:109B880004137B7032781AB9204615F01DF913E0DA
:109B9800531E6A49002B184603EA0101B8BF02F1B7
:109BA8001E004011002903DA013961F01F0101315B
:109BB80015F056F90023337015F082FA0DF040FCC9
:109BC800FEF7A4FF5E4B1A7842F006021A705D4A4F
:109BD8001378013BDBB213705B4A52F82330524AC8
:109BE800C8F8003000231370504A8AF80030137008
:109BF8004C4A2B70136060E32A2B3CD1474A1278F9
:109C0800002A40F0A58046490B784BB14648012B05
:109C180002704648027040F2B480013B0B70B0E01D
:109C28002878002800F0AD803E4A1368002B00F029
:109C3800A880092B1AD84FF4A071614301384FF05E
:109C48000A0E0EFB00103A491F1F0818C17806209B
:109C5800013900FB0171374800EB810151F8040D0F
:109C6800013B002856D1032BF8D853E00B2B40F0CA
:109C78008880023B4EE0442B1AD1284A1278002AE9
:109C880066D1274B1B78002B7BD12878431EDBB28B
:109C98001E2B76D8214615F080F9C0B2002870D066
:109CA800204A13680C2B6CD00A2B6AD028701BE052
:109CB800552B4DD1194A1278002A49D1184B1B78D7
:109CC800002B5ED1287801285BD90238214615F08F
:109CD80075F9C0B2002854D0124A13680C2B50D022
:109CE8000A2B4ED019490870043B042B13D84FF4A3
:109CF800A071614301380A2707FB00100C490818B6
:109D0800C1780620013900FB01330A4951F8233094
:109D18000BB904331360FEF7F9FE32E0DF180020B8
:109D2800C9180020E0180020211800204A18002037
:109D380065360020840D0020851900201F00008052
:109D480009190020F7180020F8180020D31800205F
:109D5800303BDBB2092B14D89C4A1268043A042A17
:109D68000FD89B4A117861B99A4A12784AB19A4A2F
:109D78000A27107807FB0033DBB2402B137088BF2B
:109D880011702F78DFF8B482002F5FD198F80000A7
:109D980010F0010012D114B92046904900E0904912
:109DA800FEF7F0FD98F8003043F6DF2043F001039A
:109DB80088F8003007F0ACF98A4B1870337813B97B
:109DC80089488A4901E0884889490A22F6F7B8FD96
:109DD800204615F0D1F8874D0146022205F11900F9
:109DE800FEF7F6FD844B1B7803F08003DBB22BB340
:109DF800824B1B88EB81337803BB814B18781A465A
:109E080018B9204614F0ACFF18E07E4B411E01EA59
:109E18000303002B03DA013B63F01F0301334FF404
:109E2800A07161430A2505FB03137749CB18DB783A
:109E380013B915F073F801E0002313702A2303FB0C
:109E48000494637843F01003637036E24FF4A07310
:109E58006343013F0A2202FB07336B4EF31893F862
:109E680003B06301FF1898F80030FFB213F0010F38
:109E780046D16648FEF72CFD07EB071101F5E641D0
:109E88005F311022624807F054F9604B594811229B
:109E98009A7144230370173BC370791C01300F3A41
:109EA800FEF796FD494B1B6813B9102059491FE06E
:109EB800012B02D1102058491AE0022B02D11020A0
:109EC800564915E0092B02D11020554910E00A2BFC
:109ED80002D1102053490BE00B2B02D1102052491C
:109EE80006E00C2B02D11020504901E05049162001
:109EF800FEF748FD98F8003043F0010388F8003079
:109F0800334B1A789846002A00F0EB8007EB0717C6
:109F180007F5E6475F3710223648394607F009F952
:109F280000229146334B995C9A4641B109F10109E7
:109F38005FFA89F90132B9F1100FF3D106E003EBAA
:109F480009002021C2F11002F6F724FA98F800005F
:109F580048450BD90138C01907F0DAF830B91C4B5D
:109F6800202118780138C01907F0C8F8DFF8D09018
:109F780099F8003018460193FEF7C0FD4A46019B48
:109F8800DFF8C09018B9432B40F0858001E0432BDF
:109F980004D1002389F80030202173E0DFF8A8E01D
:109FA80024499EF800C024489C454FD10B78ACF159
:109FB800300C0133DBB24FF00A0E0B700EFB0C3382
:109FC800C35C002B54D10B7052E000BFE018002096
:109FD800C9180020DF18002084190020F0030308A6
:109FE80074040308B0320020FA01002019050308A0
:109FF8003A050308F4010020C0310020A57D0308BC
:10A00800851900201F0000806536002018190020DF
:10A018001F190020420603082106030863060308E7
:10A02800CE070308EF0703081008030831080308E0
:10A03800520803084A18002018900208091900203D
:10A0480004180020211800201E1800208EF8003067
:10A0580099F800304FF0000C81F800C043B198F82F
:10A0680000300F2B04D803F1010E954B83F800E064
:10A07800402389F8003013780978303B0A2202FB24
:10A088000313C15C98F8000001380AF8001038186A
:10A0980007F034F80EE08B4B1B7803F08003DBB23B
:10A0A80043B199F800302BB998F80030FF22534497
:10A0B80003F8012C99F8003013B1834A013B13705F
:10A0C80099F80030012B11D198F800300F2B02D8E5
:10A0D8007B4A013313707D4A002389F800301370DE
:10A0E80004E004200C217A4AFEF704FC794B1F682F
:10A0F8001FBB4FF4A07254432B780A22013B02FB8A
:10A108000344361975782D090F2D00F0D680724C4E
:10A11800A52104F11C00063AF6F73CF9FF23237742
:10A12800002D00F0CA80012D637700F0C680022D53
:10A13800A37700F0C280E377BFE0012F18D14FF476
:10A14800A07254432B780A21013B01FB03443619C2
:10A15800737803F00F030F2B00F0AF80092B04DC9A
:10A1680001335E485943BD3AA2E05C4859436AE06E
:10A17800022F38D10BF1FF3B5FFA8BFBBBF1070FC6
:10A1880098BF574BDFF850819CBF5B4493F86470CD
:10A1980008F11B0088BF002720210522F6F7FAF8EE
:10A1A8002878C7EB08080138002318E04FF4A0729C
:10A1B80062430A2101FB0022B25C08EB07011A4145
:10A1C80012F0010FC7F1000202D08A18DB2101E06A
:10A1D8008A18A52182F82010013308F10108DAB2A3
:10A1E800BA42E3D369E0032F2FD14FF4A07254434E
:10A1F8002B780A25013B05FB0343F218F35C13F0A7
:10A20800400F02D01020374906E093785A1ED2B288
:10A21800FD2A06D93449102003B0BDE8F04FFEF7F7
:10A22800B1BBFE2B02D110203049F5E71020304990
:10A23800FEF7A8FB2F4B30481B78013B05FB034476
:10A248002E4D2C19A178832232E0043F042F34D8F4
:10A258000622FFB20BF1FF3B02FB0B7B284B294880
:10A2680053F82B100A31F6F76BFB274B1B7893B189
:10A27800144B1B7803F08003DBB23BB12348202149
:10A28800022203B0BDE8F04FF6F784B8204B1F4810
:10A29800197882220CE02B780A22013B53434FF4B1
:10A2A800A07202FB04343619F71918487979BE3AB6
:10A2B80003B0BDE8F04FFEF78BBB03B0BDE8F08FED
:10A2C800C9180020C0310020211800204A18002099
:10A2D80018190020E0180020F40100200F020020C7
:10A2E800189002088C07030884060308A5060308CB
:10A2F800AD070308D318002011020020653600209E
:10A30800840D002004020020DF1800201202002023
:10A31800841900202DE9F0474C4C4D4F2378F0224A
:10A3280043F0010323704B4BDFF85C911A703B68D4
:10A33800494A9E6847F25B33F01A464246EB0006EC
:10A348002A217143555C5318C5F300055FFA85F857
:10A358009246B8F1000F23D140464049FEF712FB60
:10A3680099F80030232B6FD1FEF7D0FB23783C4AB5
:10A3780043F0060323701378013BDBB21370394AAC
:10A3880052F823303B60384B1D70384B1D70384BEA
:10A398001D70384BC3F80080374B1D70BDE8F0873F
:10A3A80099F80020232A23D15A786FF304125A709F
:10A3B80014F086FE0DF044F8FEF7A8FB2378284A2F
:10A3C80043F0060323701378013BDBB21370254A70
:10A3D80052F82330244A3B6000231370234A137039
:10A3E800234A1370234A1360234A1370BDE8F08789
:10A3F800532A0DD15A78C2F300144CB942F0100216
:10A408005A7021463046013414F02AFD202CF8D128
:10A41800304614F0B1FD2A2303FB06A67378C1B2B7
:10A4280013F0100F0AD0202902D10020134901E0AF
:10A4380013490020BDE8F047FEF7A4BA11480222EC
:10A44800BDE8F047FEF7C4BABDE8F0870919002057
:10A458003C18002015190020C83100204B030308C0
:10A46800F7180020F8180020211800204A180020AA
:10A47800C9180020E0180020D3180020CD4D03088B
:10A48800EE4D03080D020020041800202DE9F041CC
:10A498002D4E2E4F307800F5E6403D3006F038FE60
:10A4A8003B78C4B213F0010F26D0294D2B78552BD9
:10A4B8000AD1EC2C01D0013CE4B23078214600F5F9
:10A4C800E6403D3006F01AFE2B78442B0DD1A4F15E
:10A4D8001403DBB2D72B01D90134E4B2307821461A
:10A4E80000F5E6403D3006F009FE2B78532B03D1EA
:10A4F800FEF70CFB0CF0A4FF164B1B7803F080034F
:10A50800DBB253B13B7813F0010F06D0124820217B
:10A518000422BDE8F041F5F73DBF14F0800F0F4865
:10A5280005D12B230A2103746143113006E02D2342
:10A538000374373B5C43113004F520610322BDE806
:10A54800F041FEF745BA00BFC918002009190020DC
:10A5580004180020C031002004020020F40100206B
:10A568001FB5204B20491A781AB1087840F001002D
:10A57800087009781C4C11F0010F31D01B4909787B
:10A58800532901D00AB103E082B901221A700DE003
:10A5980023290BD1002018701549FEF7F3F9FEF7AF
:10A5A800B5FA237843F00603237019E01B78012BD2
:10A5B80016D120210A460F48F5F7ECFE0E4B6846E7
:10A5C8001B681022996806F0B4FD002409491DF89B
:10A5D800040001EB4401013418F0E0FD102CF5D122
:10A5E8001FBD00BFC9180020091900200418002049
:10A5F80006510308F40100203C180020034B1B7887
:10A60800532B01D1FEF782BA704700BF041800200F
:10A61800084BFF281A68936807D1917B41B1064916
:10A62800927C097801FB023302E0927C02FB003342
:10A63800184670473C180020C91800204328F8B570
:10A6480004460D46174608D1114B0A261A7891FB85
:10A65800F6F66FF3C3021A7000E00E462046FEF7C6
:10A668004DFA90B10A4B303C1A780A2602F00801DC
:10A67800C9B2002918BF002506FB05466FF3C302BF
:10A6880036B21A70BE42A8BF3E4630B2F8BD00BF0F
:10A6980009190020644B2DE9F3411A689846157C86
:10A6A800977C624C2DB1624821780222FEF790F91E
:10A6B80000E02570FF01237807F50C4707F5DE77E2
:10A6C80007EB43075B4E0BB90DB10FE015B901A8B5
:10A6D800394601E001A8B91E022206F02AFD9DF8BC
:10A6E8000430F3759DF80530337605E006F1170060
:10A6F8003F210222F5F74EFE5B23B37502337376D2
:10A708004D4B1B7813F0010F61D04C4B1B78A3F114
:10A718003002D2B2092A35D822780AB9002D40D1A0
:10A72800474A117814469942464A01D000211170CF
:10A73800DFF814E10DF1080C9EF800E0A3F13000F9
:10A74800E644DFF810C1117800EB8000604400EBAC
:10A75800010C0131C9B240189CF86CC090F86C002B
:10A768000EF804CC117008B1032901D90021117029
:10A7780023700DB9384600E0B81E01A9022206F080
:10A78800D2FC17E0232B04D12F4B1A7892B901324F
:10A7980005E02A2B05D12C4B1A785AB1013A1A70C8
:10A7A80008E0532B06D1294A533B1370264A1370ED
:10A7B800FFF724FF264B1B7803F08003DBB2002B46
:10A7C8002FD0214B1B78F6182023F37529E045B3C9
:10A7D8001A4B1878A0F13003DBB2092B10D81B4AAA
:10A7E800137803B92370013303F001031370D8F809
:10A7F80000302178B3F91020FFF720FF207005E022
:10A80800432803D1114B1B7803B92370104B1B78D5
:10A8180003F08003DBB223B1054820210222F5F7BB
:10A82800B9FDBDE8FC8100BF3C1800204B18002092
:10A8380002020020F4010020091900200418002059
:10A848001E1800204A1800201C180020D3180020C9
:10A85800C031002018900208F7B5394E394D3378C9
:10A86800394C6FF34103337017F03EF9FFF7C6FE1A
:10A8780002238DF807302B788BB1344AD17941F017
:10A888000101D171324A207802EBC303D3F8A070DA
:10A8980093F8A5203978FFF7D1FE38700DE03378AA
:10A8A80013F0010F06D02378303BDBB2062B9CBF98
:10A8B800264AD37003238DF80730337813F0010F3D
:10A8C80012D0244B1B7803F08003DBB263B12978E4
:10A8D8001F4B214803EBC10393F8A4309DF80720D0
:10A8E800C0182021F5F756FD2378232B09D11B4AE0
:10A8F8002B781268927C013A934202DA114A0133AA
:10A90800137023782A2B04D12B7813B10D4A013BFD
:10A9180013702378532B0FD114F088FF0B4B0021B1
:10A928002970DA7961F30002DA71FFF767FE0C4BE0
:10A938009A7942F004029A7100232370FEBD00BF89
:10A9480009190020D318002004180020EC38002032
:10A9580018900208C0310020F40100203C180020A3
:10A96800341A00202DE9F74F864E874C3378874DEF
:10A97800232B874F25D12368986843F6F123984203
:10A9880017D1DFF83482296898F8000000F56A507A
:10A99800713006F0B3FB98F80000013000F00100B8
:10A9A80088F8000000F56A50713006F0B1FB2860A5
:10A9B80007E000B2FEF756F828603B7843F008033A
:10A9C8003B703378532B40F06E81236848F6695208
:10A9D8009B68934202D12A686E4B15E04AF20A52EC
:10A9E800934202D12A686C4B0EE04AF287429342A6
:10A9F80002D12A68694B07E048F6BA52934204D15B
:10AA08002A68674B02B101221A7023689A6843F6D4
:10AA1800DD239A420AD1634B29681A7861F3000250
:10AA28001A7006F0E9FE08B106F004FF236843F641
:10AA3800E0229B68934206D15A4B29681A7861F341
:10AA4800C7121A7019E043F6EA22934206D1554B11
:10AA580029685A7861F300025A700EE043F6E7223B
:10AA680093420AD12968504B19B11A6842F0005232
:10AA780002E01A6861F35D721A6023689A684AF204
:10AA8800A0539A420AD12968484B19B11A7842F062
:10AA9800200202E01A7861F345121A7023689A6856
:10AAA8004AF22D639A4202D1287817F085FD23686F
:10AAB80043F6DA229B68934202D12A683C4B05E0B0
:10AAC80043F6E822934203D12A683A4B1A7008E009
:10AAD80048F67252934204D12B6813B92B4B0122CA
:10AAE8001A6023689A684AF22E639A420BD1324A56
:10AAF8002B6812783149032B8B5404D1304B5A7987
:10AB080042F010025A71236848F6B2529B68934289
:10AB180002D129682B4A05E048F6B552934203D181
:10AB28002968294A117016E048F6B652934203D1B3
:10AB38002968264A117015E048F6B852934203D1A5
:10AB48002968234A11704DE048F6B952934202D160
:10AB58002A68204B13E043F60452934202D12A6834
:10AB68001D4B0CE049F2C072934202D12A681B4B7C
:10AB780005E04AF21E52934234D12A68184B1A70E3
:10AB88003BE000BF041800203C180020E01800201B
:10AB9800091900205C210020A83100209F2B0020EB
:10ABA8000218002086190020C0310020984100209A
:10ABB8007A3B00202A320020C9180020A012002069
:10ABC80004210020603600205E36002091350020E8
:10ABD80005350020B41A0020DE10002039170020A7
:10ABE800BA17002048F66A52934206D12A68A14B48
:10ABF80001201A7001460DF05FFA2368986843F641
:10AC0800F12398420DD1DFF87882296898F800007E
:10AC180000F56A50713006F071FA002388F80030A8
:10AC280002E000B2FDF744FF23689A6843F69813E0
:10AC38009A4236D12968DFF844B2DFF84CA20BEB10
:10AC4800C1031B79DFF83882C3F34113012BDFF806
:10AC58003C9221DD98F8000000F56650203006F09F
:10AC68004DFA98F80030DAF8001009EB0302117277
:10AC78000BEBC1021279C2F34112032A0CD17E4AAE
:10AC8800126890681030C01806F038FA98F800304A
:10AC9800DAF800204B441A7498F800302A6809F84A
:10ACA8000320FFF7ABFC3B78DFF8E48113F0010FDA
:10ACB80000F0F080216843F698128B68934240F0C8
:10ACC80081806E4A2B68914602EBC3010979C1F372
:10ACD8004111012906DD6A4A1278072A02D9FDF7CF
:10ACE80015FFE3E03278442A36D15FFA83F82DE085
:10ACF80008F10108614B5FFA88F803EBC8031B7978
:10AD0800C3F34113012B06DD5E4B1B7823BB5C4B61
:10AD18001B78072B20D8DFF868A19AF800301F2B82
:10AD280008D806F069FD70B109EBC8031B7913F068
:10AD3800100F08D19AF800301F2B07D909EBC80368
:10AD48001B79DB0902D0C5F8008005E009EBC803D0
:10AD58001B7913F0080FCBD03378552B40F0A68021
:10AD68002E782CE0013EF6B209EBC6031B79C3F33B
:10AD78004113012B09DD434B1B78002B40F09680D3
:10AD88003F4B1B78082B00F29180DFF8F48098F88D
:10AD980000301F2B08D806F02FFD70B109EBC60351
:10ADA8001B7913F0100F08D198F800301F2B06D923
:10ADB80009EBC6031B79DB0901D02E6076E0002E73
:10ADC800D0D173E04AF22E6293420BD006DCA3F591
:10ADD8002442A2F58F72012A0ED803E04AF28B6250
:10ADE800934209D133782F2B60D9B1F91020303232
:10ADF80093425BDC303B30E043F6F122934207D1CB
:10AE08001F4B1B7823B13078B5F900103B222CE09A
:10AE180006F0F2FC18B3236843F6C4219A688A4204
:10AE280003D047F24D218A4204D13078B5F9001099
:10AE38002D221AE0A2F56A516139052903D943F692
:10AE4800E9218A4201D1012307E043F6E0218A4241
:10AE580002D00A318A4203D100232B6026E02368FE
:10AE68003078B5F90010B3F91020FFF7E7FB286038
:10AE78001CE000BF063400203C1800201404002009
:10AE8800C9180020820D0020E0180020E8230020C7
:10AE9800091900202368B3F90800FDF7E3FD2860CD
:10AEA80098F8003043F0080388F80030FFF7A6FB55
:10AEB800236843F6D222986890420BD12B6813B9C5
:10AEC8009C489D4901E09B489C490222F5F738FDC2
:10AED8000226B0E14AF28B6290420AD12B6813B97C
:10AEE8009748984913E0012B95480CBF9649974914
:10AEF8000DE04AF22E62904218D12B68012B02D144
:10AF08008F48934903E0022B05D18D4891491022BF
:10AF1800F5F716FD8EE1032B02D189488E49F6E735
:10AF2800042B87480CBF8D498D49F0E74AF21E5221
:10AF380090420AD12B6813B981488A49E7E7022B66
:10AF48007F480CBF88498949E1E74AF21F5290427D
:10AF58000AD12B6813B97A488549D8E7012B40F004
:10AF6800698177488349D2E748F6B752904203D0BF
:10AF780043F6EE2290420ED128680A21B0FBF1F286
:10AF880001FB12017C4B3031D97730322E21997771
:10AF98005A7703264FE143F6F12290423ED1774B90
:10AFA8001B78E3B9022229687548FDF711FD43F6BD
:10AFB800F220FDF757FD022201465E48FDF708FD25
:10AFC8003B7813F0010F00F086816E4B1B7803F07D
:10AFD8008003DBB2002B00F07E81694819E0FDF7A1
:10AFE80041FD022201466648FDF7F2FC0222514863
:10AFF8002968FDF7EDFC3B7813F0010F00F06B8139
:10B00800604B1B7803F08003DBB2002B00F06381F8
:10B01800484820210222F5F7BDF95CE143F6981271
:10B02800904240F0F5802B68574EDFF8508156F873
:10B03800331010224248F5F783FC0DF1060298F808
:10B0480000000DF107010FF0F5F84246334620B332
:10B0580016784E49895D03291FD0296803EBC10181
:10B068000979C1F34111012917D1072E15D948498A
:10B078000B224848F5F764FC4748711C0222FDF78B
:10B08800A7FC9DF80710454801310222FDF7A0FCF6
:10B098009DF806104248013118E02E68157803EB38
:10B0A800C601097903EBC6063679C1F341110129B6
:10B0B80006F00706C8BF05F00705012E0ADC394966
:10B0C80034480B22F5F73CFC3348691C0222FDF793
:10B0D8007FFCAFE0022E0BD133490B222D48F5F748
:10B0E8002FFC32462C48691CFDF772FC0E36A2E094
:10B0F800032E0BD12D490B222648F5F721FC2648B3
:10B10800691C0222FDF764FC0D3694E0042E51D12F
:10B1180027490B221F48F5F713FC1F48691C022218
:10B12800FDF756FC1D4805F109010222FDF750FC08
:10B138000C3680E012020020E8900208EA9002082B
:10B1480004020020EA3C03082C3D03080B3D0308D9
:10B15800C13B0308E23B0308033C0308243C030803
:10B16800A03B03088F3D0308D13D0308B03D030809
:10B17800133E0308343E0308F4010020C9180020D8
:10B188000F020020C031002014040020E823002012
:10B1980078570308F9010020FA010020FE01002079
:10B1A8000102002036570308915603081557030873
:10B1B800D3560308052E11D148490B224848F5F704
:10B1C800BFFB4848691C0222FDF702FC464805F10E
:10B1D80009010222FDF7FCFB0B362CE0062E29D1D3
:10B1E80042490B223E48F5F7ABFB3E48691C022258
:10B1F800FDF7EEFB3C4805F109010222FDF7E8FBEB
:10B208003B4805F111010222FDF7E2FB0A3612E084
:10B21800B3F91060092E04DD632ECCBF0326022685
:10B2280000E0012633482968801B46F08002FDF7BC
:10B23800CFFB00E010263B7813F0010F0BD02E4B0C
:10B248001B7803F08003DBB22BB12A482021801B36
:10B258003246F5F79FF8294EB37803F00203DBB2C4
:10B26800002B38D0FDF7BCFA254D034628B92878BD
:10B27800F11D6522FDF7D2FA08E0B2792978B38882
:10B28800F01D01FB023109B205F053FF236847F2B4
:10B298004D229B68934213D006DC43F6C4229342A6
:10B2A8000ED043F69A5209E047F2CD22934207D0D6
:10B2B80048F67252934203D047F28D2293420AD144
:10B2C80005200B210D4AFDF715FB29780D480131A2
:10B2D8000222FDF77DFBBDE8FE8F00BFB2560308D2
:10B2E800F9010020FA010020FE010020F4560308AD
:10B2F8000202002014020020C0310020181900208A
:10B30800C9180020F5010020F0B5114B1F78114B2A
:10B31800303F1E680DE0D6F814C01CF803C0013396
:10B32800644501D112E00023DAB28242F3D3013539
:10B338000D70094B0622094902FB07330D785B198A
:10B3480093F8D440002CEED10C70F9321046F0BDC1
:10B35800041800203C180020189002084A18002001
:10B368002DE9F74F974C984E23689A6843F6055392
:10B378009A4203D133780BB9013333702368934F62
:10B388009968B3F910303A78B3F1010848BF03F16E
:10B3980006084FEAE808337808F1010812F0010FAF
:10B3A80003FB08188A4D00F0AD808A4B1A7899463D
:10B3B800432A4DD128780FFA88FA0AEBD00005F015
:10B3C800A7FE2268844B916846F6440291421860B1
:10B3D80001D12A783AB12A78012102F0070211FA3C
:10B3E80002F250401860287819780AEBD00005F06E
:10B3F80085FE236847F22D329B68934209D1744B2E
:10B408001A78764B03EBD203734A126883F8A021AB
:10B418001EE046F6F542934205D13178002001310D
:10B428000DF0BCF914E046F60B1A4FF0000B236838
:10B438009B68534504D101200BEB00010DF0AEF9D8
:10B448000AF1080A46F62B139A450BF1010BEED1C7
:10B4580099F80030232B10D122682B78927C013A7E
:10B4680093420ADA5A4A013313705D4B9B7803F012
:10B478000203DBB20BB1FDF781F999F800302A2BF2
:10B488000CD12B7853B1524A013B1370544B9B7823
:10B4980003F00203DBB20BB1FDF770F999F8003045
:10B4A800552B14D12368997C0F2910D92A7808398B
:10B4B8008A42474B01DA083200E000221A70484BF2
:10B4C8009B7803F00203DBB20BB1FDF757F999F84B
:10B4D8000030442B42D123689A7C0F2A3ED9297820
:10B4E8003B4B072902D90839197001E0083A1A704C
:10B4F8003B4B9B7803F00203DBB2002B2ED0FDF709
:10B508003DF92BE048F6295399420ED1314B1B786F
:10B51800A3F13101C9B2032907D842F006023A70F3
:10B5280007225343284A573B137023689A6843F607
:10B5380005539A4212D133781B2B08D9284B46F66B
:10B54800E1529A809A7842F002029A7006E0590114
:10B55800C918244B0020C918FDF714FAFFF74EF854
:10B56800214A2B7811789346994288BF1370127834
:10B578000F32934202DD1C4A0F3B137023684FF0D1
:10B58800000A93F81290B9F10F0F9ABFC9F1200978
:10B598005FFA89F94FF010099BF800004FFA8AF317
:10B5A80018180FFA88F202EBE000019305F0B0FDDD
:10B5B8009BF80020019B5FFA80FC9B1803F00703AF
:10B5C8002BE000BF3C180020C918002009190020F2
:10B5D800D318002004180020E0180020E8230020D9
:10B5E8001819002044400308CB1800204CFA03F037
:10B5F8006549013300F0010000280CBFA520DB20BD
:10B60800DBB201F809000AF1010A09F10109082B66
:10B618005FFA8AFA5FFA89F903D0B9F1200FE5D108
:10B6280009E0B9F1200F06D023684FFA8AF19B7C14
:10B6380089189942B0DB3B7813F0010F15D02368C5
:10B6480052499B7C09780F2B01F0800198BFC3F108
:10B658001003C9B294BFDBB2002331B1297810318D
:10B668008A1A4949CB185F219954DFF8288198F83C
:10B678000230474603F00203DBB2002B64D0FDF72B
:10B68800AFF8034600BB226846F6F54192688A4245
:10B6980006D024318A4203D043F6E5118A4204D108
:10B6A80030783B496522002309E043F605518A4278
:10B6B80008D130781C38C0B208F107016522FDF7BF
:10B6C800ADF818E02878F7E7236846F6B5429B6896
:10B6D800934203D043F6F822934202D1BA793178E3
:10B6E80001E0BA792978BB88294801FB0231BA7987
:10B6F80009B205F01EFD23689A7C102A02D905209C
:10B708000B211EE09B6846F6B54293420ED006DC3C
:10B7180043F6E512934209D043F6F82204E046F6D0
:10B72800F542934202D02432934201D1102007E01F
:10B7380043F60552934202D10020102101E0002077
:10B748000721144AFDF7D6F8226846F6595193683E
:10B758008B4216D046F613418B4212D043F6ED21A8
:10B768008B4202D1084BDB219977937C102B08D9A7
:10B77800297809480131022203B0BDE8F04FFDF7EE
:10B7880027B903B0BDE8F08FF4010020C0310020D4
:10B798001F19002018190020F5010020114B002264
:10B7A80070B50D461A7118B11B7803B92023437080
:10B7B800BDB10D48F5F73EF80446681C5CB10A496E
:10B7C8002246F4F73FFD022C0BDC601C28182021D0
:10B7D800C4F1030201E020210322BDE87040F4F720
:10B7E800D9BD70BDB8180020B918002038B5054675
:10B7F800002408E0601905F08BFC3038C0B2092835
:10B8080008D80134E4B2044B1B78303B9C42F1DB8E
:10B81800012038BD002038BD2018002008B505F0EB
:10B8280077FC0023C0B2064AD25C824201D12028AC
:10B8380004D10133082BF6D1002008BD012008BD32
:10B848002891020870B506460D4600240DB12D2337
:10B858002B55A0190021013405F050FC062CF5D118
:10B8680070BD00002DE9F04F974C984F206839784B
:10B878008368068A9AB201FB06260D4647F69011A0
:10B888008B4287B0B6B20BD1914B1A785B7802F035
:10B898000702C3F3420303EBC20306EBC3062BE024
:10B8A80047F650318B4212D1894B8A481A78597819
:10B8B80002F0070288235A43C1F34201773B03FB96
:10B8C800012320210822F618F4F764FD14E047F656
:10B8D80008718B420BD17E4B1A785B7802F0070215
:10B8E800C3F3420303EBC2039B01F61804E0B3F56C
:10B8F800E97F08BF02EB4506774B784D1A789846E2
:10B9080012F0010F53D123689A6847F255139A42EF
:10B9180004D046F655739A4240F04481704B1B7828
:10B928002A2B3BD16F4B93F8009009F1010909F0DC
:10B93800010983F80090B9F1000F1AD046F6557343
:10B948009A4208D1684B46F6E1529A809A7842F0BA
:10B9580002029A7026E1202110226448F4F71AFDA9
:10B968003B7800205901C918614BC918FDF70AF83E
:10B9780018E15D48FCF7ACFF236848469A6846F62C
:10B9880055739A420CBF5B495B49FCF7FBFF39785A
:10B998005A4801310222FDF71BF803E1552B02D06A
:10B9A800442B40F0FF804F4B00221A70FAE02368C6
:10B9B8005869F4F73FFF4A4B834693F800A099462D
:10B9C800BAF1450F02D14E4B00221A705046FDF7CE
:10B9D80095F800284DD04B4B5FFA8BFB1A785245EF
:10B9E8000ED15846FFF790FCFF2804D15846FFF7C0
:10B9F8008BFCFF283DD0444B1A7801321A7015E0B1
:10BA0800DFF804A100228AF8002058460593FFF7C2
:10BA18007BFCFF28059B04D09AF8002001328AF8A5
:10BA2800002099F80020FF281A7022D02168374A90
:10BA38004B6910601B5C886847F255118842136097
:10BA480092460FD1562B01D0542B0BD13B78123B89
:10BA5800DBB2022B06D82B7830B2C01805F058FBA1
:10BA6800CAF800002B7830B2C018DAF8001005F0D8
:10BA780045FB99F80030552B17D12368997C0F297D
:10BA880013D92A7808398A42144B01DA083200E0BF
:10BA980000221A70144B9B7803F00203DBB20BB13F
:10BAA800FCF76CFE184B00221A7099F80030442BF2
:10BAB8003BD123689A7C0F2A37D92978074B072965
:10BAC80026D90839197025E03C180020C91800202B
:10BAD800CE1800200402002009190020D3180020E5
:10BAE800041800201419002018190020F40100205F
:10BAF8006738030878360308BA360308F5010020CA
:10BB08001C1800201E1800204A180020E0180020E9
:10BB1800083A1A70964B9B7803F00203DBB20BB11C
:10BB2800FCF72CFE934B00221A7099F80030432B37
:10BB38000CD1236830B25B6919788F4B19602B7868
:10BB4800C01805F0DBFA8B4B00221A7099F8003008
:10BB5800232B13D122682B78927C013A93420DDA79
:10BB6800864A01331370834B00221A70804B9B78EE
:10BB780003F00203DBB20BB1FCF700FE99F80030CA
:10BB88002A2B0FD12B786BB17C4A013B1370794B70
:10BB980000221A70764B9B7803F00203DBB20BB1DC
:10BBA800FCF7ECFDFEF72AFD754A2B7811789246D2
:10BBB800994288BF137012780F32934202DD704A9F
:10BBC8000F3B137023684FF0000B93F81290B9F1F4
:10BBD8000F0F9ABFC9F120095FFA89F94FF01009D0
:10BBE8009AF8000033B218185844059305F090FAF3
:10BBF800644A02F8090009F101095FFA89F9B9F103
:10BC08001F0F059B05D821680BF1010B897C8B451B
:10BC1800E6DB98F8001011F0010F16D021685A4899
:10BC2800897C00780F2900F0800098BFC1F11001CD
:10BC3800C0B294BFC9B2002138B128789AF8006020
:10BC480010305218801B5F2111542268906849F205
:10BC5800BE7290420AD14D4B1B78532B2FD105F061
:10BC680057FA4B4B187005F04DFB28E0B0F5E97F0B
:10BC780025D1464A1278532A21D11846FFF7CEFD1E
:10BC88000646E0B93B78DA00D31A03F11200FFF751
:10BC9800ADFD60B1FF2300933E4B01961B787920E0
:10BCA8000133029331460422334605F0AFFA3B785C
:10BCB8000021DA00D31A03F11200FFF7C3FD2C4E5E
:10BCC800B37803F00203DBB2002B6ED0FCF788FDDB
:10BCD800034680B9226847F6087192688A420AD0FA
:10BCE80046F655718A4214BF28783878F11D6522C6
:10BCF800FCF794FD0FE02368B2799B682648B3F5FA
:10BD0800E97F0CBF39782978B38801FB0231B27911
:10BD180009B205F00EFA23689A7C032A08D99A68B2
:10BD280047F690118A4203D046F655718A4214D1DB
:10BD38009B6847F6901293420CD198F8003013F0A4
:10BD4800010F01D010202CE0202107221348F4F71E
:10BD580021FB2AE0B3F5E97F02D105200B2121E080
:10BD680046F6557293421BD1002010211AE000BFFD
:10BD7800181900204A180020E0180020D3180020C5
:10BD8800CB180020F4010020C03100200418002046
:10BD980020180020C91800201F19002004020020C4
:10BDA80000200721104AFCF7A5FD23689A7C032A86
:10BDB80016D9B27802F00202D2B28AB19B6847F66D
:10BDC800901293420CD046F65572934208D02978C7
:10BDD80006480131022207B0BDE8F04FFCF7F8BD74
:10BDE80007B0BDE8F08F00BF18190020F50100204A
:10BDF8002DE9F04F7A4E8BB033689D6893F8129016
:10BE0800122D01D00B2D09D1764A122D92F80090EF
:10BE1800A9F130095FFA89F915D01DE04AF23B63B0
:10BE28009D4203D028339D4240F055836E48282117
:10BE3800F4F72EFB8046002800F0508301302821BB
:10BE4800F4F726FB4AE39F7B37B9684BB846D879A5
:10BE5800FEF7DEFB044615E00027B846FF20FEF794
:10BE6800D7FB4AF22C439D4204460BD14AF20B50B1
:10BE780005F04EF9C0B2089020B15C4B9B790BB12C
:10BE8800FCF744FE33685A4D9A68122A1AD19B7BF4
:10BE9800C3B12B7813F0010F08D12046FFF7A6FC99
:10BEA800544B10B101221A7000E018704F4B9B7967
:10BEB80043B12046FFF79AFC20B14E4B1B780BB1DB
:10BEC800FCF724FE2978DFF848A111F0010100F001
:10BED80089819AF80030DFF83CB118460793FCF7DF
:10BEE8000DFE079B002800F0B7804349002008702A
:10BEF8004248434A90F800C013609C45414940F0CD
:10BF08008B8033689B8903F00F03032B21D1ACF19D
:10BF1800300C0A2000FB0CF03B4BDFF8F0C093F824
:10BF280000E00590704409900EF1010E1CF8000025
:10BF3800DDF814C05FFA8EFE106083F800E00CEBA9
:10BF48000E00DFF8C8E01EF80000002871D1187054
:10BF58006FE0082B2BD12C48ACF1300C03780CEB9C
:10BF68008C0E0993294B9E44099B734493F86CE00B
:10BF78000993264BBEF1000F01D180F800E090F83C
:10BF880000E00CEB8C0C634403EB0E0C0EF1010E7D
:10BF98005FFA8EFE73449CF86CC093F86C30C2F85C
:10BFA80000C080F800E0002B43D1174811E0072BB0
:10BFB80011D1BCF1300F10D11348037823B14FF0E1
:10BFC8002B0EC2F800E001E0C2F800C0013303F014
:10BFD800010303702DE0062B2BD10B78013327E0EA
:10BFE8003C1800202018002004020020D618002049
:10BFF80009190020670E00207F3B00201E18002032
:10C00800E0180020D31800204A18002018900208D1
:10C018000418002021180020DFF898E203709BF82C
:10C0280000304FF0010C8EF800C013B10B78634458
:10C038000B7040238BF800300B784B4503D39B4B98
:10C0480009F1FF30187008781168201805F056F8C3
:10C058002B7843F004032B709AF80030232B2FD150
:10C06800924B09F1FF311A788A4229DA72B932689B
:10C078004AF23B6192688A4208D028318A4205D048
:10C088002046079305F044F8079BC8B1187801309B
:10C09800C0B21870201805F03BF828B9834B20214E
:10C0A8001878201805F02AF8814B40221A702B784E
:10C0B800804A43F004032B7000238BF80030137080
:10C0C8009AF800302A2B10D1784B1A786AB1013AC5
:10C0D8001A70774B40221A702B78764A43F0040383
:10C0E8002B7000238BF8003013709AF80030432B24
:10C0F8001FD16E4B1878484505D220182021079388
:10C1080004F0FCFF079B9BF800203AB91B7809F163
:10C11800FF32934202DA654A013313702B78644A7E
:10C1280043F004032B7000231370624A8BF800302D
:10C1380013709BF8003013B15F4A013B13709BF8F2
:10C148000030012B0ED1594B1A784A4501D20132E1
:10C158001A70584A002313702A7842F004022A7091
:10C168008BF800302B7803F00402D2B2002A71D089
:10C17800524A6FF382031370002111225048F4F7DA
:10C1880009F9504A494B11781B78994288BF1370B6
:10C1980011780F318B4202DD4A490F3B0B70117841
:10C1A80047481022611804F0C4FF4548F4F742FBE1
:10C1B80033684AF23B619B68C2B28B4202D0283195
:10C1C8008B4205D122B94048F4F734FB421CD2B265
:10C1D8000F2A3FD83A4820218018C2F11002F4F7FC
:10C1E800D9F837E0DFF8D8B011225846F4F7D2F87A
:10C1F80033684AF23B629B68934202D028329342EA
:10C2080009D1214604222E4804F093FF40463946BE
:10C21800FFF7C4FA1EE021461022584604F089FFB1
:10C228005846F4F707FB02462021C2F11002584491
:10C23800F4F7B0F821464A46244804F07AFF244A25
:10C248001020937882F8069043F002039370014619
:10C25800FCF750FB9AF80030532B75D133689A6875
:10C268004AF22C439A4208D1204604F051FF20B1EB
:10C278004AF20B50012104F041FF3368DFF838A07F
:10C288009B68122B40D12046FFF7B0FA834600285E
:10C2980030D0104BFF2219780F4BF9B90092019159
:10C2A8001B78782001330293FB3A1FE0D318002053
:10C2B8007F3B00204A18002021180020091900207F
:10C2C800B8180020CB180020B918002053180020F7
:10C2D8004C180020670E0020C91800200021009289
:10C2E80001911B787A200133029304220B4604F053
:10C2F8008DFF09E08AF800007D492046FFF7A2FA81
:10C308007C4B83F800B0EFE020464946FCF748FB39
:10C31800794B0020187033688AF800009B6849F24E
:10C32800D272934202D10090013005E04AF24E42A7
:10C33800934206D1012300930146024603460CF0BE
:10C3480059FA6E48FCF7C4FAFEF758F92B7813F03F
:10C35800010F17D033684AF23B629B68934202D0C0
:10C368002832934204D140463946FFF717FA09E0CC
:10C378005F4B634A03F1100153F8040B8B4242F8F8
:10C38800040BF9D133689A68122A1ED19B7BE3B15A
:10C398002046FFF72BFAC0B12B7813F0010F14D108
:10C3A800584B9A7922B9DA79574B1B789A420CD0B4
:10C3B800564B1A780023303A05E055492A20C91807
:10C3C80001330874DBB29342F7DB326893680B2BB6
:10C3D80001D0122B0AD14A4B991D13F8010B2028C2
:10C3E80002D10D3003F8010C8B42F6D192684AF263
:10C3F8002C439A4214D1434B9B798BB1089878B15E
:10C408004FF0000909EB040004F082FE18B1404B1C
:10C418002A224B441A7409F10109B9F1100FF1D11C
:10C428002B7813F0010F25D03A4B1B7803F08003CB
:10C43800DBB2FBB133689A684AF23B639A422D4BF0
:10C4480003D04AF263618A420CD11B7833B9B8F140
:10C45800000F0FD05F3388F801300BE057B15F222F
:10C46800FA5407E0244A1B78127810339B1A284A9A
:10C478005F21D154284CA37803F00203DBB2002BD0
:10C4880032D0FCF7ADF92049034628B9087865226F
:10C49800E11DFCF7C3F912E03068B4F90430A27961
:10C4A80084680978122C01FB023105D1807B18B908
:10C4B8001449C97902FB0131184804F03AFE33687F
:10C4C8009B68122B10D10820134A01460BB0BDE817
:10C4D800F04FFCF70FBA0027B84600E0074609F10D
:10C4E800FF395FFA89F9B9E40BB0BDE8F08F00BFF6
:10C4F800B8180020D3180020CB1800204C180020B2
:10C5080004020020D6180020C91800202018002096
:10C51800F4010020C0310020181900201F19002044
:10C5280024282DE9F041144626D16B4B43F63832C6
:10C538001B686A4D9B686A4E934206D12B7813F0AC
:10C54800010F0ED02438674909E04AF2636293422A
:10C558000AD12B7813F0010F03D063490020FCF7B0
:10C5680011FA2978490800E02978301901310222A6
:10C57800FCF72EFA0234AAE0E72809D1574B5848AD
:10C588001978801801310322FCF722FA03349EE05F
:10C59800A3282AD1514D2B783F2B15D81046534943
:10C5A800FCF7F0F95148F4F745F92A2124184C48CA
:10C5B800E4B2F3F76DFF002800F08A8029780222A0
:10C5C8000131FCF705FA83E05901494DC91869188A
:10C5D80001F582411046DF31FCF7D4F905F59240A8
:10C5E800FE30F4F727F9241871E0F22821D13B4FE7
:10C5F8003B4D3978072605EB0208B1FBF6F14046BA
:10C6080001310222FCF7E4F939782D23B1FBF6F663
:10C6180088F80230F3009E1B8B1B364FDBB207EB0A
:10C6280083031988E21CA9529B78A81883700634E2
:10C638004DE025280BD1304B46F6E1529A80452231
:10C648009A719A78053842F002029A703CE05E28A6
:10C658000BD1294B46F6E1629A8045229A719A7865
:10C668003E3842F002029A702EE07C280BD1224B11
:10C6780046F244129A8011229A719A785C3842F0F4
:10C6880002029A7020E0EC280BD11B4B46F625726B
:10C698009A8045229A719A78CC3842F002029A70B0
:10C6A80012E0A7280BD1144B46F645729A80452212
:10C6B8009A719A78873842F002029A7004E0E0286A
:10C6C80001D1541C03E018B1054B18550134E4B2EC
:10C6D8002046BDE8F08100BF3C180020C9180020A2
:10C6E800F4010020CC3003088A30030846380308D8
:10C6F80048EE0208C11A03081819002038B50A4B79
:10C7080046F68A451B78002405FB030507E0074B1E
:10C7180022461978FFF704FF041B2D1904462878D0
:10C7280008B11F2CF3D938BD1F180020C9180020E4
:10C7380070B5002543F61C64204604F0E9FC064663
:10C7480004F1080004F0E4FC16F0FF0F06D020F016
:10C758007F0010F0FF0F01D00135ADB246F23B1358
:10C768009C4201D00934E7E7284670BD70B5B0F99E
:10C7780000500E4605EBC50505F5785524352846C5
:10C7880004F0C6FCC3B213F0800F064C08D03EB9C3
:10C7980022882846013A03F07F01228004F0AEFC8B
:10C7A800208870BD1A180020454B2DE9F74F1B88CB
:10C7B800444A044689461788DFF80C8123B14FF0B4
:10C7C800000A0AE09A4608E00529FBD198F80030EB
:10C7D80043F0040388F8003070E098F8003013F054
:10C7E800030F0BD013F0010F02D0B4F1FF3F05D1B6
:10C7F80003F00203DBB21BB1012C01D03F19BFB219
:10C808003BB2B3F1FF3F04D0B3F57A7F08BF0027EE
:10C8180001E040F2E7370FFA87FB0BEBCB0303F598
:10C82800785303F11C00019304F072FC10F0FF0F21
:10C83800019B16D0B9F1050F09D103F1240004F0CA
:10C8480067FC20F07F0010F0FF0FC6D022E0B9F19E
:10C85800000F1FD003F1240004F05AFC00F07F06FB
:10C8680018E00AF1010AB4F1FF3F1FFA8AFA04D16D
:10C8780098F8003043F0010305E0012C05D198F841
:10C88800003043F0020388F80030BAF57A7F0DD003
:10C898003D46A2E74E4505D0B9F1000F02D0B9F1E7
:10C8A800050F9AD1BAF1000F05D000E03D46054AC0
:10C8B8002DB2156002E0034BC3F800B0BDE8FE8F4F
:10C8C8001A180020E0180020E41800202DE9F04193
:10C8D800037890465A1ED2B2792A9AB00F4600F2CF
:10C8E800CA805E01654AF3189B18654A46F68A466F
:10C8F8001278457806FB0236E7213046F3F7C8FD83
:10C908000446F0B930467C21F3F7C2FD0446C0B9AD
:10C9180030462521F3F7BCFD044690B93046242162
:10C92800F3F7B6FD044660B930464021F3F7B0FD91
:10C93800044630B93046F921F3F7AAFD0446002829
:10C9480078D0A41B0FB14F4800E04046314622463C
:10C95800A619F3F7F5FF3046E721F3F799FD30B153
:10C9680028466946652246F62573FBF757FF304689
:10C978007C21F3F78DFD50B1691EC9B201EB01119D
:10C9880001F5C24168464431112204F0D2FB304619
:10C998002521F3F77DFD38B1681EC0B269466522CE
:10C9A80046F6E153FBF73AFF3046F921F3F770FDFD
:10C9B80038B1681EC0B26946652246F6E163FBF7E6
:10C9C8002DFF30464021F3F763FD50B1691EC9B20F
:10C9D80001EB011101F5E64168465F31112204F0CF
:10C9E800A8FB30462421F3F753FD58B117B1254869
:10C9F800201801E008EB040029460222FBF7E8FFB3
:10CA080002340CE017B11F48201801E008EB0400BD
:10CA18006946F3F7B1FE6846F3F70CFF0419002FD7
:10CA280029D0194A9378141943F00203937000230C
:10CA3800E37116E03046F3F7FDFE05461FB94046A0
:10CA480031462A4615E0102810DD2A460D483146A1
:10CA5800F3F776FF0C4A9378551943F00203937065
:10CA6800EC7110200146FBF745FF04E0074831460A
:10CA78001022F3F765FF1AB0BDE8F0812B200308F8
:10CA88001F1800201F190020181900200402002078
:10CA98000C4B1A7812F0010302D000200A4905E075
:10CAA80002F00200C0B218B108491846FBF76ABF85
:10CAB80002F00402D2B20AB10549F7E7054801219C
:10CAC800FFF704BFE418002004F60208E3F50208A3
:10CAD80025F602080B19002070B5124D124C0020E3
:10CAE8001249FBF75FFE2846A1780222FBF770FF88
:10CAF800E81CE1780222FBF76BFF05F108002179B9
:10CB08000222FBF765FF05F10B0061790222FBF7B2
:10CB18005FFFA17905F10E000222BDE87040FBF726
:10CB280057BF00BFF40100200B1900203191020803
:10CB38002DE9F341544F554C3B689D7C237813F005
:10CB4800010F33D1022243F61A610DF1060004F0F9
:10CB5800F0FA4F4EBDF806304FF0FF3033602946EB
:10CB6800FFF722FE237843F001032370494B1B781B
:10CB780013F0030F18D1B6F90010474801EBC101B3
:10CB880001F578511C31092204F0D3FA434B1B8874
:10CB98003BB1434B30461978C1F34001FFF7E6FD3E
:10CBA80010B90020F9F7E6FAFFF796FF3D4E337803
:10CBB800552B0DD1DFF8DC803B48FBF789FE98F850
:10CBC80000304FF0FF306FF3410388F800300DE07C
:10CBD800442B2FD1DFF8BC803348FBF779FE98F857
:10CBE800003001206FF3000388F800302946FFF772
:10CBF800DBFD98F8003013F0030F19D1244D2648B7
:10CC0800B5F90010092201EBC10101F578511C3179
:10CC180004F08FFA214B1B883BB1214B2846197829
:10CC2800C1F34001FFF7A2FD10B90020F9F7A2FAFD
:10CC3800FFF752FFFFF72CFF3378232B22D1154B38
:10CC4800194E1A7802F0FC026FF382021A70FBF791
:10CC58005DFFB3786FF34103B370144B1D7835B99A
:10CC6800FBF78CFD3046FBF733FE3D600AE0227887
:10CC7800013DEDB242F0060222701D700C4B53F8D4
:10CC880025303B60BDE8FC813C18002009190020D4
:10CC9800E0180020E41800200B1900201A180020C2
:10CCA800C34600200418002018190020F718002097
:10CCB800F81800202DE9F0411646104A0F4653781F
:10CCC8000E21C3F342034B43117803F5F24320339B
:10CCD8000B4D01F00701044603EB4101022204F069
:10CCE80028FAE81921780222FBF772FE6178A81960
:10CCF8000222BDE8F041FBF76BBE00BFCE18002052
:10CD0800F4010020044B02225978044BC1F342017C
:10CD180018180131FBF75CBECE180020F401002082
:10CD280010B5074B074C1B78074A03F0070304EBC1
:10CD380083031C88111814529B788B7010BD00BF98
:10CD4800CE180020C11A0308F4010020084B1B78F4
:10CD58009B0902D0012B06D102E01020054904E00E
:10CD68001020054901E005491020FBF70BBE00BF64
:10CD7800CE180020A6020308C7020308E802030829
:10CD88002DE9F041DFF868800F4698F80010174D3C
:10CD9800C1F382010446164605F10800013102225A
:10CDA800FBF716FE98F80010042201F01C0101F5AB
:10CDB8000C41204601F5847104F0BBF9E81921788B
:10CDC8000222FBF705FEF81C281861780222FBF7FF
:10CDD800FFFDA819A1780222FBF7FAFDF01CE17803
:10CDE80028180222BDE8F041FBF7F2BDF40100204B
:10CDF8001D180020064B1B7803F08003DBB233B10B
:10CE0800435C04482021C0180222F3F7C3BA7047D4
:10CE1800C0310020F40100202DE9F743654D664C30
:10CE28002B6821789B68022203EB41010DF1060073
:10CE380004F07FF92B68A9469A6843F6F4239A42CE
:10CE480008D100205D49FBF79DFDBDF806804FF431
:10CE5800B46303E0BDF806804FF46163B8FBF3F1F7
:10CE680003FB11883C221FFA88F8B8FBF2F302FB97
:10CE78001388CFB2DEB2022251483946FBF7A8FD2B
:10CE88005FFA88F802224F483146FBF7A1FD0222DB
:10CE98004D484146FBF79CFD4C4B1B7813F0010FA6
:10CEA8006ED04B4B4B4D1878232804D12B78012B8F
:10CEB80062D8013305E02A2805D12B78002B5BD0F6
:10CEC800013B2B7058E0A0F13003DBB2092B01D9EC
:10CED80043284BD12B7873B9D9F8003039B29A6806
:10CEE80043F6F4239A4201D10A2200E01122FDF709
:10CEF800A5FBC7B216E0012B0ED1D9F8003031B22C
:10CF08009A6843F6F4239A4201D1172200E03B22A3
:10CF1800FDF794FBC6B205E041463B22FDF78EFBC8
:10CF28005FFA80F8D9F800309A6843F6F4239A42F9
:10CF380009D13C235E434FF4B46303FB0767B8444D
:10CF4800ADF8068006E03846314642460EF00DFE42
:10CF5800ADF80600D9F8003020789B680DF106017D
:10CF680003EB4000022204F0DEF805E0532803D169
:10CF780000232B70FDF742FB17482978FFF73AFF8B
:10CF8800D9F800309A6843F6F4239A4210D02078F2
:10CF9800124965220023FBF741FC05200B21104AAA
:10CFA800FBF7A8FC21780F4801310222FBF710FD9E
:10CFB800BDE8FE833C180020C9180020CB340308C4
:10CFC800040200200A020020120200200919002091
:10CFD80004180020D3180020429102081F190020CD
:10CFE80018190020F501002073B59A4B9A4D1A784C
:10CFF80012F0010F05D12A7812F0380204BF2A7006
:10D008006A701A78934E42F001021A702B78924C8B
:10D0180013F038023ED191490978552904D113F00B
:10D02800070F2FD0DA1D0AE044290CD103F00702BC
:10D0380001323D3992FBF1F1C800411A521A62F3EC
:10D04800020323701EE053290AD1C3F3C201013140
:10D0580061F3C5032370637862F34303637011E0DF
:10D0680023290FD1FBF752FD33787D4A43F006039D
:10D0780033701378013BDBB213707A4A52F82320DD
:10D08800794B1A6000207949FBF77CFC1C20FFF7DC
:10D0980047FEDDE0082A2ED175490020FBF772FC17
:10D0A8000620FFF72FFE0C20FFF73AFE1521182265
:10D0B80001A8FFF7FFFD694B1B78552B06D1637854
:10D0C80003F0FE03C3F34202013A07E0442B0BD1FD
:10D0D800637803F0FE03C3F34202013202F0030255
:10D0E80062F343036370B3E0532B28D0232B40F043
:10D0F800AF802378A6E0102A51D15D490020FBF7C4
:10D1080041FC0620FFF7FEFD0C20FFF709FE152164
:10D11800182201A8FFF7CEFD6178564801F00101F9
:10D12800FFF768FE4D4B1878232801D02A2804D130
:10D138006378DA4362F30003D4E7532804D12378F1
:10D14800C3F3C202013280E0A0F13003DBB2092B45
:10D1580001D943287CD16B7802AA03F001033B2153
:10D16800D41883F001024B43172606FB023214F849
:10D17800041CFDF763FA04F8040C6B780E22C3F361
:10D1880042035343287803F5F243203300F00700A5
:10D1980003EB400001A90C3A03F0C5FF58E0182A38
:10D1A8004DD133490020FBF7EDFB0620FFF7AAFD20
:10D1B8000C20FFF7B5FDFFF7C9FD284B1B78552B51
:10D1C80007D1237813F0C00F42D0C3F38112013A7C
:10D1D80006E0442B07D123789A09012A38DC01326A
:10D1E80062F3871333E0232B04D12378C3F3C202FD
:10D1F800023A2AE0532B2BD1FBF788FC33781E4ADE
:10D2080043F006033370164B1648197840F821206E
:10D21800013119702378C3F3C201013161F3C503E9
:10D22800C3F381112370104B11B1012904D101E01E
:10D238001C3202E0114A00E0114A1A6008E0114A63
:10D2480000211170C3F3C202013A62F3C5032370CF
:10D258007CBD00BF09190020CE180020041800204A
:10D26800F7180020F81800203C1800206402030872
:10D278008502030845910208489102088091020836
:10D288009C910208D318002073B5494B494D1A7870
:10D2980012F0010F04D12A7812F0030208BF2A7095
:10D2A8001A78434E42F001021A702B78414C13F061
:10D2B80003022ED1404A1278552A03D1C3F38202C1
:10D2C800013A04E0442A06D1C3F38202013262F330
:10D2D8008403237017E0532A03D15A1C62F3010315
:10D2E800F7E7232A0FD1FBF711FC3378334A43F0D1
:10D2F800060333701378013BDBB21370304A52F8DF
:10D308002320304B1A6001A810211B22FFF738FD9B
:10D318004DE0012A4BD101A810211A32FFF730FD48
:10D32800254B1878232804D12378C3F341120132FE
:10D3380005E02A2807D12378C3F34112013A62F3A2
:10D34800461323702DE0532804D12378DA1C62F3A6
:10D358000103F6E7A0F13003DBB2092B01D943281A
:10D368001FD12B7802AAC3F34113D4180C215A1CDD
:10D3780003F001034B4302F001021F2614F8041CBA
:10D3880006FB0232FDF75AF904F8040C287801A9C3
:10D3980000F01C0000F50C4000F58470042203F036
:10D3A800C2FE29780848C1F34111FFF723FD7CBD6F
:10D3B800091900201D18002004180020F718002063
:10D3C800F81800203C180020B8910208064B1B787A
:10D3D80003F08003DBB233B1435C04482021C0185A
:10D3E8000322F2F7D7BF7047C0310020F4010020B4
:10D3F8004328F8B504460D46174606D1104B0026BB
:10D408001A786FF3C3021A7000E00E462046FBF745
:10D4180075FB90B10A4B303C1A780A2602F00801D5
:10D42800C9B2002918BF002506FB05466FF3C302E1
:10D4380036B21A70BE42A8BF3E4630B2F8BD00BF31
:10D44800091900202DE9F3416E4F6F4E3B7843F0E8
:10D4580001033B70347844B94AF2834003F058FE24
:10D468006A4B6B491860204617E0012C02D1002056
:10D47800684912E0022C02D1002067490DE0032C14
:10D4880002D10020654908E0042C02D1002064493B
:10D4980003E0052C03D163490020FBF773FA3178C8
:10D4A800D9B9614B1B78312B01D1013101E0302B07
:10D4B80005D1564B4AF28340196003F01FFE5B4BBF
:10D4C8001A785B4B02F08002D2B20AB1202202E045
:10D4D8004E4A12683032DA776EE001290BD0022901
:10D4E8000CD003290DD004290ED04AF27F45052916
:10D4F80018BF00250AE04AF26F4507E04AF2734573
:10D5080004E04AF2774501E04AF27B4529460422C5
:10D5180001A803F00EFE474B474A03F1100153F8E8
:10D52800040B8B4242F8040BF9D1032243489DF8BF
:10D538000410FBF74DFA032241489DF80510FBF74C
:10D5480047FA03223F489DF80610FBF741FA3E4888
:10D5580003229DF80710FBF73BFA334B3B4C187836
:10D56800232804D12378022B22D8013304E02A2867
:10D5780004D12378E3B1013B237019E0A0F1300313
:10D58800DBB2092B01D9432812D194F8008002AAF2
:10D59800904418F8041CFF22FFF72AFF08F8040C2F
:10D5A800207802AA131813F8041C281803F0A6FD03
:10D5B80027482178FFF70AFF1B4B1B78532B1FD1F5
:10D5C800224B00221A7033780133DBB2062B3370FA
:10D5D80004D0012B14D10D4B1B688BB1FDF70EF84D
:10D5E800002333703B781B4A43F006033B701378E3
:10D5F800013BDBB21370184A52F82320174B1A600C
:10D60800BDE8FC8109190020C9180020E018002095
:10D61800514E03087A4F03089B4F0308BC4F030879
:10D62800DD4F0308FE4F030804180020C031002016
:10D63800F4010020987D0308040200200502002060
:10D64800090200200D02002011020020D31800203A
:10D65800BC910208F7180020F81800203C18002098
:10D6680070B5174C0D460646002120464FF4C1728E
:10D67800F2F790FEFF2D0AD1B10001F5DA412046FC
:10D68800E131042203F055FD23789BB970BDFE2DCE
:10D6980001D1173E02E0FD2D02D10136267009E0C6
:10D6A800B60006F5DA40E130401903F031FDC0B2AA
:10D6B800207020B10248BDE8704016F003BB70BD71
:10D6C8002C1B00202DE9F04116F02EFB60B1102034
:10D6D8008F49FBF757F98F4B1B78432B40F0EF81AD
:10D6E800BDE8F04116F042BB16F030FB002826D00A
:10D6F800894C23786BB110208849FBF743F9884897
:10D708002D211030F2F7C4FE002800F0D8812178CE
:10D7180010E010208349FBF735F981482D2110309E
:10D72800F2F7B6FE0446002800F0C98116F026FB81
:10D73800014620468222BDE8F041FBF749B97A4C00
:10D7480043F6CC2223689B68934250D0774E744DA1
:10D75800307803EB800003F0DBFC032201467448B9
:10D76800FBF736F92368986846F6457398422BD03C
:10D77800203B984228D03378013000EB830003F037
:10D78800C7FC0322014605F11500FBF721F92368C0
:10D7980030789B68023303EB800003F0B9FC032266
:10D7A800014605F11900FBF713F9236830789B68E7
:10D7B800033303EB800003F0ABFC0322014605F1C1
:10D7C8001D00FBF705F90EE02D2103225948F2F759
:10D7D800E1FD2D2103225848F2F7DCFD57482D21A1
:10D7E8000322F2F7D7FD20232B772B762B75544B8A
:10D7F8001B7813F0010F00F0BD80236843F6CC229C
:10D808009B68444D934261D04E4E484F32783878E9
:10D81800D31803EB800003F07BFC4B4B01461860E8
:10D8280028789846A0F13002D2B2092A01D94328B3
:10D838000FD109B2BA22FCF701FF236832789B683E
:10D848000146C8F800003878D31803EB800003F0CD
:10D8580055FC2B782A2B04D1337813B1394A013B74
:10D8680013702B78232B0ED13378022B0BD8226818
:10D8780046F6257192688A4205D020318A4202D044
:10D88800304A013313702B78552B01D0442B0FD11C
:10D89800236831789B68A3F5DA43B3F1E10248BF06
:10D8A800A3F1DE023B7803EBA202D0B2FFF7D8FE69
:10D8B800264B1B7803F08003DBB23BB13278184B60
:10D8C80003EB820320225A749A74DA742B78532B50
:10D8D80006D023689A6843F6CC239A4240F0EF803A
:10D8E800FBF714F9236846F6E1529B68934203D18B
:10D8F8000E4B0220197806E046F64572934227D16E
:10D908000A4B002019780131BDE8F0410AF046BF02
:10D918008037030804180020D81000205736030861
:10D92800F4010020A13703083C180020C918002082
:10D9380005020020090200200D020020110200202B
:10D9480009190020D3180020E0180020C031002059
:10D9580046F62572934204D15A4B012019780918CA
:10D96800D2E746F6E162934240F0A980554B032086
:10D978001978C8E7236849F2D2729B6893423FD16D
:10D98800504E10205049FAF7FDFF31784F4D01EB0A
:10D99800011101F5164101F5E9711022284603F03D
:10D9A800C8FB2B4605F110012A461078474F78B975
:10D9B8004749FAF7E7FF3846E721F2F769FD78B1FA
:10D9C8003178401B381801310322FBF701F807E0D2
:10D9D80013F8010B10B9203003F8010C8B42E4D185
:10D9E8003C4D2B782A2B03D13078FD21FFF738FEE8
:10D9F8002B78432B63D1307823680130C0B259E0CB
:10DA080043F6CC229342334E1AD010203249FAF70B
:10DA1800B9FF33782A2B52D1304B1B689B68A3F58A
:10DA2800DA43B3F1E10248BFA3F1DE02254BFF213F
:10DA38001B7803EBA202D0B2BDE8F041FFF710BE9D
:10DA48003378204D552B04D12B78142B01D1033B6F
:10DA58002B703378442B05D12B78122B02D1194B1C
:10DA680015221A702B78DFF878805901C9184144BB
:10DA780001F5944100201F31FAF784FF08F592411F
:10DA8800102017312F78FAF77DFF3378112F8CBFCC
:10DA9800032700272A2B05D12878FE21C01BC0B2F6
:10DAA800FFF7DEFD3378432B09D12B78173BDF1BBB
:10DAB8002368F8B2997CBDE8F04116F01DB9BDE8BD
:10DAC800F08100BFC91800205F370308F401002067
:10DAD8006F180308041800201D3703083C1800209D
:10DAE80048EE020810B50E4B1B78452B17D10D4B8D
:10DAF8001A7842F006021A700B4A1378032B0ED8D4
:10DB08000A490B4C086844F82300013313708368F2
:10DB18000B60FAF73FFEBDE81040FAF7F7BF10BDFB
:10DB28000418002009190020F71800203C180020CC
:10DB3800F818002010B50C4B04462146D8790DF092
:10DB4800D8FF60B1204655210DF032FE48B120467D
:10DB58000DF0C4FED0F1010038BF002010BD022036
:10DB680010BD022010BD00BFD618002008B50DF06A
:10DB7800AFFFC0B208BD00002DE9F047634B644C0D
:10DB88001A78994612F0010F624D65D02078FFF798
:10DB9800D1FF614A2B181178604F93F8A831604E75
:10DBA80044293870336090460AD12D2B08D038B9F3
:10DBB80095F8A91101233B7031602078FFF7D6FF53
:10DBC80098F80030552B10D133682D2B0DD03B78A9
:10DBD8005BB1013B514ADBB21370EB1893F8A81103
:10DBE8004F4B20781960FFF7C1FF98F80030232BBE
:10DBF80019D14C4B20781B689B7C013B984212DA68
:10DC0800434B0130C0B21870FFF794FF38702818E2
:10DC180090F8A8313360444B9B7803F00203DBB2E1
:10DC28000BB1FAF7ABFD98F800302A2B14D1207805
:10DC380090B1374B0138C0B21870FFF77BFF3870CE
:10DC4800281890F8A8313360374B9B7803F002030B
:10DC5800DBB20BB1FAF792FD344EFCF7CFFC237818
:10DC680032789A4288BF337032780F32934202DD9D
:10DC78002E4A0F3B1370DFF8C4800027307838181D
:10DC8800C0B2FFF757FF281890F8A8310137102FB6
:10DC980008F8013F07D0254B1A78224BBA181B68A1
:10DCA8009B7C9A42EADB99F8003013F0010F13D0FD
:10DCB8001F4B1A781F4B02F08002D2B22AB1227889
:10DCC80031781032521A5F2105E02278317810320B
:10DCD800521A134909689954134DAB7803F002039B
:10DCE800DBB25BB12078E91D652246F6E163FAF7FD
:10DCF80095FD05200B212A46FAF7FCFD21780E48F0
:10DD080001310222BDE8F047FAF762BE0919002086
:10DD1800D318002018900208041800201C180020AE
:10DD2800E01800203C18002018190020CB1800200B
:10DD3800C0310020F4010020F5010020030200207A
:10DD48002DE9F041002480460D461646234601275A
:10DD580017FA04F298F80010E0B2914206D146F69C
:10DD6800257329463246FAF759FD3B460134042CFF
:10DD7800EDD1043C0A4AE0B2A218917898F8002044
:10DD88008A4207D132B146F6457329463246FAF738
:10DD980045FD01230134042CECD11846BDE8F0817F
:10DDA800D61800202DE9F041074610460D461446C6
:10DDB800F2F740FDC3B28046B3B1AB4214D80B4E64
:10DDC80020212A46F019F2F7E5FA2046F2F732FD4B
:10DDD800C8EB05056D08EDB2EF1902462146F019AA
:10DDE800BDE8F041F2F72EBABDE8F081F401002059
:10DDF800312200230178194111F0010F02D00449A2
:10DE0800C9188A7501330132042BD2B2F2D1704796
:10DE1800F40100202DE9F04F87B09DF8405080466E
:10DE2800072D0E4605929A4637D1002427463378A7
:10DE3800234113F0010F2CD0012523B24FF0000825
:10DE48000293512029462A462B460095CDF8048096
:10DE580003F0DCF91B20414662194346CDF80080E7
:10DE6800F4F74AFC37B9112039463A462B46009751
:10DE7800F4F742FC534B204613F8242001276FF394
:10DE8800000203F824201199F5F7E4FA2046F5F783
:10DE9800E5FC0134042CCAD1F7E1012D03780CD13B
:10DEA8000BB90B7823B3FF2300930021464B019154
:10DEB8001B780C200133029316E0022D09D10BB90F
:10DEC8000B78ABB10021FF2300930191029134201C
:10DED8000AE0062D0CD10BB90B784BB10021FF23BA
:10DEE800009301910291652004220B4603F08EF9FC
:10DEF800BAF1010F98F800302BD13BB1334B002019
:10DF0800D979024653460090F4F7F6FB33783BB1D3
:10DF18002E4B0120D979002203460092F4F7ECFB3E
:10DF28000020F5F74DFA98F80030002B5BD0284B0D
:10DF38001978002957D1274B5B78002B53D0FF2342
:10DF480000933A2001220B460191029103F05EF9F9
:10DF580049E063B1052D4FF0000102D100910F2077
:10DF680001E000910B200A460123F4F7C5FB337842
:10DF780083B1052D4FF0000106D110200A46012378
:10DF88000091F4F7B9FB12E00C200A460123009136
:10DF9800F4F7B2FB022D25D0032D01D10E4B02E080
:10DFA800042D02D10D4B1F781DE0052D01D10C4B1E
:10DFB800F9E7012D01D1044BF5E7062D0CBFFF272A
:10DFC800002710E013150020E0150020D6180020C7
:10DFD800FE140020670E0020E01A0020573A0020A7
:10DFE80013340020FF2798F80030002B00F09D80A4
:10DFF800914C237803F02003DBB26BB18F4B197877
:10E0080011F0010108D1FF230093282001220B46BB
:10E018000191029103F0FAF8237803F01003DBB2C0
:10E0280073B1864B197801F00201C9B241B9FF23D7
:10E038000093292001220B460191029103F0E6F892
:10E04800E37813F0010F0ED07C4B197801F004012E
:10E05800C9B241B9FF2300932A2001220B4601913E
:10E06800029103F0D3F8E37803F00203DBB273B153
:10E07800724B197801F00801C9B241B9FF23009326
:10E088002B2001220B460191029103F0BFF8E3789F
:10E0980003F00403DBB273B1684B197801F0100187
:10E0A800C9B241B9FF2300932C2001220B460191EC
:10E0B800029103F0ABF8E37803F00803DBB273B125
:10E0C8005E4B197801F02001C9B241B9FF230093D2
:10E0D8002D2001220B460191029103F097F810F0D0
:10E0E80015F970B1554B197801F04001C9B241B921
:10E0F800FF230093492001220B460191029103F06E
:10E1080085F8E37803F04003DBB273B14B4B197821
:10E1180001F08001C9B241B9FF2300934E200122CA
:10E128000B460191029103F071F8119B444A19784A
:10E13800444B51B198F80010117032781A70337846
:10E148000BB1542005E0522003E0117032785320BF
:10E158001A7003F037FC119B00241A783A4B1A7096
:10E1680098F80030234113F0010F2DD0214605986F
:10E1780014F0F9FF0122014628B923B20190009258
:10E188000293104605E0002123B200920191029308
:10E1980024200B4603F03AF8BAF1010F05D12B4BB6
:10E1A8008020DA790521013208E0022D07F1010209
:10E1B80002D18020072101E0802006212346F5F7BF
:10E1C8007DFE2046F5F71EFB3378234113F0010F3F
:10E1D80057D000214FF0010B23B2029302205A4678
:10E1E8000B46CDF800B0019103F010F8DA45DFF8DE
:10E1F80068900CD119F8243013EA0B0334D1134A70
:10E208000520D1790093594404EB0B022AE019F850
:10E21800243013F0010327D1022D1FD10C4B1B789A
:10E2280003F02403042B04BF0A4B83F800B0002337
:10E238000093072014E000BFC0310020A216002080
:10E248004B1500204C150020BF160020D6180020C2
:10E25800C8160020600E0020131500200093062029
:10E26800791C621CF4F748FA11992046F5F7F2F880
:10E278002046F5F7F3FA19F824306FF3000309F88C
:10E2880024300134042C7FF46BAF07B0BDE8F08F65
:10E298002DE9F04180460E46174646F60B15002438
:10E2A8003846214614F05FFF88B1294608220B48FA
:10E2B80002F03FFF0948414614F002FF074814F0F6
:10E2C80025FF20B90123A34032781343337001346A
:10E2D8000835042CE4D1BDE8F08100BFB716002052
:10E2E8002DE9F04387B08046894604A847F23531C6
:10E2F800082202F01EFF002440462146E7B214F02F
:10E3080032FF002843D03846F3F732FF0025661C59
:10E318000246314611202B460095F4F7EDF901230A
:10E3280021462A4604200095F4F7E6F9F80800F596
:10E338002640333002F0ECFE04F00703C1B2194165
:10E3480011F001014FF002024FF001030AD00092D0
:10E35800019336B27720294692182B46029602F08E
:10E3680055FF14E00092019336B2232004220B4695
:10E37800029602F04BFFB9F1000F08D004A821461D
:10E3880014F0F1FE18B10548214614F0D6FE013408
:10E39800402CB1D107B0BDE8F08300BF281500209C
:10E3A8002DE9F74F9846137805460C4617469DF811
:10E3B80030909DF834B09DF83800DFF8C4A073B1F0
:10E3C800294A51786FF3820151703B7800EA0303C0
:10E3D8003B7021789AF800208A18D31A2B7023787A
:10E3E80083B122482146F5F7E5F921491F4814F081
:10E3F80067FE1E480121FFF773FF1C48414622466D
:10E40800FFF746FF1B4B00261E70297843F6F720BE
:10E4180002F074FE494646F6490002F06FFE2046B7
:10E4280039464A46F4F790FF134B39469E704246E8
:10E438004B462046CDF800B00195FFF7EBFC284687
:10E44800F7F7D0FE2B780D480D498AF80030F5F71C
:10E45800B1F988F800603E7026702E7003B0BDE8F0
:10E46800F04F03F0BFB900BF0F340020C0160020E2
:10E478004315002008190020670E0020A31600206D
:10E48800FE14002010B50B4B0B4C024603CB20604A
:10E4980061600A48114614F034FE2146074814F01A
:10E4A8000FFE064814F032FED0F1010038BF0020FC
:10E4B80010BD00BF78250020AD160020B71600203B
:10E4C80010B50A4C637C4BB100200949FAF75AFA97
:10E4D800084B1B78432B01D1433B6374607C20B904
:10E4E8000549BDE81040FAF74DBA10BD06180020DE
:10E4F800B11803080418002090180308034B1A7871
:10E5080001321A7001230370704700BF08190020F8
:10E5180010B50C48FAF7DCF90B4A002414700B4AC2
:10E528000B4B14700B4ADC7014700B4A9C701470FF
:10E538000A4A1C7114700A4A1470FAF7E7FA094B70
:10E548001C6010BD18190020D618002005180020DE
:10E55800670E00200A190020161900204018002014
:10E56800081900203C1800202DE9F04F944B954ED7
:10E5780093F800903368DFF898829C7C924BF022E5
:10E588001A7098F800308BB00C2B354647463FD1AF
:10E598008E4B93F803C0BCF1010F04D9ED3A5A71C0
:10E5A80000208B492FE01AD10024DC70894A8A4B5D
:10E5B8008A498B488B4D04701C7014700C70CDF810
:10E5C80000C001942D780295FFF7EAFEFAF79EFA4B
:10E5D800854834600BB0BDE8F04FFAF779B9834845
:10E5E8007E49F5F7E7F8824B824A03CB824B1060ED
:10E5F8001B785160532B57D198F800307F4901336D
:10E6080088F8003000200BB0BDE8F04FFAF7BAB92F
:10E61800082B0FD1784B1B78532B3DD1784B002218
:10E628001A700C2388F80030764B1A7842F00602EC
:10E638001A707FE20D2B37D16F4B1B78532B2BD1E0
:10E6480071496A4814F03CFD6848FFF71BFF04460F
:10E6580040B198F800300522013B88F800305B4B48
:10E66800DA7067E2082246F64A01624802F061FD64
:10E678006049664814F045FD01230093594B019405
:10E688001B78574802935549524A534BFFF788FE67
:10E69800FAF73CFA34604DE2232B40F04B820BB082
:10E6A800BDE8F04FFFF734BF631E48BFA31DDB1062
:10E6B800013303FB09F91FFA89F909F5D046A9F5D1
:10E6C800B249A9F1CD094F4BCDF81C901A784A36BA
:10E6D80012F0010F4A4C00F01E81474B1A789946F8
:10E6E800432A40F0C7803B780C2B40F0C3803F485A
:10E6F800217814F038FD002800F0BC803D482178CE
:10E7080014F031FD002840F0B580079920780FFA01
:10E7180081FB0BEBD00002F0FBFC23784FF0010AE1
:10E7280003F007020AFA02FADFF8E8805FFA8AFAC9
:10E7380010EA0A0FC8F8000027D0244B5B78002B9A
:10E7480040F09880274BD879F7F7AAFC002800F00A
:10E758009180D8F80010CAF1FF0A20780AEA01016E
:10E76800C8F800100BEBD00002F0C8FC20780FFAB4
:10E7780086FB0BEBD00002F0CBFC00EA0A01207804
:10E78800C8F800100BEBD0005FE032B202EBD30008
:10E79800059202F0BDFC10EA0A0FC8F800003BD150
:10E7A80040EA0A01059B2078C8F8001003EBD00066
:10E7B80002F0A4FC2178154814F0BFFC5AE000BF11
:10E7C800C91800203C18002015190020670E0020E9
:10E7D800561903080A1900200518002016190020E8
:10E7E80040180020D618002018190020C016002054
:10E7F80078250020F4140020041800201C1A0308AF
:10E80800D3180020091900203815002043150020CE
:10E8180008190020E0180020924B5B7823B9924B2E
:10E82800D879F7F73DFCB8B92078DDF814C0CAF1FB
:10E83800FF0A0CEBD00002F06BFC8C4A00EA0A01DC
:10E84800059B2078116003EBD00002F057FC21787B
:10E85800874814F07DFC0DE020780BEBD00002F027
:10E8680057FC40EA0A012078C8F800100BEBD000EA
:10E8780002F044FC99F80030232B10D12A68237841
:10E88800927C013A93420ADA7A4A013313707A4B3E
:10E898009B7803F00203DBB20BB1F9F76FFF99F82D
:10E8A80000302A2B0CD1237853B1724A013B1370E4
:10E8B800714B9B7803F00203DBB20BB1F9F75EFFF3
:10E8C80099F80030552B12D129682278897C694B38
:10E8D80008398A4201DA083200E000221A70664BD1
:10E8E8009B7803F00203DBB20BB1F9F747FF99F805
:10E8F8000030442B0FD122785E4B072A9CBF2A6830
:10E90800927C083A1A705C4B9B7803F00203DBB2E6
:10E918000BB1F9F733FFFBF771FE584A23781178EA
:10E928009246994288BF137012780F32934202DDE3
:10E93800524A0F3B13702B684FF0000B93F812806C
:10E94800CDF818B0B8F10F0F9ABFC8F120085FFAD8
:10E9580088F84FF0100839784FFA8BF30C2905D155
:10E968009AF800209B18DB10454A04E09AF800202A
:10E978009B18444ADB10D35C9AF8002005934FFAA1
:10E988008BF39A180C2902F007094FEAE20202D128
:10E998003D49895C0691DDF81CC004930FFA8CF0A0
:10E9A800101802F0B5FBC0B2049B08909AF800005A
:10E9B80032B2181802EBE00002F0AAFB39789AF894
:10E9C8000020049BC0B209919A1846E0059BDDF827
:10E9D80024C043FA09F12D4B01F0010100290CBFB5
:10E9E800A521DB21BCF10C0F03F8081014D128492C
:10E9F8004FEAE20C11F80C1041FA09F111F0010F7D
:10EA080008D0DDF818C04CFA09F111F0010F03D055
:10EA1800582110E02D210EE0DDF820C04CFA09F154
:10EA280011F0010F01D0502105E040FA09F111F071
:10EA3800010F02D0542103F8081009F101095FFA07
:10EA480089F90BF1010B08F101080132B9F1080F3E
:10EA58005FFA8BFB5FFA88F81CD0B8F1200FB5D1AC
:10EA680025E000BF670E0020D6180020E01800201F
:10EA780043150020D318002018190020CB180020B7
:10EA88003815002098150020F4140020F401002007
:10EA9800C0160020B8F1200F09D09AF800304FFABC
:10EAA8008BF2D2182B689B7C9A42FFF654AF23490D
:10EAB8000B7813F0010F17D02B68214A9B7C127832
:10EAC8000F2B02F0800298BFC3F11003D2B294BF9B
:10EAD800DBB2002342B122789AF800101032521AA1
:10EAE8001849CB185F219954174EB37803F00203E5
:10EAF800DBB293B1F11D652246F6E1532078F9F7B0
:10EB08008DFE2B689B7C102B02D905200B2101E080
:10EB1800002007213246F9F7EDFE2B689B7C102B6D
:10EB280008D921780948013102220BB0BDE8F04F1D
:10EB3800F9F74EBF0BB0BDE8F08F00BF09190020F0
:10EB4800C0310020F401002018190020F501002030
:10EB58001FB5044611B100200B4901E008460B49D6
:10EB6800F9F710FF217810220139C9B201EB011120
:10EB780001F5C2414431684602F0DBFA1020014633
:10EB88006A46FFF70FF91FBD58F002089AF002080D
:10EB98000B4B1B78442B06D0552B037801D013B1AF
:10EBA8007047013B01E003780133037003780BB928
:10EBB800203302E0212B01D1203B0370FFF7C8BFAF
:10EBC800041800202DE9F74FDFF8CC91DFF8D8A121
:10EBD80099F80030554643F0010389F800309AF857
:10EBE8000130644C23F07F039B46D3B10020624977
:10EBF800F9F7C8FE61482A21F1F74AFC18B12178D3
:10EC08008222F9F7E5FE2278002A40F0AF802B68CF
:10EC180062F3CF332B605A4B1A7842F003021A7012
:10EC2800A4E0574F23703B783E4603F00202D2B26D
:10EC38000192DFF87881002A44D013F001092BD023
:10EC480058465049F9F79EFE98F80030232B0CD10E
:10EC58004D4B4E4A4E481A600121FFF779FF3B7829
:10EC680003F0FE036BF341033B7098F800302A2B46
:10EC78007CD1337803F0FE036FF3410333702B68C4
:10EC880043F400432B600F232370414B187803B0E3
:10EC9800BDE8F04F0EF054BD48463E49F9F772FE04
:10ECA80098F80030232B61D1374B384A38481A601E
:10ECB8000121FFF74DFF3B7869F3000369F3410336
:10ECC8003B7053E00EF08DFC054600282FD0012143
:10ECD8002F48FFF75DFF98F80030532B12D13B788F
:10ECE800019A03F0F10362F300033B70DAF8003095
:10ECF80043F40043CAF800300F232370244B1878DC
:10ED08000EF01EFD98F80030232B2FD13378002207
:10ED180003F0FD036FF3000333701D4B1A70F9F70E
:10ED2800F5FE1D4A137843F00603137014E01B49DF
:10ED3800F9F728FE98F80030232B17D13B7865F3B4
:10ED4800410365F300033B70F9F7E0FE99F80030E2
:10ED580043F0060389F80030114A1378013BDBB20F
:10ED68001370104A52F82320074B1A6003B0BDE80D
:10ED7800F08F00BF623B0020DCF00208F4010020A5
:10ED880023340020FDF002083C180020C49102083A
:10ED9800D31800201EF10208091900203FF10208CB
:10EDA800F7180020F8180020C031002004180020AF
:10EDB8002DE9FF41364C374D237843F0010323708A
:10EDC800297801F00401C9B211B93348FFF7E0FE10
:10EDD8002B7803F00402D2B232B1304A12781AB951
:10EDE8002C4A43F0080313702D4E3378232B26D179
:10EDF8002B782A4A6FF3C303002113F004082B7001
:10EE0800284F117009D0234A61F382031370264BEF
:10EE180021483B60FFF79CFE11E0F9F777FE237865
:10EE2800224A43F0060323701378013BDBB21370C8
:10EE38001F4A52F823303B60174B83F80080337821
:10EE4800532B23D12B780424144A03F0F4032343CF
:10EE580014702B70104B0B221D781649013DEDB232
:10EE680002FB05F000F5CA40843002F05CF900208E
:10EE78001149F9F787FDFF2300210093013516207A
:10EE880022460B460191029502F0C0F9BDE8FF81C8
:10EE98000919002023340020D3180020623B0020E9
:10EEA800041800203C180020E0910208F718002000
:10EEB800F818002018340020BBF002082DE9F041B2
:10EEC800984B04469A7812F0010F00F017811B88BE
:10EED800002B40F01381944D95F820303F2B40F2E1
:10EEE800D780012C14D1914B1B7803F00203DBB2BD
:10EEF800002B00F0C48095F820208B4B402A03D1CA
:10EF0800013283F82020FBE0482283F82020B6E075
:10EF1800022C03D1482385F82030B0E0844E3378A2
:10EF280003F02002D2B28AB195F82020402A0DD1F0
:10EF3800032C0BD07F4B804A03F1100153F8040BCC
:10EF48008B4242F8040BF9D1412395E003F01003FA
:10EF5800DBB28BB195F82030412B0DD1032C0BD0AF
:10EF6800764B754A03F1100153F8040B8B4242F8B3
:10EF7800040BF9D142237FE0F37813F0010F0FD08F
:10EF880095F82020422A0BD16D4B6B4A03F11001F2
:10EF980053F8040B8B4242F8040BF9D143236BE07E
:10EFA80003F00202D2B27AB195F82020432A0BD19D
:10EFB800644B614A03F1100153F8040B8B4242F889
:10EFC800040BF9D1442357E003F00402D2B27AB11A
:10EFD80095F82020442A0BD15B4B574A03F11001C6
:10EFE80053F8040B8B4242F8040BF9D1452343E054
:10EFF80003F00803DBB28BB195F82030452B0DD117
:10F00800032C0BD0514B4C4A03F1100153F8040B5D
:10F018008B4242F8040BF9D146232DE00FF076F924
:10F02800A0B14B4B1B788BB195F82030462B0DD1F6
:10F03800032C0BD0474B404A03F1100153F8040B43
:10F048008B4242F8040BF9D1472315E0F37803F01B
:10F058004003DBB29BB195F82030472B0FD1032C2E
:10F068000DD03D4B344A03F1100153F8040B8B4289
:10F0780042F8040BF9D1482385F8203078E095F858
:10F0880020300133DBB2472B85F820307FF629AFDB
:10F0980095F82060472E04D9234B002683F820607A
:10F0A80001E00136F6B206F14007FFB212E02B4844
:10F0B800314614F058F808B1032C04D1284B9B5D55
:10F0C80023B1032C02D185F820600FE00136F6B297
:10F0D800BE4203D03F2EEAD9402E07D1214B1E2233
:10F0E8001A70402385F82030BDE8F08195F820009B
:10F0F8001149652246F6E153F9F790FB012C37D107
:10F10800194B0D4A03F1100153F8040B8B4242F8D6
:10F11800040BF9D1044B93F820303F2B3CD9002045
:10F1280012493EE018190020F401002002150020C1
:10F13800C031002090F702081F190020B1F702081B
:10F14800D2F70208F3F7020814F8020835F80208A3
:10F158006036002056F8020898F802089815002032
:10F168004E150020D4180020905A03084EF70208C4
:10F17800104BD87800F02000C0B220B1022C06D085
:10F1880000200D490DE0032C01D10C4909E00C4B7E
:10F1980093F820303F2B02D800200A4901E00A49A1
:10F1A8000020F9F7EFFB1020084A0146BDE8F041BE
:10F1B800F9F7A0BBC031002069EE02086FF702081A
:10F1C800F40100200CF7020877F80208181900204B
:10F1D80010B5F9F79BFC084B1B7803F00403DBB26E
:10F1E8002BB106490020BDE81040F9F7CBBB02203F
:10F1F800BDE81040FFF762BE021500203EF5020888
:10F2080070B5224B06461B78214CF3B9257819E0D6
:10F218002048294613F0A7FF78B123689D4202D9F8
:10F22800FF2E02D007E0FF2E02D19D4208D202E055
:10F2380036B91DB913B9256012E00EB9013500E0E1
:10F24800AD19EDB23F2DE3D90AE0013B2021124868
:10F2580010222360F1F79EF800201049F9F792FB7D
:10F268000F48F9F735FB46F6E15320780D4965223A
:10F27800F9F7D4FA084D216805F11000013102228E
:10F28800F9F7A6FB2D23AB7470BD00BFC918002089
:10F29800E018002042180020F40100200C3903086F
:10F2A800181900201F190020F8B5544BF0225448B3
:10F2B8001A700378044613F00E0518D1514A43F02A
:10F2C8000203156000F8013B13F0F2FE2C464E4B8A
:10F2D800E35C1BB14D48214613F02FFF0134402C4D
:10F2E800F5D14B4B1A7842F001021A70F8BD13F0B1
:10F2F8000C0543D12E464548294613F034FF08B182
:10F308000136F6B20135402DF5D11EB9237843F008
:10F31800040331E000253F482946EFB213F023FFEC
:10F3280068B1394BEB5C53B13B4B01371F70002080
:10F33800FFF766FF237843F00803237002E00135E6
:10F34800402DE8D1354D3A212846F1F7A1F838B1DA
:10F35800401BC0B20130281831460222F9F738FBA9
:10F368002F4B1B78532B47D12B4B00201870FFF7DE
:10F3780047FF237843F008032370F8BD6FF3410378
:10F38800037003F00403DBB2254D23B100202549A7
:10F39800F9F7F8FA0EE02B78552B01D1FF2002E09F
:10F3A800442B02D10120FFF72BFF13200D211E4A09
:10F3B800F9F7A0FA2B78232B1ED1227802F0020449
:10F3C800D4B90F4902F0FB0264F3C3020A700D4A74
:10F3D8001460F9F79BFB0E4B1A7842F006021A707C
:10F3E800124A1378013BDBB21370114A52F82320FA
:10F3F800104B1A60084B1C70F8BD00BF151900208F
:10F4080041180020E0180020E823002042180020BE
:10F418000919002003150020C9180020F401002054
:10F4280004180020524A030818190020F718002071
:10F43800F81800203C18002070B505460C46164602
:10F448003BB143004AF20D5018184018114601F01C
:10F4580055FE054B292202FB0535F3092C1906F048
:10F468007F066370E67070BDEB32002038B510B3CC
:10F47800A0F14103DBB2432B1FD9C50900F07F047B
:10F488000BD0052C19D90021601E0A460BF084FA0E
:10F49800D0F1010038BF002038BD082C0FD9601EFC
:10F4A800C0B229462A460AF0C5FE50B9202C8CBFA6
:10F4B8000020012038BD012038BD002038BD284675
:10F4C80038BD284638BD0000F7B5614C3123237498
:10F4D800604F01332376053B637463763B784AF2C9
:10F4E8000D505B00181801F013FEC0B220F07F0227
:10F4F80000F07F01D2B28DF804108DF8002004F1DD
:10F50800120359B9544A04F115001188927861829E
:10F518009A7020210222F0F73DFF0CE0D20904EB9B
:10F528008202526A10886082927804F115009A70FB
:10F538000222F9F74DFA3878400000F5244000F52A
:10F54800877001F0E5FDC0B220F07F0300F07F0175
:10F55800DBB28DF805108DF80130404851B93E4BAB
:10F5680020311A889B786283837002220330F0F777
:10F5780011FF0BE0DB0904EB83035B6A1A886283E3
:10F588009B78022283700330F9F722FA344B1B78F8
:10F5980013F0010F5AD0334D02A92A788B1813F8AB
:10F5A800041C13F8086C304B1B78232B04D1002A59
:10F5B80041D1223B2B703EE02A2B04D1002A3AD0BD
:10F5C800013A2A7037E0552B46EA010611D10DE0C1
:10F5D8002B7802AAD318013E13F8081CF6B230465D
:10F5E800C90913F8042CFFF741FF98B9002EEFD191
:10F5F80021E0442B19D115E02B7802A9CB1801364C
:10F6080013F8081CF6B23046C90913F8042CFFF7A2
:10F618002DFF38B1134B3878197832460123FFF79C
:10F628000BFF08E0872EE7D905E0532B03D1533BA6
:10F638002B70FAF7E3FF0D4B1B7803F08003DBB266
:10F6480023B12B782022023304F83320FEBD00BFFB
:10F65800F4010020C91800204F5603080E020020AC
:10F6680009190020D318002004180020C0310020F8
:10F67800024800210922F0F78DBE00BFE5180020DE
:10F6880070B50A46002405E01B19811A2A250134A1
:10F698005D54E4B20F4D104B295D09B19442F3D18A
:10F6A800801A001918182021121BF0F773FE0B4B53
:10F6B8001E7876B1432E07D114B1013CE4B201E0C3
:10F6C800074B1C7000232B553046F9F717FA00B189
:10F6D8002E5570BDE5180020F40100200418002004
:10F6E8001719002038B5184C184DA07800F01000F4
:10F6F800C0B250B91649F9F745F9FFF7B9FF2368C1
:10F7080043F4801323600F232B702A782AB92368C7
:10F71800FF2062F31453236038BD0E48C5792DB914
:10F728001C200821FFF7ACFF284638BD23680A498A
:10F738006FF3145308222360F1F7ACF800280CBFCC
:10F748000120FF2038BD00BFC0310020171900205C
:10F75800A1F50208E51800208E750308F0B55B4C8A
:10F7680085B0667806F01006F6B2002E3ED1584BEA
:10F778001A78584B013A53F82230574A934204D129
:10F78800564B1A7842F0020207E002F11C018B4244
:10F7980008D1524B1A7842F00402022161F3C702E1
:10F7A8001A7019E03832934216D1FFF79BFF0028F0
:10F7B80000F08A800128494D06D12B78022243F0B7
:10F7C800010362F3C70306E030464549F9F7DAF862
:10F7D8002B7866F3C7032B70424B1A7842F001026C
:10F7E8001A70236843F4805323606DE03B4D2B78F7
:10F7F80013F0F80606D03C49002005B0BDE8F040FB
:10F80800F9F7C0B813F0070F3FD003F00202D7B2E0
:10F818004FB1122031460FF00DFFFF2300930196E0
:10F828000296432028E003F00406F6B296B1394662
:10F8380038460FF0FFFE0FF049F90AF0CBFA0DF049
:10F84800F7FEFF23009301970297442039460422CC
:10F858003B4614E013F0010F13D0012143F61C605E
:10F868000FF0E8FE3046F6F785FC204B45201E8059
:10F87800FF2300930196029631460422334601F095
:10F88800C5FC00201A49F9F77DF82B7803F0FA0334
:10F898006FF341032B70174B1B78232B14D123686C
:10F8A8006FF30C332360F9F731F90E4B1A7842F0F5
:10F8B80006021A70064A1378013BDBB21370054A38
:10F8C80052F823200C4B1A6005B0F0BDC03100205F
:10F8D800F7180020F8180020FC910208E5380020ED
:10F8E800C2F5020809190020EE4D03081A18002075
:10F8F800CD4D0308041800203C1800201FB504460D
:10F90800F6F724FDA8B14B2002F05CF8FF23009322
:10F918000121FF3B0193392004220B460134029454
:10F9280001F074FC064B01205A7842F004025A7028
:10F9380004E0044B1888003818BF012004B010BD3B
:10F94800F8330020783B0020F0B5204E0024337AAD
:10F958000546013385B00F46337210202146012237
:10F9680023460094F2F7C8FE55B9FF2300934F20B1
:10F97800294604222B460195029701F047FC0EE028
:10F98800012D0CD1FF230093502023462146042249
:10F998000194029701F03AFC337A013B3372337ACF
:10F9A800052B11D1FA3301210024009327200B469F
:10F9B80004220194029401F029FC044B1C7205B046
:10F9C800BDE8F04001F0D0BF05B0F0BDD61800206A
:10F9D800074B292202FB00335B7913F0100F05D087
:10F9E800044B283A9A711A710932DA71704700BFCC
:10F9F800EB320020670E0020044B1878A0F1010CB0
:10FA0800DCF1000040EB0C00704700BF3818002004
:10FA1800034B1878A0F10202504240EB02007047F5
:10FA280038180020034B1878012894BF00200120C3
:10FA3800704700BF38180020064B1A7802F0F7020A
:10FA48006FF304121A70044B00221A70034B03322E
:10FA58001A707047E4180020171900203818002081
:10FA680010B52148214903680A789C7B944203D940
:10FA78009C8914F0200F18D09A8912F0800F01D1B8
:10FA880005E01C3B9A8912F0400FFAD000E01C33C5
:10FA9800036000230B7003689B8913F0200F16D0B6
:10FAA800134BDA79114B1A7011E00132D2B20A7095
:10FAB800986843F60553984209D101E00132D2B261
:10FAC800162A03D80B4853B29840F7D40A700A4A4A
:10FAD800136843F480731360F8F75CFE074B1A78D9
:10FAE80042F006021A7010BD3C180020C918002008
:10FAF800D618002000060088C0310020091900200F
:10FB080010B52349234A0B78D3B11068848914F0BF
:10FB1800200F15D1013BDBB20B70846843F6055208
:10FB2800944228D104E013B1013BDBB200E0837BAF
:10FB3800162B03D8184C5AB29440F4D40B701AE020
:10FB48001368988910F0400F01D106E01C3398899A
:10FB580010F0800FFAD0136002E00E481C3B0360DF
:10FB680013689A7B0A709B8913F0200F03D00B4B04
:10FB7800DA79074B1A700A4A136843F480731360E2
:10FB8800F8F708FE074B1A7842F006021A7010BD03
:10FB9800C91800203C18002000060088D61800204C
:10FBA800C031002009190020074B084A1B689342FE
:10FBB80002D01C32934205D1054B1878003818BF83
:10FBC80001207047002070473C180020509202081E
:10FBD800FE140020074B084A1B68934202D01C32CF
:10FBE800934205D1054B1878003818BF012070479B
:10FBF800002070473C18002088920208FE1400205C
:10FC080070B50A4C0546E07100F56A50783001F08D
:10FC18007FFA207005F5D840B53001F079FA6070A8
:10FC28002046BDE87040F6F7BDBA00BFD6180020E0
:10FC38002DE9F0479A4B86B01A7806460F461C46BF
:10FC48001AB1012A40F0DA812FE0964B1A68964BD8
:10FC58009A4200F0D581F6F701F8944B5B7803F0EF
:10FC68000203DBB253B9924B5B7803F08003DBB23B
:10FC780023B901F09FFE08B90AF0ACF88D4B1A6859
:10FC88006FF310421A6037B98B4B1878F8F736FFC4
:10FC9800002800F0B581FFF7EBFC884B3C221A7076
:10FCA800F8F778FD237801332370844B1B7813B958
:10FCB800FFF7C2FEA4E1012130460AF0ADF8F8F7DB
:10FCC8005DFD00207E49F8F75DFE06211B20FFF749
:10FCD800D7FC7C4B7C491A7898468A1812F8312C44
:10FCE800002A00F08D81794A7949137891F80090BB
:10FCF800C3F3C00AC3F3001503F0F7036FF304134B
:10FD080009F00109137017B10223237000E027706E
:10FD18000B21062204A801F00CFA98F8002004A888
:10FD28006949303AF0F75CFA044610B1122700240A
:10FD380029E049F2BF7001F0EBF90028F6D0654DD3
:10FD48002C72F6F7E9F80446002840F05981624A17
:10FD5800544B21461A60FF2300930190029004221D
:10FD68000820234601F052FA012223460E2021469C
:10FD78000094F2F7C1FC594B1A7842F004021A7049
:10FD88000123AB713CE13946062204A801F0D1F900
:10FD980098F8002004A84C49303AF0F721FA0028D6
:10FDA80040F020812046FFF7A9FD002840F0288177
:10FDB800DFF82081012188F808002046F6F7BAF814
:10FDC80049EA0A090746F6F7A7F8002840F0BF8075
:10FDD80038464349F0F7E2FBC0B901F003FD314B67
:10FDE800B9F1000F02D115B93E4A24E035B13E4AB7
:10FDF8001A603E4B1A786FF3410205E03C4A1A60DC
:10FE08003A4B1A7865F341021A70E5E038463949E9
:10FE1800F0F7C4FB20B138463749F0F7BFFB78B993
:10FE2800B9F1000F40F0EC80002D40F0E98001F0BE
:10FE3800D9FC324A1B4B1A603046FFF7C9FDCBE0AC
:10FE480038462F49F0F7AAFB50B949F2BD70012195
:10FE580001F054F9174A136843F400531360DFE7BD
:10FE680038462849F0F79AFB40B9B9F1000F40F03D
:10FE7800C780002D40F0C480234A0DE0384623494E
:10FE8800F0F78CFB002845D1B9F1000F40F0B8809D
:10FE9800002D40F0B5801E4A024B1A609CE000BF5E
:10FEA800381800203C18002050920208AA2B002085
:10FEB80007340020C0310020041800201719002042
:10FEC80048EE020820180020E5180020E418002059
:10FED800C3460020D6180020C09202082221002024
:10FEE800F17D03080C950208949602080919002070
:10FEF8006C9202086D7D0308FD7F0308B096020826
:10FF0800A87D0308AA7D0308E8960208BA7F0308BB
:10FF18008892020838463C49F0F740FB00285BD13C
:10FF280001F060FCB9F1000F07D0384A384B1A606D
:10FF3800384B1A786FF3410261E0002D60D0364AE1
:10FF4800334B1A60334B1A7869F3410257E038464D
:10FF58002D49F0F723FB054628B901F043FCB9F118
:10FF6800000F4DD01EE038462C49F0F717FB00284B
:10FF780046D038462A49F0F711FB40B9B9F1000FCD
:10FF88003ED1284A224B88F807401A6038E03846A4
:10FF98002549F0F703FB054660B9B9F1000F16D003
:10FFA80001F020FC194A1A4B1A601A4B1A7865F3AB
:10FFB800410224E038461D49F0F7F0FA20B13846EE
:10FFC8001B49F0F7EBFA10B9B9F1000F18D1194A2B
:10FFD8000F4B1A6001F006FC2046FFF711FE202C9B
:10FFE8000ED105E00134E4B20737202C7FF4CBAE04
:08FFF800711C0020C9B2FFF7E3
:020000040801F1
:10000000A7FC01E000221A7006B0BDE8F08700BF2F
:10001000AC7D03086C9202083C18002009190020EE
:1000200094960208AA7D0308BA7F03088892020802
:10003000F17D03086D7D0308A87D03083C97020845
:10004000034B1B7853FA00F000F00100704700BF2B
:10005000D6180020034B1B189878003818BF0120D1
:10006000704700BFD6180020F8B504460D460E783C
:10007000FFF7F0FF18B3144A13199F7810460023B6
:10008000021992781A4112F0010F4FF001020DD0BF
:10009000BE42297803D09A4042EA010104E09A4026
:1000A000C2F10F0202EA0101297005E09A402978A5
:1000B000C2F10F020A402A700133042BE0D12B78E1
:1000C00003B92E70F8BD00BFD618002070B57E4B66
:1000D000044631B11B78532B40F0F580533B03703D
:1000E00070BD1A78302A33D1784B1A795AB1784AD0
:1000F00078491278292000FB0212527912F0100F71
:1001000001D001221A71744A25781278154012D054
:10011000DD79002D40F0D780E8B2FFF791FF30B1D4
:100120000123AB402278C3F10F0313402370013544
:10013000042DF1D141E0E8B2FFF782FF20B10123A5
:10014000AB402278134323700135042DF3D134E002
:10015000A2F13101C9B203293BD85C4E32795AB1C0
:100160005B4A5C491278292000FB0212527912F096
:10017000100F01D0012232711D78313DEDB22846B9
:10018000FFF75EFF002800F09E80237853FA05F207
:1001900012F0010F0BD0F279002A40F09480013266
:1001A00012FA05F5C5F10F0505EA030304E0012283
:1001B00012FA05F545EA030323700021122247488D
:1001C000F0F7ECF8454920461022BDE87040FDF7F5
:1001D000BBBD132A0CD0552A18D13D4B3D4A1B7884
:1001E000292101FB03235B7913F0200F03D170BD9C
:1001F000364B01221A7100202146FFF735FF0020FF
:10020000FFF728FF00285ED0002054E0142A0CD00D
:100210002A2A18D12E4B2F4A1B78292101FB0323B0
:100220005B7913F0200F03D170BD284B01221A71A6
:1002300001202146FFF718FF0120FFF70BFF0028E0
:1002400041D0012037E0152A0CD0232A18D1204BA9
:10025000204A1B78292101FB03235B7913F0200F2F
:1002600003D170BD194B01221A7102202146FFF7FC
:10027000FBFE0220FFF7EEFE002824D002201AE049
:10028000162A0CD0442A1ED1114B124A1B78292160
:1002900001FB03235B7913F0200F03D170BD0B4BDF
:1002A00001221A7103202146FFF7DEFE0320FFF72B
:1002B000D1FE40B103200949102246F64573BDE83E
:1002C0007040F8F7AFBA70BD04180020670E002028
:1002D000CC180020EB320020D61800200618002091
:1002E0002DE9F043002387B08DF81730794B1B7848
:1002F000012B00F06E82784C227872B1774B5B78DC
:10030000002B40F06682764D2B78002B40F0AA80BF
:10031000F8F700FC08232B70A4E0714B19781D46F8
:10032000072900F29F806F490978232913D11A7099
:10033000F8F7F0FB6C496D4A0B7853B16C48013B00
:100340000478DBB244F0060404700B70694951F87C
:1003500023301360B1E2664B1A7812F0010F04D11A
:1003600001210A438DF817101A70F2F7FDFD28B924
:100370002B781BB90DF11700FEF7C4F8F2F702FE57
:1003800030B92B78012B03D10DF11700FEF7BAF825
:10039000F2F706FE30B92B78022B03D10DF11700CE
:1003A000FEF7B0F8F2F708FE30B92B78032B03D133
:1003B0000DF11700FEF7A6F8F2F70CFE48B9F2F7B8
:1003C00025FE30B92B78042B03D10DF11700FEF771
:1003D00099F8F2F759FE30B92B78052B03D10DF1BE
:1003E0001700FEF78FF8F2F743FE30B92B78062B93
:1003F00003D10DF11700FEF785F8F2F7F9FD30B9DA
:100400002B78072B03D10DF11700FEF77BF89DF831
:1004100017303BB32B78072B1FD8DFE803F0040716
:100420000C0F1215181B0020334901E0334900203E
:10043000F8F7ACFA13E000203149F9E70020314920
:10044000F6E700203049F3E700203049F0E70020CC
:100450002F49EDE700202F49EAE7F8F75BFB2A7800
:100460002D4B1A701E4F3B783D46082B40F0BC8048
:100470001F4B1C4F1978984611F001015BD1274E94
:1004800012223046EFF78AFF0123737413F05AFFEC
:1004900010B92278224B1A70237803B97374737CD5
:1004A00013B1204B00221A70FEF70EF81C48717C25
:1004B000FFF70CFE98F8003003F0FD0343F0010352
:1004C00088F80030184B1A7882B33A7000221A70FC
:1004D00031E000BF15190020FE140020670E002037
:1004E0000819002004180020F71800203C180020EC
:1004F00009190020F8180020021F0308E11E030854
:10050000231F0308441F0308651F0308861F0308F1
:10051000A71F0308C81F030859460020061800201B
:1005200040180020600E0020CD18002013F00AFFB4
:1005300008B930233B703B78884E13B93379112BBF
:100540004ED1DFF86892FDF7BFFF854899F811108A
:10055000FFF7BCFD824B1A78984622B1002010218B
:100560004A46FDF723FC237898F800407D4A24EAA8
:10057000030111707C4A23EA040111703A78A2F158
:100580005200C0B2012803D93079744F11280CD120
:10059000002333711CB911B10133009311E104231D
:1005A000F3702B7801332B701AE0432A18D1BBB9B2
:1005B0007C78ACB96D4BD879F5F776FD38B96C49D4
:1005C000F8F7E4F90523FB7007332B7004E02046AD
:1005D0006849F8F7DBF9FC70674A684B1A606CE110
:1005E0005F48FDF709FC68E1092B31D15D4807F050
:1005F0007FF8C6B2594C36B3E378042B02D1002001
:100600005F4903E0022B04D15E490020F8F7BEF9F0
:1006100002E00BB90433E370314602225A48F8F77E
:10062000DBF95A4B1E78232E00F0D3803046F8F7C2
:1006300069FA002800F04181312E40F03E812B788C
:1006400001332B7002E03B7801333B70042332E02E
:100650000A2B32D1434807F031F8C6B23F4C36B3CB
:10066000E378042B02D10020494903E0022B04D196
:1006700048490020F8F78AF902E00BB90433E37027
:10068000314602224048F8F7A7F9404B1E78232E46
:1006900000F09F803046F8F735FA002800F00D8111
:1006A000312E40F00A812B7801332B7002E03B7829
:1006B00001333B700823E370FFE00B2B40F0FD801B
:1006C000284806F0E1FF0021C4B2264806F0B2FF38
:1006D000002C6DD0214EB3782BB9BE2013F06CFBEB
:1006E000B3780133B370F3781C4A092B02D9002088
:1006F0001F4915E010D11D4B00241C70D470264BEF
:10070000194A1849164801251C7014700C700470A1
:100710000095019402949EE0082B04D11F4900200B
:10072000F8F734F911E0062B02D100201C49F7E755
:10073000042B02D100201B49F2E7022B02D100203A
:100740001949EDE70BB90833D370F378082B3CD87F
:100750000D4821460222F8F73FF936E0670E0020E7
:1007600040180020161900200A190020D618002071
:1007700056190308D2180308589702083C1800209D
:10078000DA190308FB190308F401002004180020FB
:1007900098190308B919030805180020F31803086D
:1007A00014190308351903087719030806180020DF
:1007B000012543484349444A2B460095F3F7B0F9D5
:1007C0000095424B01941B7840E0414F3C78232C2C
:1007D00002D1FDF7A1FE70E02046F8F793F900285A
:1007E0006BD0303CE4B2631EDBB2012B3C7039D8D5
:1007F000022C364D1ED1E879F5F756FC002838D08A
:100800002F48FDF743FE002833D1082246F64A015F
:10081000304800F092FC2A492E4812F060FC2D4925
:10082000082246F64A0000F082FC2A492A4812F0C3
:100830006CFC06E0012322482249234A0093F3F787
:100840006FF901230024009301942B78029323482D
:100850001D49234A1B4BFDF7A7FDF8F75BF9214B18
:100860001C602AE0032C28D1184BD879F5F71CFC22
:1008700010B90C23F37020E013F064FD70B9044646
:100880000F48214612F073FC28B1E02013F094FACF
:10089000204613F0CDFA0134402CF1D1124A002346
:1008A0001370F3702B78114A01332B700D4B1A60C3
:1008B0000F4B1A7842F006021A7007B0BDE8F083B9
:1008C000C01600200518002016190020D618002098
:1008D00004180020F41400204315002040180020C4
:1008E0000A1900203C180020D3180020589702084D
:1008F00009190020184A00231360184A1848137079
:10090000184A1178037001F0F60163F307111170B2
:10091000154A1648117863F301011170144A1178D1
:1009200063F3C5011170134A1370134A117801F073
:10093000FC0163F382011170104A1168037021F405
:10094000805163F3CF3111600D4A117801F0F40149
:1009500063F38201117070473C180020F7180020E3
:10096000D3180020091900201D1800201419002098
:10097000CE180020D5180020E4180020C031002037
:10098000233400202DE9F04F6A4B6B4D1970A0F114
:100990001103DBB2012B87B00E46287006D812284F
:1009A00001D1113800E00020F5F746FC2B78522BDE
:1009B0000DD1F2F7B5FB28B9F2F7A6FB10B9F2F7A3
:1009C000C7FB20B15D4B1A7842F008021A705C4BED
:1009D0005C4C1B782BB922685B4B9A4201D0FFF725
:1009E00089FF2368002B40F04081584F7B7803F04B
:1009F0002003DBB273B1564B93F80080B8F1000FBF
:100A000008D149F2BD70414600F07CFB3B6868F3B9
:100A10004D333B604F4B187810F01E0002D0002081
:100A20004D4907E04D4B93F805909846B9F1000FFA
:100A300005D04B4907B0BDE8F04FF7F7A7BF494FC6
:100A400097F801B0BA46BBF1000F2DD0BBF1070FEC
:100A500015D94548F7F740FF4449B878652246F66E
:100A6000E163F7F7DFFE3878072310F003007B70AF
:100A70000EBF3F4948463F49F7F788FF0CE0BBF1FE
:100A8000020F09D83848437823B1F7F725FF87F8D4
:100A900001908AE202237B701020334A014607B09E
:100AA000BDE8F04FF7F72ABF334B9A795AB183F874
:100AB00006B000F093FC8E20594601225B46CDF82B
:100AC00000B0F1F71DFE0020F2F77EFC2B4A2C4906
:100AD00013782C4843F00603137000230B702A4947
:100AE00023600B7088F8013088F8043003702933D4
:100AF0007343264F9146F95C8346C1F3C00111B997
:100B00003046FFF799F8292303FB06777B7913F02A
:100B1000100F04D02A78133AD2B2032A3AD913F02C
:100B2000200F5DD02B78442B34D031D8232B31D0FB
:100B30002A2B2EE0CC18002004180020401500209D
:100B4000151900203C18002058970208C0310020D9
:100B5000FE140020613B0020ABEE0208670E00206F
:100B60000A200308D0180020181900201F1900209F
:100B7000B3EF020892EF0208D618002009190020EE
:100B8000F7180020CD180020C9180020EB320020F3
:100B9000552B25D1844B1B7813BB844B1F78FFB991
:100BA00043F6DB2000F0B8FA0128014618D188F896
:100BB00001001F200591FFF727F899F80030304613
:100BC00067F3410389F80030059909F029F9F7F72F
:100BD000A1FF774B2360774B1F602B788BF8003099
:100BE0002B78432B0AD1714B1B783BB90121724BF7
:100BF00088F801103046236009F012F92878173878
:100C0000C3B2072B27D86D49FF220AF0D7FF9AF805
:100C100000106B4B60F301018AF8001001F0030132
:100C2000022918D00122032041B1009001929B7843
:100C300068309B1802930021033206E00090019275
:100C40009B786C200133029304220B4600F0E2FAF9
:100C5000FF238AF8013098F80630002B00F0A581B8
:100C600052232B70574B00229A712268524B9A42A2
:100C700050D12878A0F14303DAB2122A22D8524A7E
:100C80005BB29A401ED5432840F08F81464B1B78BB
:100C9000002B40F08A8100F0B3FD4C4B48B11A782C
:100CA00003201109013191FBF0F000EB4000091A1B
:100CB00004E01A781109013101F0070161F307120C
:100CC0001A7072E1F7F71EFF002823D03F4F3B78E0
:100CD00013F0F00108D161F307133B703C4B216026
:100CE0001A7842F008020EE0102913D100F088FDB6
:100CF00080B13B7800216FF307133B70344B2160C8
:100D00001A7842F0100230461A7007B0BDE8F04F72
:100D1000FEF792BF2F4B1E211A78254F61F3460232
:100D20001A702B78232B1CD12368BB4219D12A4B74
:100D3000292202FB0636737913F0100F11D0274BCE
:100D40001B7873B1264EF7F7E5FEFDF7E5FBF0796A
:100D500000F56A50783000F0DFF93070AA20F2F721
:100D600033FB1A4E337813F0010F41D02368BB4296
:100D70000BD01C4A934208D0FEF71AFF28B9FEF7A1
:100D80002DFF10B9AA30F2F71FFB2268164B9A42CA
:100D900002D10020F2F718FB2B78522B40F0CA80CA
:100DA000124B53221A70C5E0FE14002038180020A0
:100DB0003C970208F818002050920208D218002030
:100DC000D0180020670E0020002000C00919002064
:100DD000E418002086190020EB320020F7180020CC
:100DE000D6180020589702087497020804180020AB
:100DF0002368BB420BD06E4A934208D0FEF7D8FE60
:100E000028B9FEF7EBFE10B9AA30F2F7DDFA2B781D
:100E1000552B1ED1FEF778FE3378664843F0060363
:100E200033708378644F03F00203DBB24BB1F7F702
:100E300053FD23681868FBF765FC3B786FF34103AB
:100E40003B705E48837803F00203DBB20BB1F7F727
:100E500043FD2B78442B1ED1FEF706FE3378554810
:100E600043F0060333708378534F03F00203DBB281
:100E70004BB1F7F731FD23681868FBF743FC3B786B
:100E80006FF341033B704D48837803F00203DBB2FC
:100E90000BB1F7F721FD2B78522B09D133780022C3
:100EA00043F001033370464B1A70464B45321A70BB
:100EB000454B00271F702B78232B3BD1434B3D48DC
:100EC0001F70434B1F70F7F707FD3C48F7F704FD11
:100ED0003378404943F0060333700B78364A1BB32E
:100EE0003D4A013B17703D4ADBB20B7052F823308C
:100EF0003B4A23609B68934202D109F08DFF19E0C1
:100F000002F59A718B4203D002F5E0718B4204D155
:100F10000120014607F0D4F80CE002F5EE7293428E
:100F200008D1304B1F7005E0117863F30711117081
:100F300023603AE02C4B5B7813B10020F2F744FABF
:100F400023681F7B17F00F0702D1FCF7CFFD1BE0D2
:100F5000012F02D1F9F70AFD16E0022F02D1FAF7AC
:100F600085FC11E0082F05D84FF09C53BB4001D5FC
:100F7000FAF742FF042F03D123689B69984703E0E7
:100F8000052F01D1FAF7F0F9337803F00203DBB251
:100F90001BB123681868FBF7B5FB33786FF3410387
:100FA00033702B780BB1084A137007B0BDE8F08F8F
:100FB0005897020818190020091900204C18002021
:100FC000D3180020041800201E180020D518002077
:100FD00014190020F7180020C9180020F818002064
:100FE000909702084B180020670E0020034B1868EA
:100FF000034BC11A484240EB010070473C180020E7
:1010000088920208044B1868044BC3EB000CDCF117
:10101000000040EB0C0070473C1800203C97020891
:10102000034B1868034BC31A584240EB0300704748
:101030003C1800206C920208034B1868034BC21A3C
:10104000504240EB020070473C1800200C9502080B
:10105000034B1868034BC11A484240EB010070472C
:101060003C180020B096020808B5FFF7F1FF28B938
:10107000FFF7E2FF003818BF012008BD012008BDBE
:10108000044B1868044BC3EB000CDCF1000040EB90
:101090000C0070473C18002058970208014A024B88
:1010A0001A607047C49102083C180020014A024BA4
:1010B0001A607047E09102083C180020B0380A4BD3
:1010C00004280ED8DFE800F0030507090B00074AE3
:1010D00008E0074A06E0074A04E0074A02E0074A38
:1010E00000E0074A1A6070473C1800209C9B0208E9
:1010F000B89B0208D49B0208F09B02080C9C0208D3
:101100006C92020807B502AB03F8011D19460122D3
:10111000002305F0FBFB0EBD07B5002302A901F873
:10112000013D012205F05AFC9DF807000EBD08B5EF
:10113000002305F0EBFB002008BD034610B5084670
:101140001446194605F04AFCE0B210BD10B503463E
:10115000002484540846194605F040FC204610BD82
:1011600037B50546002400E01446012260190DF150
:10117000070105F033FC9DF80730621C203BDBB211
:101180005A2BF1D920463EBDF8B500252C461E4B02
:101190001C21585D01FB0431400000F574506230A1
:1011A000043102220134FFF7C2FF1C355C2CEED162
:1011B0004FF46F5420B2042205341449FFF7B7FFEF
:1011C000A4B243F6D4339C42F4D1002548F6BC5770
:1011D0002C4615E007EB460004EB440100B2591819
:1011E0000222FFF7A4FF0136F6B2094B5A19927892
:1011F000B242EFD8013480370335142CBFB201D08E
:101200000026F2E7F8BD00BF3CC202086F7D03086C
:101210004CCC02082DE9F347044615468A460222C3
:1012200043F61A610DF106001E46BDF930909DF897
:1012300028809DF82C70FFF780FF2F4B2F499A785C
:10124000BDF906008A705A7800EBC000CA701A799E
:1012500000F578500A715A791C304A719A791B78D6
:1012600045EAC6158A710C7081F80190CB710D7238
:1012700000B20922FFF75BFF1EB1214B1A88013231
:101280001A80BDF8063001339BB2B3F57A7FADF812
:10129000063002D30023ADF8063002220DF106011C
:1012A00043F61A60FFF743FFBDF80600154B1880A0
:1012B00000B200EBC00000F5785000F11C052430AE
:1012C00000B2FFF729FF10F0800F03D00C4B1A88F3
:1012D000013A1A8028B20021FFF714FF0A4B03F8E5
:1012E000148003EB44046770BAF1000F02D00120B0
:1012F000F4F744FFBDE8FC87EC380020EE1800202E
:101300001A180020A82B00203D2900202DE9F743C2
:10131000314B1D78303DEDB2C5F10606F6B23EB355
:1013200005F11207202413E008F101080FFA89F0F3
:1013300000215FFA88F8FFF7E5FE09F10109B045E1
:101340001FFA89F9F0D1013C0737E4B2BFB21CB1F2
:10135000B9464FF00008E7E70B35013428B2002109
:10136000E4B20135FFF7CEFEB442ADB2F5D131E0C3
:10137000122425B2684629460622FFF7DEFE9DF8B4
:10138000003043B19DF805302BB99DF803308DF83E
:1013900004308DF805300734062228466946A4B289
:1013A000FFF7C5FEF22CE4D168460B210622FFF7B9
:1013B000C4FE9DF8003043B19DF805302BB99DF86F
:1013C00003308DF804308DF805300B206946062275
:1013D000FFF7ADFEBDE8FE832018002070B509F0D0
:1013E0001BFD0CF0C5F906F02FF805F055FFF2F7DC
:1013F00087FAA648F4F7F4FE43F6D120FFF78CFEF7
:10140000A34BA44C187043F6D020FFF785FEA24BE7
:10141000187043F6DC20FFF77FFEA04B187043F6F0
:101420000350FFF779FE9E4B187043F60450FFF708
:1014300073FE9C4B187043F6DA20FFF76DFE9A4B53
:10144000187043F6D920FFF767FE984B187043F6E3
:10145000CF20FFF761FE964B187043F6CC20FFF7C4
:101460005BFE944B187043F6D220FFF755FE924B6B
:10147000187043F6DF20FFF74FFE904B187043F6CD
:10148000E820FFF749FE8E4B187043F6DD20FFF78A
:1014900043FE237801280CBF43F001036FF30003E0
:1014A000237043F6E020FFF737FE237801280CBFB6
:1014B00043F080036FF3C713237043F6E720FFF771
:1014C0002BFE804B01281A6843F6ED200CBF42F03A
:1014D00000526FF35D721A60FFF71EFE7A4B18B967
:1014E0001A7860F3000202E01A7842F001021A70E2
:1014F00043F6EA20FFF710FE637801280CBF43F0A3
:1015000001036FF300036370704843F66E210822F5
:10151000FFF713FE6E4B00241C705C706B48235C5D
:10152000312B03D11030214611F00BFE0134082C71
:10153000F4D1224643F6F6116448FFF7FEFD224639
:1015400043F63A216348FFF7F8FD47F2573104228A
:101550006148FFF7F2FD47F25B3104225F48FFF775
:10156000ECFD0DF041FDF5F743F943F6E120FFF7FF
:10157000D3FD5B4C237860F30003237043F6E22035
:10158000FFF7CAFD237860F34103237043F6E4209C
:10159000FFF7C2FD237860F3C303237043F6E62010
:1015A000FFF7BAFD237860F34513237043F6E92073
:1015B000FFF7B2FD237860F38613237043F6E5202E
:1015C000FFF7AAFD237860F30413237043F6EB20A2
:1015D000FFF7A2FD237860F3C713237043F6E320DF
:1015E000FFF79AFD237860F3820323703D48FFF7ED
:1015F00093FD3D4B3D49052218703D48FFF79DFD89
:101600003C48FFF789FD3C4B18703C48FFF784FDD0
:101610003B4B18703B48FFF77FFD3B4B18703B4836
:10162000FFF77AFD3A4B18703A48FFF775FD3A4BD1
:1016300018703A48FFF770FD394B18703948FFF7BA
:101640006BFD394B1870FFF761FE3848FFF764FDFA
:10165000374B18703748FFF75FFD374B1870374826
:10166000FFF75AFD364B18703648FFF755FD364BDD
:1016700018703648FFF750FD354B18703548FFF7A6
:101680004BFD354B002869D1187069E034180020F3
:10169000620E002086190020610E0020640E0020DA
:1016A00071140020DE1000207A3B00200000002092
:1016B000B51600201F180020630E0020B032002055
:1016C0002A320020C031002020290020953300203C
:1016D000A53300209D330020CC310020F6310020BE
:1016E000A2160020B28DFFFF603600202EA6FFFF5D
:1016F000A0120020B58DFFFF5E360020B68DFFFFE3
:1017000091350020B88DFFFF05350020B98DFFFF12
:10171000B41A0020C097FFFF391700201EA5FFFF55
:10172000BA170020BE97FFFF201800200AA5FFFF70
:10173000A831002087A4FFFF9F2B002084A4FFFF77
:10174000332A002086A4FFFFA72B002085A4FFFFDB
:10175000A12B0020BA8DFFFF0218002001221A7071
:101760004AF20D55002428B2FFF7D6FC00210246AC
:101770000B462046FDF764FE681C00B2FFF7CCFC68
:10178000012102460023204601340235FDF758FEB0
:10179000042CADB2E7D10E48FFF7BEFC0D4B18701C
:1017A0000D48FFF7B9FC0D4B01281A780C480CBF07
:1017B00042F020026FF345121A70FFF7ADFC094B9F
:1017C00018700948FFF7A8FCBDE8704010F0F8BE9B
:1017D0006A8DFFFF06340020A0A5FFFF984100207E
:1017E000698DFFFF5C2100202DA6FFFF034B1E210A
:1017F0001A7861F346021A70704700BF86190020FC
:10180000024B187800F00100704700BF86190020D5
:10181000014B1878C00970478619002008B5FFF7FA
:10182000F7FF38B9044B1B7813F07E0F0CBF002074
:10183000012008BD012008BD86190020F8B547F237
:101840004D242046FFF768FC2D2803DD20462D217E
:10185000FFF758FCA4F56256353E3046FFF75CFCB6
:10186000414FC0B207EBC0000579C5F30015A5B91B
:101870000DE03D4B3D4953F83500EEF793FE20B99E
:1018800030462946FFF73EFC07E00135EDB207EB95
:10189000C5031B7913F0080FEBD0013447F28D23F9
:1018A0009C42CED143F6C4242046FFF735FC2D28B8
:1018B00003DD20462D21FFF725FC013443F6C82324
:1018C0009C42F1D1012143F6E120FFF71BFC0121ED
:1018D00043F6E220FFF716FC012143F6E420FFF770
:1018E00011FC012143F6E620FFF70CFC012143F631
:1018F000E920FFF707FC012143F6E520FFF702FC92
:10190000012143F6E320FFF7FDFB012143F6EB2025
:10191000FFF7F8FB002143F6E020FFF7F3FB00217F
:1019200043F6EA20FFF7EEFB002143F6EC20FFF739
:10193000E9FB012143F6DC20FFF7E4FB002149F23B
:10194000BF70FFF7DFFB48F628500121FFF7DAFBF5
:1019500047F235342046FF21FFF7D4FB013447F22C
:101960003D339C42F6D1F8BD1404002046590308CB
:1019700010B508F00BFA0BF029FE074B4FF4167266
:101980001A80012147F24530FFF7BCFB4C20BDE82F
:10199000104000F01BB800BF783B002010B508F0E5
:1019A0001DFA0BF049FE044B002147F24530198027
:1019B000BDE81040FFF7A6BB783B0020024B18881B
:1019C000003818BF01207047783B0020542873B5B9
:1019D000044663D83D4BDB7803F02003DBB2002BD9
:1019E00072D13F2801D812F00FFA394D35F8146042
:1019F000002E69D1E10001F5DE416846553108222B
:101A0000FFF79BFB3348214611F0B1FB50B1F3B215
:101A1000072B07D03F2C05D80122B240D243D2B2C7
:101A20002D4B27E01DF806300122542B08D0562BF1
:101A300003D0532B284B1AD100E0284BB24007E0CB
:101A4000B240254BD2B2195D42EA01011955234B30
:101A5000195D0A431A55FFF7D3FE98B1204B1B7846
:101A600083B13F2C0ED81E3325F814300AE0B24063
:101A7000D243D2B2195D02EA01011955174B195D23
:101A80000A401A550136082EBCD1134B1A5D134B70
:101A90001B5D134318D125F8143015E0C10001F582
:101AA000DE41684655310822FFF747FB00231DF849
:101AB00003202D2A05D001219940074A105D0143DA
:101AC00011550133082BF2D17CBD00BFC03100207D
:101AD0008A19002070250020561E0020B11C00200D
:101AE000321700201FB501F015F910B901F026F9E1
:101AF00048B10021FF2300930B2004220B460191E3
:101B00000291FFF787FBAD220023D9B24D2909D0FE
:101B1000012A07D90D48002119540D4819540D48C0
:101B200020F8131001330132552BD2B2EDD1074BFF
:101B3000002183F85510084B08481970084B0822FB
:101B4000197005B05DF804EBEEF728BC561E0020B6
:101B5000B11C00208A190020151B0020F41A002057
:101B60008819002059B1064B0C2202FB0030437A41
:101B7000C918837A417208300BB93C3383707047BF
:101B8000BC250020072813B5044624D9124B1B5C42
:101B9000022B20D10DF107010DF1060208F04EFBDA
:101BA00058B19DF80610012010FA01F19DF8073098
:101BB0000A4AD05C0143D1540DE0083CE4B2E3088A
:101BC000012104F0070411FA04F4054A0133D15C41
:101BD00041EA0404D4541CBDE823002061320020F3
:101BE00057320020044B0C2202FB00330C3A5A728D
:101BF0009A72FFF7C7BF00BFBC25002010B504468E
